 phoneutilityG

 Timestamp is 548ff537 (Tue Dec 16 17:02:47 2014)

 Preferred load address is 00010000

 Start         Length     Name                   Class
 0001:00000000 0002f970H .text                   CODE
 0001:0002f970 00004a40H .text$yc                CODE
 0002:00000000 0001c464H .rdata                  DATA
 0002:0001c464 0000007aH .rdata$debug            DATA
 0002:0001c4e0 00000280H .xdata                  DATA
 0002:0001c760 00000050H .idata$2                DATA
 0002:0001c7b0 00000014H .idata$3                DATA
 0002:0001c7c4 0000037cH .idata$4                DATA
 0002:0001cb40 00000614H .idata$6                DATA
 0002:0001d154 00000000H .edata                  DATA
 0003:00000000 0000037cH .idata$5                DATA
 0003:0000037c 00000004H .CRT$XCA                DATA
 0003:00000380 00000004H .CRT$XCAA               DATA
 0003:00000384 00000630H .CRT$XCU                DATA
 0003:000009b4 00000004H .CRT$XCZ                DATA
 0003:000009b8 00000004H .CRT$XIA                DATA
 0003:000009bc 00000004H .CRT$XIZ                DATA
 0003:000009c0 00000004H .CRT$XPA                DATA
 0003:000009c4 00000004H .CRT$XPZ                DATA
 0003:000009c8 00000004H .CRT$XTA                DATA
 0003:000009cc 00000004H .CRT$XTZ                DATA
 0003:000009d0 0000050cH .data                   DATA
 0003:00000ee0 000061e4H .bss                    DATA
 0004:00000000 000016d0H .pdata                  DATA
 0005:00000000 000000a0H .rsrc$01                DATA
 0005:000000a0 000003e0H .rsrc$02                DATA

  Address         Publics by Value              Rva+Base       Lib:Object

 0000:00000000       ___safe_se_handler_count   00000000     <absolute>
 0000:00000000       ___safe_se_handler_table   00000000     <absolute>
 0001:00000000       ?WriteAdvVOCODER@@YAHXZ    00011000 f   advanceddlg.obj
 0001:00000110       ?ReadAdvVOCODER@@YAHXZ     00011110 f   advanceddlg.obj
 0001:0000022c       ?WriteCAIRev@@YAHXZ        0001122c f   advanceddlg.obj
 0001:000003ac       ?ReadCAIRev@@YAHXZ         000113ac f   advanceddlg.obj
 0001:000004c0       ?WriteTermSid@@YAHXZ       000114c0 f   advanceddlg.obj
 0001:000005a4       ?ReadTermSid@@YAHXZ        000115a4 f   advanceddlg.obj
 0001:000006c0       ?WriteLockCode@@YAHXZ      000116c0 f   advanceddlg.obj
 0001:000007bc       ?ReadLockCode@@YAHXZ       000117bc f   advanceddlg.obj
 0001:000008dc       ?WriteTermNid@@YAHXZ       000118dc f   advanceddlg.obj
 0001:000009c4       ?ReadTermNid@@YAHXZ        000119c4 f   advanceddlg.obj
 0001:00000ad8       ?WriteTermHome@@YAHXZ      00011ad8 f   advanceddlg.obj
 0001:00000bbc       ?ReadTermHome@@YAHXZ       00011bbc f   advanceddlg.obj
 0001:00000cd0       ?ReadScm@@YAHXZ            00011cd0 f   advanceddlg.obj
 0001:00000d1c       ?SaveDDTM@@YAHXZ           00011d1c f   advanceddlg.obj
 0001:00000e88       ?PopulateData@@YAHXZ       00011e88 f   advanceddlg.obj
 0001:00001270       ?InitializeAdvanceDlg@@YAHPAUHWND__@@@Z 00012270 f   advanceddlg.obj
 0001:0000184c       ?SaveValues@@YAHXZ         0001284c f   advanceddlg.obj
 0001:000018d8       ?InitAdvanceDlg@@YAHPAUHWND__@@@Z 000128d8 f   advanceddlg.obj
 0001:00001b0c       ?WndProcAdvance@@YAHPAUHWND__@@IIJ@Z 00012b0c f   advanceddlg.obj
 0001:00001c98       ?CreateAdvanceDlg@@YAHPAUHWND__@@@Z 00012c98 f   advanceddlg.obj
 0001:00001f48       ?UpdateMenu@@YAXH@Z        00012f48 f   authkey.obj
 0001:00002024       ?OnMenuPopup@@YAHPAUHWND__@@I@Z 00013024 f   authkey.obj
 0001:00002190       ?UpdateCancelMenu@@YAXH@Z  00013190 f   authkey.obj
 0001:00002228       ?RenderAllUIControls@@YAXPAUHWND__@@H@Z 00013228 f   authkey.obj
 0001:00002484       ?InitializeAuthKey@@YAHPAUHWND__@@@Z 00013484 f   authkey.obj
 0001:00002654       ?OnSaveAkey@@YAHPAUHWND__@@@Z 00013654 f   authkey.obj
 0001:000028d4       ?OnSaveMNAuthenticator@@YAHPAUHWND__@@@Z 000138d4 f   authkey.obj
 0001:00002cec       ?OnChangeMnAuthr@@YAXPAUHWND__@@@Z 00013cec f   authkey.obj
 0001:00002d84       ?OnChangeAkey@@YAXPAUHWND__@@@Z 00013d84 f   authkey.obj
 0001:00002e10       ?InitAuthKeyDlg@@YAHPAUHWND__@@@Z 00013e10 f   authkey.obj
 0001:000030e4       ?ProcessAuthKeyCtlChange@@YAHIJ@Z 000140e4 f   authkey.obj
 0001:000031a4       ?WndProcAuthKey@@YAHPAUHWND__@@IIJ@Z 000141a4 f   authkey.obj
 0001:000033e0       ?CreateAuthKeyDlg@@YAHPAUHWND__@@@Z 000143e0 f   authkey.obj
 0001:000036ac       ?InitializeBrowserDlg@@YAHPAUHWND__@@@Z 000146ac f   browserdlg.obj
 0001:000036d8       ?InitBrowserDlg@@YAHPAUHWND__@@@Z 000146d8 f   browserdlg.obj
 0001:000038c4       ?WndProcBrowserDlg@@YAHPAUHWND__@@IIJ@Z 000148c4 f   browserdlg.obj
 0001:00003a0c       ?CreateBrowserDlg@@YAHPAUHWND__@@@Z 00014a0c f   browserdlg.obj
 0001:00003cb4       ?ResetCounts@@YAXXZ        00014cb4 f   bwmeterdlg.obj
 0001:00003f10       ?UpdateMeters@@YAXXZ       00014f10 f   bwmeterdlg.obj
 0001:000046e0       ?InitializeBWMeterDlgClass@@YAHPAUHWND__@@@Z 000156e0 f   bwmeterdlg.obj
 0001:00004a9c       ?PollingThreadProc@@YAKPAX@Z 00015a9c f   bwmeterdlg.obj
 0001:0000534c       ?KillPollingThread@@YAXXZ  0001634c f   bwmeterdlg.obj
 0001:000053f0       ?IsInDataCall@@YAHXZ       000163f0 f   bwmeterdlg.obj
 0001:00005430       ?OnSetActive@@YAHPAUHWND__@@@Z 00016430 f   bwmeterdlg.obj
 0001:0000569c       ?OnTimer@@YAXPAUHWND__@@I@Z 0001669c f   bwmeterdlg.obj
 0001:000057e8       ?OnRxMaxSelect@@YAHPAUHWND__@@H@Z 000167e8 f   bwmeterdlg.obj
 0001:0000598c       ?OnTxMaxSelect@@YAHPAUHWND__@@H@Z 0001698c f   bwmeterdlg.obj
 0001:00005b38       ?InitBWMeterDlgClass@@YAHPAUHWND__@@@Z 00016b38 f   bwmeterdlg.obj
 0001:00005d70       ?CloseBWDialog@@YAXPAUHWND__@@@Z 00016d70 f   bwmeterdlg.obj
 0001:00005db0       ?WndProcBWMeter@@YAHPAUHWND__@@IIJ@Z 00016db0 f   bwmeterdlg.obj
 0001:00006040       ?CreateBandWidthMeterDlg@@YAHPAUHWND__@@@Z 00017040 f   bwmeterdlg.obj
 0001:0000619c       ?InitializeConfigDlg@@YAHPAUHWND__@@@Z 0001719c f   configdlg.obj
 0001:00006778       ?InitConfigDlg@@YAHPAUHWND__@@@Z 00017778 f   configdlg.obj
 0001:00006998       ?WndProcConfig@@YAHPAUHWND__@@IIJ@Z 00017998 f   configdlg.obj
 0001:00006ae0       ?CreateConfigDlg@@YAHPAUHWND__@@@Z 00017ae0 f   configdlg.obj
 0001:00006db0       ?InitializeEVDODlg@@YAHPAUHWND__@@@Z 00017db0 f   evdo.obj
 0001:000070e4       ?UpdateTechHdrInfo@@YAHXZ  000180e4 f   evdo.obj
 0001:00007fd0       ?InitEVDODlg@@YAHPAUHWND__@@@Z 00018fd0 f   evdo.obj
 0001:00008220       ?WndProcEVDODlg@@YAHPAUHWND__@@IIJ@Z 00019220 f   evdo.obj
 0001:000084c8       ?CreateEVDODlg@@YAHPAUHWND__@@@Z 000194c8 f   evdo.obj
 0001:00008784       ?UpdateFingerInfo@@YAXXZ   00019784 f   finger.obj
 0001:00008d08       ?InitializeFingerDlg@@YAHPAUHWND__@@@Z 00019d08 f   finger.obj
 0001:00009244       ?InitFinger@@YAHPAUHWND__@@@Z 0001a244 f   finger.obj
 0001:00009484       ?WndProcFinger@@YAHPAUHWND__@@IIJ@Z 0001a484 f   finger.obj
 0001:000096d0       ?CreateFingerDlg@@YAHPAUHWND__@@@Z 0001a6d0 f   finger.obj
 0001:0000997c       ?FormatLatLon@@YAXHPAG@Z   0001a97c f   gpsdatadlg.obj
 0001:00009bbc       ?TimeFromSecs@@YAXKPAGI@Z  0001abbc f   gpsdatadlg.obj
 0001:00009c48       ?OnLBSMenuPopup@@YAHPAUHWND__@@I@Z 0001ac48 f   gpsdatadlg.obj
 0001:00009cdc       ?updateLbsData@@YAHXZ      0001acdc f   gpsdatadlg.obj
 0001:00009e8c       ?ReaddataFromCtrl@@YAHXZ   0001ae8c f   gpsdatadlg.obj
 0001:00009ffc       ?ReadGpsPDdata@@YAHXZ      0001affc f   gpsdatadlg.obj
 0001:0000a130       ?PopulateLBSDataCtrls@@YAHXZ 0001b130 f   gpsdatadlg.obj
 0001:0000a2cc       ?EnableControls@@YAHH@Z    0001b2cc f   gpsdatadlg.obj
 0001:0000a354       ?InitializeGPSDataDlgClass@@YAHPAUHWND__@@@Z 0001b354 f   gpsdatadlg.obj
 0001:0000a50c       ?OnStopTrack@@YAHPAUHWND__@@@Z 0001b50c f   gpsdatadlg.obj
 0001:0000a650       ?OnStartTrack@@YAHPAUHWND__@@@Z 0001b650 f   gpsdatadlg.obj
 0001:0000a840       ?InitGpsDataDlgClass@@YAHPAUHWND__@@@Z 0001b840 f   gpsdatadlg.obj
 0001:0000aab4       ?WndProcGPSData@@YAHPAUHWND__@@IIJ@Z 0001bab4 f   gpsdatadlg.obj
 0001:0000ae08       ?CreateGpsDataDlg@@YAHPAUHWND__@@@Z 0001be08 f   gpsdatadlg.obj
 0001:0000b0b8       ?IsValidPortID@@YAHPAG@Z   0001c0b8 f   gpssettingsdlg.obj
 0001:0000b238       ?IsValidIP@@YAHPAG@Z       0001c238 f   gpssettingsdlg.obj
 0001:0000b398       ?updateLBSSetsData@@YAHXZ  0001c398 f   gpssettingsdlg.obj
 0001:0000b568       ?PopulateLBSSetsCtrls@@YAHXZ 0001c568 f   gpssettingsdlg.obj
 0001:0000b914       ?GetdataFromCtrls@@YAHXZ   0001c914 f   gpssettingsdlg.obj
 0001:0000bda4       ?ReadGpsSettings@@YAHXZ    0001cda4 f   gpssettingsdlg.obj
 0001:0000bea4       ?SaveGpsSettings@@YAHXZ    0001cea4 f   gpssettingsdlg.obj
 0001:0000c010       ?InitializeGpsSettingsDlgClass@@YAHPAUHWND__@@@Z 0001d010 f   gpssettingsdlg.obj
 0001:0000c210       ?InitGpsSettingsDlgClass@@YAHPAUHWND__@@@Z 0001d210 f   gpssettingsdlg.obj
 0001:0000c44c       ?WndProcGPSSettings@@YAHPAUHWND__@@IIJ@Z 0001d44c f   gpssettingsdlg.obj
 0001:0000c67c       ?CreateGpsSettingsDlg@@YAHPAUHWND__@@@Z 0001d67c f   gpssettingsdlg.obj
 0001:0000c928       ?UpdateGSM2GInfo@@YAHPAUHWND__@@@Z 0001d928 f   gsm2G.obj
 0001:0000c9dc       ?InitializeGSM2G@@YAHPAUHWND__@@@Z 0001d9dc f   gsm2G.obj
 0001:0000cadc       ?InitGSM2G@@YAHPAUHWND__@@@Z 0001dadc f   gsm2G.obj
 0001:0000cd18       ?WndProcGSM2G@@YAHPAUHWND__@@IIJ@Z 0001dd18 f   gsm2G.obj
 0001:0000cf10       ?CreateGSM2GDlg@@YAHPAUHWND__@@@Z 0001df10 f   gsm2G.obj
 0001:0000d108       ?DeallocateListView@@YAXPAUHWND__@@@Z 0001e108 f   gsm3G.obj
 0001:0000d200       ?ParseAndBuildDynamicList@@YAXPAUHWND__@@PAG@Z 0001e200 f   gsm3G.obj
 0001:0000d48c       ?UpdateGSM3GItemnizeInfo@@YAHPAUHWND__@@J@Z 0001e48c f   gsm3G.obj
 0001:0000d56c       ?InitializeGSM3G@@YAHPAUHWND__@@@Z 0001e56c f   gsm3G.obj
 0001:0000d618       ?InitGSM3G@@YAHPAUHWND__@@@Z 0001e618 f   gsm3G.obj
 0001:0000d820       ?WndProcGSM3G@@YAHPAUHWND__@@IIJ@Z 0001e820 f   gsm3G.obj
 0001:0000dadc       ?CreateGSM3GDlg@@YAHPAUHWND__@@@Z 0001eadc f   gsm3G.obj
 0001:0000dce0       ?InitializeGSM3GItemnize@@YAHPAUHWND__@@J@Z 0001ece0 f   gsm3G.obj
 0001:0000de2c       ?InitGSM3GItemnize@@YAHPAUHWND__@@J@Z 0001ee2c f   gsm3G.obj
 0001:0000e07c       ?WndProcGSM3GItemnize@@YAHPAUHWND__@@IIJ@Z 0001f07c f   gsm3G.obj
 0001:0000e298       ?CreateGSM3GDlgItemnize@@YAHPAUHWND__@@@Z 0001f298 f   gsm3G.obj
 0001:0000e490       ?DeallocateGSMBandListView@@YAXPAUHWND__@@@Z 0001f490 f   gsmband.obj
 0001:0000e580       ?ParseAndBuildDynamicList@@YAXPAUHWND__@@KPAUtagRILBANDINFO@@@Z 0001f580 f   gsmband.obj
 0001:0000e720       ?GetGSMBandInfo@@YAHPAUHWND__@@@Z 0001f720 f   gsmband.obj
 0001:0000e7c8       ?InitializeGSMBand@@YAHPAUHWND__@@@Z 0001f7c8 f   gsmband.obj
 0001:0000e868       ?InitGSMBand@@YAHPAUHWND__@@@Z 0001f868 f   gsmband.obj
 0001:0000ea64       ?WndProcGSMBand@@YAHPAUHWND__@@IIJ@Z 0001fa64 f   gsmband.obj
 0001:0000ed94       ?CreateGSMBandDlg@@YAHPAUHWND__@@@Z 0001fd94 f   gsmband.obj
 0001:0000ef8c       ?InitializeIOTADlg@@YAHPAUHWND__@@@Z 0001ff8c f   iota.obj
 0001:0000efb8       ?InitIOTADlg@@YAHPAUHWND__@@@Z 0001ffb8 f   iota.obj
 0001:0000f1a8       ?WndProcIOTA@@YAHPAUHWND__@@IIJ@Z 000201a8 f   iota.obj
 0001:0000f2f0       ?CreateIOTADlg@@YAHPAUHWND__@@@Z 000202f0 f   iota.obj
 0001:0000f598       ?CreateListView@@YAPAUHWND__@@PAU1@@Z 00020598 f   listview.obj
 0001:0000f6d4       ?CleanupListView@@YAXPAUHWND__@@@Z 000206d4 f   listview.obj
 0001:0000f70c       ?InitializeList@@YAXPAUHWND__@@0@Z 0002070c f   listview.obj
 0001:0000ff48       ?OnListViewNotify@@YAJPAUHWND__@@J@Z 00020f48 f   listview.obj
 0001:00010164       ?FillServiceOption@@YAXPAUHWND__@@@Z 00021164 f   loopbackdlg.obj
 0001:00010264       ?onCallHangup@@YAHPAUHWND__@@@Z 00021264 f   loopbackdlg.obj
 0001:0001035c       ?onCallEstablish@@YAHPAUHWND__@@@Z 0002135c f   loopbackdlg.obj
 0001:0001059c       ?InitializeLoopBackDlg@@YAHPAUHWND__@@@Z 0002159c f   loopbackdlg.obj
 0001:000106e0       ?CheckForCallStatus@@YAXXZ 000216e0 f   loopbackdlg.obj
 0001:00010e64       ?InitLoopBackDlg@@YAHPAUHWND__@@@Z 00021e64 f   loopbackdlg.obj
 0001:0001125c       ?OnChangeNumber@@YAHPAUHWND__@@0@Z 0002225c f   loopbackdlg.obj
 0001:000114b0       ?ProcessLoopbackCtlChange@@YAHPAUHWND__@@IJ@Z 000224b0 f   loopbackdlg.obj
 0001:00011560       ?WndProcLoopBackDlg@@YAHPAUHWND__@@IIJ@Z 00022560 f   loopbackdlg.obj
 0001:00011710       ?CreateLoopBackDlg@@YAHPAUHWND__@@@Z 00022710 f   loopbackdlg.obj
 0001:000119bc       ?CreateMainMenu@@YAHPAUHWND__@@@Z 000229bc f   mainfrm.obj
 0001:00011a94       ?InitializeTabFromIndex@@YAHPAUHWND__@@KHH@Z 00022a94 f   mainfrm.obj
 0001:000127b0       ?PrepareResourceDlg@@YAHPAUHWND__@@@Z 000237b0 f   mainfrm.obj
 0001:00012c10       ?OnCreateMainWnd@@YAHPAUHWND__@@@Z 00023c10 f   mainfrm.obj
 0001:00012ce8       ?MainWndProc@@YAJPAUHWND__@@IIJ@Z 00023ce8 f   mainfrm.obj
 0001:00013228       ?RegisterMainWnd@@YAHXZ    00024228 f   mainfrm.obj
 0001:00013324       ?CreateMainWnd@@YAHH@Z     00024324 f   mainfrm.obj
 0001:0001344c       ?SaveMSL@@YAXPAUHWND__@@@Z 0002444c f   msldlg.obj
 0001:00013a7c       ?FillAccolc@@YAXPAUHWND__@@G@Z 00024a7c f   msldlg.obj
 0001:00013b88       ?FillSlotCycle@@YAXPAUHWND__@@G@Z 00024b88 f   msldlg.obj
 0001:00013c74       ?InitializeMslDlg@@YAHPAUHWND__@@@Z 00024c74 f   msldlg.obj
 0001:00014310       ?EnablesaveMenu@@YAXXZ     00025310 f   msldlg.obj
 0001:00014464       ?OnChangeNumberMdn@@YAXPAUHWND__@@@Z 00025464 f   msldlg.obj
 0001:000144c4       ?OnChangeNumberMsid@@YAXPAUHWND__@@@Z 000254c4 f   msldlg.obj
 0001:00014530       ?OnChangeEditSid@@YAXPAUHWND__@@@Z 00025530 f   msldlg.obj
 0001:0001462c       ?OnChangeEditNid@@YAXPAUHWND__@@@Z 0002562c f   msldlg.obj
 0001:00014728       ?OnChangeEditMcc@@YAXPAUHWND__@@@Z 00025728 f   msldlg.obj
 0001:00014824       ?OnChangeEditMnc@@YAXPAUHWND__@@@Z 00025824 f   msldlg.obj
 0001:00014910       ?ProcessMSLDlgCtlChange@@YAHIJ@Z 00025910 f   msldlg.obj
 0001:00014a80       ?InitMslDlg@@YAHPAUHWND__@@@Z 00025a80 f   msldlg.obj
 0001:00014df4       ?WndProcMsl@@YAHPAUHWND__@@IIJ@Z 00025df4 f   msldlg.obj
 0001:00015030       ?CreateMslDlg@@YAHPAUHWND__@@@Z 00026030 f   msldlg.obj
 0001:00015300       ?UpdatePwrStatus@@YAHXZ    00026300 f   network.obj
 0001:00015bb4       ?InitializeNetworkDlg@@YAHPAUHWND__@@@Z 00026bb4 f   network.obj
 0001:00015edc       ?InitNetwork@@YAHPAUHWND__@@@Z 00026edc f   network.obj
 0001:00016130       ?UpdateNetworkInfo@@YAHXZ  00027130 f   network.obj
 0001:00016ecc       ?WndProcNetwork@@YAHPAUHWND__@@IIJ@Z 00027ecc f   network.obj
 0001:000170fc       ?CreateNetworkDlg@@YAHPAUHWND__@@@Z 000280fc f   network.obj
 0001:000172fc       ?SaveOTKSL@@YAXPAUHWND__@@@Z 000282fc f   otksldlg.obj
 0001:0001758c       ?EnableSaveMenu@@YAXXZ     0002858c f   otksldlg.obj
 0001:00017618       ?OnChangeNumberMdnOtksl@@YAXPAUHWND__@@@Z 00028618 f   otksldlg.obj
 0001:00017678       ?OnChangeNumberMsidotksl@@YAXPAUHWND__@@@Z 00028678 f   otksldlg.obj
 0001:000176dc       ?ProcessOTKSLCtlChange@@YAHIJ@Z 000286dc f   otksldlg.obj
 0001:000177ac       ?InitializeOtkslDlg@@YAHPAUHWND__@@@Z 000287ac f   otksldlg.obj
 0001:000179ac       ?InitOtkslDlg@@YAHPAUHWND__@@@Z 000289ac f   otksldlg.obj
 0001:00017c80       ?WndProcOtksl@@YAHPAUHWND__@@IIJ@Z 00028c80 f   otksldlg.obj
 0001:00017ea0       ?CreateOtkslDlg@@YAHPAUHWND__@@@Z 00028ea0 f   otksldlg.obj
 0001:0001814c       ?InitializePassThruDlg@@YAHPAUHWND__@@@Z 0002914c f   passthrudlg.obj
 0001:00018360       ?InitPassThruDlg@@YAHPAUHWND__@@@Z 00029360 f   passthrudlg.obj
 0001:00018660       ?OnPasstruMenuPopup@@YAHPAUHWND__@@I@Z 00029660 f   passthrudlg.obj
 0001:000186ec       ?WndProcPassThru@@YAHPAUHWND__@@IIJ@Z 000296ec f   passthrudlg.obj
 0001:00018c10       ?CreatePassThruDlg@@YAHPAUHWND__@@@Z 00029c10 f   passthrudlg.obj
 0001:00018edc       ?GetInstanceHandle@@YAPAUHINSTANCE__@@XZ 00029edc f   PhoneUtility.obj
 0001:00018efc       ?GetResourceHandle@@YAPAUHINSTANCE__@@XZ 00029efc f   PhoneUtility.obj
 0001:00018f1c       ?GetCarrier@@YAKXZ         00029f1c f   PhoneUtility.obj
 0001:00018f3c       ?GetActiveTab@@YAKXZ       00029f3c f   PhoneUtility.obj
 0001:00018f5c       ?GetMainWnd@@YAPAUHWND__@@XZ 00029f5c f   PhoneUtility.obj
 0001:00018f7c       ?SetWindowTopMost@@YAJPAUHWND__@@@Z 00029f7c f   PhoneUtility.obj
 0001:00018fa8       ?InitializeGlobalVars@@YAXXZ 00029fa8 f   PhoneUtility.obj
 0001:000190fc       WinMain                    0002a0fc f   PhoneUtility.obj
 0001:00019824       ?ParseParam@@YAKXZ         0002a824 f   PhoneUtility.obj
 0001:00019a4c       ?CheckPhoneUtilityCanrun@@YAHXZ 0002aa4c f   PhoneUtility.obj
 0001:00019b44       ?ProcessSwapMenuBar@@YAHPAUHWND__@@0H@Z 0002ab44 f   PhoneUtility.obj
 0001:00019ba8       ?GetStatus@@YAHXZ          0002aba8 f   PhoneUtility.obj
 0001:00019bfc       ?SpcValidation@@YAHPAUHWND__@@@Z 0002abfc f   PhoneUtility.obj
 0001:00019da8       ?ValidateSpecialPassword@@YAHXZ 0002ada8 f   PhoneUtility.obj
 0001:00019dc8       ?DebugModeStart@@YAHXZ     0002adc8 f   PhoneUtility.obj
 0001:00019e50       ?DebugModeStop@@YAHXZ      0002ae50 f   PhoneUtility.obj
 0001:00019ed8       ?EnableTechHdr@@YAHH@Z     0002aed8 f   PhoneUtility.obj
 0001:00019f38       ?GetTechHdrInfo@@YAHXZ     0002af38 f   PhoneUtility.obj
 0001:0001a664       ?CheckDebugStatus@@YAHXZ   0002b664 f   PhoneUtility.obj
 0001:0001a6e4       ?GetDebugInfo@@YAHXZ       0002b6e4 f   PhoneUtility.obj
 0001:0001ad20       ?GeoSecToDegMinSec@@YAXJAAJAAH1@Z 0002bd20 f   PhoneUtility.obj
 0001:0001ae0c       ?InitializeRTNDlg@@YAHPAUHWND__@@@Z 0002be0c f   rtndlg.obj
 0001:0001af98       ?OnInitRTNDialog@@YAHPAUHWND__@@@Z 0002bf98 f   rtndlg.obj
 0001:0001b1b8       ?WndProcRTN@@YAHPAUHWND__@@IIJ@Z 0002c1b8 f   rtndlg.obj
 0001:0001b650       ?CreateRTNDlg@@YAHPAUHWND__@@@Z 0002c650 f   rtndlg.obj
 0001:0001b91c       ?ReadQcMIP@@YAHXZ          0002c91c f   simpleipdlg.obj
 0001:0001baa8       ?InitializeSimpleIPDlg@@YAHPAUHWND__@@@Z 0002caa8 f   simpleipdlg.obj
 0001:0001be70       ?SaveSimpleIPData@@YAHPAUHWND__@@@Z 0002ce70 f   simpleipdlg.obj
 0001:0001c3f8       ?InitSimpleIPDlg@@YAHPAUHWND__@@@Z 0002d3f8 f   simpleipdlg.obj
 0001:0001c630       ?WndProcSimpleIP@@YAHPAUHWND__@@IIJ@Z 0002d630 f   simpleipdlg.obj
 0001:0001c7a4       ?CreateSimpleIPDlg@@YAHPAUHWND__@@@Z 0002d7a4 f   simpleipdlg.obj
 0001:0001ca50       ?InitializeSipDlg@@YAHPAUHWND__@@@Z 0002da50 f   sipdlg.obj
 0001:0001ca7c       ?InitSipDlg@@YAHPAUHWND__@@@Z 0002da7c f   sipdlg.obj
 0001:0001cc74       ?WndProcSipDlg@@YAHPAUHWND__@@IIJ@Z 0002dc74 f   sipdlg.obj
 0001:0001cdbc       ?CreateSipDlg@@YAHPAUHWND__@@@Z 0002ddbc f   sipdlg.obj
 0001:0001d064       ?InitializeSPCValidation@@YAHPAUHWND__@@@Z 0002e064 f   spcvalidation.obj
 0001:0001d0c8       ?InitSPCValidation@@YAHPAUHWND__@@@Z 0002e0c8 f   spcvalidation.obj
 0001:0001d318       ?OnChangeSPC@@YAXPAUHWND__@@@Z 0002e318 f   spcvalidation.obj
 0001:0001d3c0       ?ProcessCtlChange@@YAHIJ@Z 0002e3c0 f   spcvalidation.obj
 0001:0001d464       ?WndProcSPCValidation@@YAHPAUHWND__@@IIJ@Z 0002e464 f   spcvalidation.obj
 0001:0001d77c       ?CreateSPCValidation@@YAHPAUHWND__@@@Z 0002e77c f   spcvalidation.obj
 0001:0001da50       ?FillComboCtrls@@YAXPAUHWND__@@@Z 0002ea50 f   systemdlg.obj
 0001:0001e09c       ?GetoModemValues@@YAHPAUHWND__@@@Z 0002f09c f   systemdlg.obj
 0001:0001e180       ?InitializeSystemDlg@@YAHPAUHWND__@@@Z 0002f180 f   systemdlg.obj
 0001:0001e210       ?SaveSelectiontoModem@@YAHPAUHWND__@@@Z 0002f210 f   systemdlg.obj
 0001:0001e658       ?InitSystemDlg@@YAHPAUHWND__@@@Z 0002f658 f   systemdlg.obj
 0001:0001e848       ?WndProcSystemDlg@@YAHPAUHWND__@@IIJ@Z 0002f848 f   systemdlg.obj
 0001:0001eac8       ?CreateSystemDlg@@YAHPAUHWND__@@@Z 0002fac8 f   systemdlg.obj
 0001:0001ed74       ?PopulatePDPListcombo@@YAHPAUHWND__@@@Z 0002fd74 f   usernamedlg.obj
 0001:0001eec8       ?GetPDPList@@YAHPAUHWND__@@@Z 0002fec8 f   usernamedlg.obj
 0001:0001ef98       ?PopulateTheProfile@@YAXPAUHWND__@@@Z 0002ff98 f   usernamedlg.obj
 0001:0001f230       ?GetMipGenProfile@@YAHPAUHWND__@@H@Z 00030230 f   usernamedlg.obj
 0001:0001f32c       ?InitializeUsernameDlg@@YAHPAUHWND__@@@Z 0003032c f   usernamedlg.obj
 0001:0001f59c       ?ConverttoHEX@@YAHPAUHWND__@@@Z 0003059c f   usernamedlg.obj
 0001:0001ffa4       ?UpdatePDPProfile@@YAHPAUHWND__@@@Z 00030fa4 f   usernamedlg.obj
 0001:00020620       ?InitUsernameDlg@@YAHPAUHWND__@@@Z 00031620 f   usernamedlg.obj
 0001:00020814       ?WndProcUsername@@YAHPAUHWND__@@IIJ@Z 00031814 f   usernamedlg.obj
 0001:00020a24       ?CreateUsernameDlg@@YAHPAUHWND__@@@Z 00031a24 f   usernamedlg.obj
 0001:00020cd4       IsDlgButtonChecked         00031cd4 f i usernamedlg.obj
 0001:00020d18       CheckDlgButton             00031d18 f i usernamedlg.obj
 0001:00020d64       ?InitializeVersionInfoDlg@@YAHPAUHWND__@@AAUtagRILVERNOINFO@@@Z 00031d64 f   versioninfo.obj
 0001:00021c68       ?InitVersionInfoDlg@@YAHPAUHWND__@@@Z 00032c68 f   versioninfo.obj
 0001:00021ec8       ?WndProcVersionInfoDlg@@YAHPAUHWND__@@IIJ@Z 00032ec8 f   versioninfo.obj
 0001:000220b0       ?CreateVersionInfoDlg@@YAHPAUHWND__@@@Z 000330b0 f   versioninfo.obj
 0001:0002235c       ?ReadVOCODER@@YAHXZ        0003335c f   vocoderdlg.obj
 0001:000224c0       ?UpdatedListItem@@YAXPAUHWND__@@G@Z 000334c0 f   vocoderdlg.obj
 0001:00022698       ?InitializeVocoderDlg@@YAHPAUHWND__@@@Z 00033698 f   vocoderdlg.obj
 0001:00022a18       ?InitVocoderDlg@@YAHPAUHWND__@@@Z 00033a18 f   vocoderdlg.obj
 0001:00022c5c       ?SaveVocoder@@YAHPAUHWND__@@@Z 00033c5c f   vocoderdlg.obj
 0001:00023094       ?WndProcVocoderDlg@@YAHPAUHWND__@@IIJ@Z 00034094 f   vocoderdlg.obj
 0001:00023250       ?CreateVocoderDlg@@YAHPAUHWND__@@@Z 00034250 f   vocoderdlg.obj
 0001:0002351c       SendMessageW               0003451c f   coredll:COREDLL.dll
 0001:0002352c       ??3@YAXPAX@Z               0003452c f   coredll:COREDLL.dll
 0001:0002353c       _wcsicmp                   0003453c f   coredll:COREDLL.dll
 0001:0002354c       LoadStringW                0003454c f   coredll:COREDLL.dll
 0001:0002355c       GetWindowTextW             0003455c f   coredll:COREDLL.dll
 0001:0002356c       wcsncpy                    0003456c f   coredll:COREDLL.dll
 0001:0002357c       memset                     0003457c f   coredll:COREDLL.dll
 0001:0002358c       wcscpy                     0003458c f   coredll:COREDLL.dll
 0001:0002359c       Sleep                      0003459c f   coredll:COREDLL.dll
 0001:000235ac       swprintf                   000345ac f   coredll:COREDLL.dll
 0001:000235bc       SetWindowTextW             000345bc f   coredll:COREDLL.dll
 0001:000235cc       GetDlgItem                 000345cc f   coredll:COREDLL.dll
 0001:000235dc       SetDlgItemInt              000345dc f   coredll:COREDLL.dll
 0001:000235ec       SetDlgItemTextW            000345ec f   coredll:COREDLL.dll
 0001:000235fc       EndDialog                  000345fc f   coredll:COREDLL.dll
 0001:0002360c       MessageBoxW                0003460c f   coredll:COREDLL.dll
 0001:0002361c       SetFocus                   0003461c f   coredll:COREDLL.dll
 0001:0002362c       DialogBoxIndirectParamW    0003462c f   coredll:COREDLL.dll
 0001:0002363c       LoadResource               0003463c f   coredll:COREDLL.dll
 0001:0002364c       FindResourceW              0003464c f   coredll:COREDLL.dll
 0001:0002365c       GetLastError               0003465c f   coredll:COREDLL.dll
 0001:0002366c       RegisterClassW             0003466c f   coredll:COREDLL.dll
 0001:0002367c       GetStockObject             0003467c f   coredll:COREDLL.dll
 0001:0002368c       RegisterWindowMessageW     0003468c f   coredll:COREDLL.dll
 0001:0002369c       EnableMenuItem             0003469c f   coredll:COREDLL.dll
 0001:000236ac       wcslen                     000346ac f   coredll:COREDLL.dll
 0001:000236bc       EnableWindow               000346bc f   coredll:COREDLL.dll
 0001:000236cc       ShowWindow                 000346cc f   coredll:COREDLL.dll
 0001:000236dc       _wtol                      000346dc f   coredll:COREDLL.dll
 0001:000236ec       PostMessageW               000346ec f   coredll:COREDLL.dll
 0001:000236fc       PostQuitMessage            000346fc f   coredll:COREDLL.dll
 0001:0002370c       __rt_sdiv                  0003470c f   coredll:COREDLL.dll
 0001:0002371c       __utos                     0003471c f   coredll:COREDLL.dll
 0001:0002372c       __gts                      0003472c f   coredll:COREDLL.dll
 0001:0002373c       __ges                      0003473c f   coredll:COREDLL.dll
 0001:0002374c       __les                      0003474c f   coredll:COREDLL.dll
 0001:0002375c       __muls                     0003475c f   coredll:COREDLL.dll
 0001:0002376c       __eqs                      0003476c f   coredll:COREDLL.dll
 0001:0002377c       __itos                     0003477c f   coredll:COREDLL.dll
 0001:0002378c       __stou                     0003478c f   coredll:COREDLL.dll
 0001:0002379c       __rt_udiv                  0003479c f   coredll:COREDLL.dll
 0001:000237ac       __dtos                     000347ac f   coredll:COREDLL.dll
 0001:000237bc       __utod                     000347bc f   coredll:COREDLL.dll
 0001:000237cc       __muld                     000347cc f   coredll:COREDLL.dll
 0001:000237dc       __dtou                     000347dc f   coredll:COREDLL.dll
 0001:000237ec       __stod                     000347ec f   coredll:COREDLL.dll
 0001:000237fc       TerminateThread            000347fc f   coredll:COREDLL.dll
 0001:0002380c       WaitForSingleObject        0003480c f   coredll:COREDLL.dll
 0001:0002381c       CreateThread               0003481c f   coredll:COREDLL.dll
 0001:0002382c       KillTimer                  0003482c f   coredll:COREDLL.dll
 0001:0002383c       SetTimer                   0003483c f   coredll:COREDLL.dll
 0001:0002384c       MultiByteToWideChar        0003484c f   coredll:COREDLL.dll
 0001:0002385c       SetWindowPos               0003485c f   coredll:COREDLL.dll
 0001:0002386c       GetClientRect              0003486c f   coredll:COREDLL.dll
 0001:0002387c       LeaveCriticalSection       0003487c f   coredll:COREDLL.dll
 0001:0002388c       memcpy                     0003488c f   coredll:COREDLL.dll
 0001:0002389c       EnterCriticalSection       0003489c f   coredll:COREDLL.dll
 0001:000238ac       __divd                     000348ac f   coredll:COREDLL.dll
 0001:000238bc       DeleteCriticalSection      000348bc f   coredll:COREDLL.dll
 0001:000238cc       InitializeCriticalSection  000348cc f   coredll:COREDLL.dll
 0001:000238dc       __itod                     000348dc f   coredll:COREDLL.dll
 0001:000238ec       __ltd                      000348ec f   coredll:COREDLL.dll
 0001:000238fc       __negd                     000348fc f   coredll:COREDLL.dll
 0001:0002390c       __dtoi                     0003490c f   coredll:COREDLL.dll
 0001:0002391c       __subd                     0003491c f   coredll:COREDLL.dll
 0001:0002392c       free                       0003492c f   coredll:COREDLL.dll
 0001:0002393c       strlen                     0003493c f   coredll:COREDLL.dll
 0001:0002394c       wcstombs                   0003494c f   coredll:COREDLL.dll
 0001:0002395c       malloc                     0003495c f   coredll:COREDLL.dll
 0001:0002396c       sscanf                     0003496c f   coredll:COREDLL.dll
 0001:0002397c       HideCaret                  0003497c f   coredll:COREDLL.dll
 0001:0002398c       GetWindowLongW             0003498c f   coredll:COREDLL.dll
 0001:0002399c       ??2@YAPAXI@Z               0003499c f   coredll:COREDLL.dll
 0001:000239ac       SetWindowLongW             000349ac f   coredll:COREDLL.dll
 0001:000239bc       GetParent                  000349bc f   coredll:COREDLL.dll
 0001:000239cc       CreateWindowExW            000349cc f   coredll:COREDLL.dll
 0001:000239dc       DestroyWindow              000349dc f   coredll:COREDLL.dll
 0001:000239ec       IsWindow                   000349ec f   coredll:COREDLL.dll
 0001:000239fc       wcscmp                     000349fc f   coredll:COREDLL.dll
 0001:00023a0c       wcscat                     00034a0c f   coredll:COREDLL.dll
 0001:00023a1c       MessageBeep                00034a1c f   coredll:COREDLL.dll
 0001:00023a2c       iswctype                   00034a2c f   coredll:COREDLL.dll
 0001:00023a3c       OutputDebugStringW         00034a3c f   coredll:COREDLL.dll
 0001:00023a4c       DefWindowProcW             00034a4c f   coredll:COREDLL.dll
 0001:00023a5c       UpdateWindow               00034a5c f   coredll:COREDLL.dll
 0001:00023a6c       GetWindowTextLengthW       00034a6c f   coredll:COREDLL.dll
 0001:00023a7c       abs                        00034a7c f   coredll:COREDLL.dll
 0001:00023a8c       __addd                     00034a8c f   coredll:COREDLL.dll
 0001:00023a9c       LoadBitmapW                00034a9c f   coredll:COREDLL.dll
 0001:00023aac       NKDbgPrintfW               00034aac f   coredll:COREDLL.dll
 0001:00023abc       CloseHandle                00034abc f   coredll:COREDLL.dll
 0001:00023acc       SetForegroundWindow        00034acc f   coredll:COREDLL.dll
 0001:00023adc       FindWindowW                00034adc f   coredll:COREDLL.dll
 0001:00023aec       DispatchMessageW           00034aec f   coredll:COREDLL.dll
 0001:00023afc       TranslateMessage           00034afc f   coredll:COREDLL.dll
 0001:00023b0c       GetMessageW                00034b0c f   coredll:COREDLL.dll
 0001:00023b1c       CreateMutexW               00034b1c f   coredll:COREDLL.dll
 0001:00023b2c       LoadLibraryW               00034b2c f   coredll:COREDLL.dll
 0001:00023b3c       _wcsupr                    00034b3c f   coredll:COREDLL.dll
 0001:00023b4c       _isctype                   00034b4c f   coredll:COREDLL.dll
 0001:00023b5c       SendDlgItemMessageW        00034b5c f   coredll:COREDLL.dll
 0001:00023b6c       _wtoll                     00034b6c f   coredll:COREDLL.dll
 0001:00023b7c       wsprintfW                  00034b7c f   coredll:COREDLL.dll
 0001:00023b8c       SetActiveWindow            00034b8c f   coredll:COREDLL.dll
 0001:00023b9c       SHInitDialog               00034b9c f   aygshell:AYGSHELL.dll
 0001:00023bac       SHCreateMenuBar            00034bac f   aygshell:AYGSHELL.dll
 0001:00023bbc       ?LogC@@YAXPBGZZ            00034bbc f   sw_utilityG:sw_utilityG.dll
 0001:00023bcc       ?LogStoreFileLine@@YAXPAGH@Z 00034bcc f   sw_utilityG:sw_utilityG.dll
 0001:00023bdc       WriteNv                    00034bdc f   sw_utilityG:sw_utilityG.dll
 0001:00023bec       ?SetNormalCursor@@YAXXZ    00034bec f   sw_utilityG:sw_utilityG.dll
 0001:00023bfc       ReadNv                     00034bfc f   sw_utilityG:sw_utilityG.dll
 0001:00023c0c       ?SetWaitCursor@@YAXXZ      00034c0c f   sw_utilityG:sw_utilityG.dll
 0001:00023c1c       SetEquipmentState          00034c1c f   sw_utilityG:sw_utilityG.dll
 0001:00023c2c       GetAdvancedMenuInfo        00034c2c f   sw_utilityG:sw_utilityG.dll
 0001:00023c3c       ?SetLimitText@@YAJPAUHWND__@@H@Z 00034c3c f   sw_utilityG:sw_utilityG.dll
 0001:00023c4c       SaveAkey                   00034c4c f   sw_utilityG:sw_utilityG.dll
 0001:00023c5c       ?WriteLog@@YAXKPBGZZ       00034c5c f   sw_utilityG:sw_utilityG.dll
 0001:00023c6c       GetByteCounter             00034c6c f   sw_utilityG:sw_utilityG.dll
 0001:00023c7c       ?InWideMode@@YAHXZ         00034c7c f   sw_utilityG:sw_utilityG.dll
 0001:00023c8c       GetRilPDData               00034c8c f   sw_utilityG:sw_utilityG.dll
 0001:00023c9c       ReadPDSMPAData             00034c9c f   sw_utilityG:sw_utilityG.dll
 0001:00023cac       EndLBTrackSession          00034cac f   sw_utilityG:sw_utilityG.dll
 0001:00023cbc       StartLBTrackSession        00034cbc f   sw_utilityG:sw_utilityG.dll
 0001:00023ccc       StartPDSMDldNotifstatus    00034ccc f   sw_utilityG:sw_utilityG.dll
 0001:00023cdc       StartPDSMLocNotifstatus    00034cdc f   sw_utilityG:sw_utilityG.dll
 0001:00023cec       StopPDSMDldNotifstatus     00034cec f   sw_utilityG:sw_utilityG.dll
 0001:00023cfc       StopPDSMLocNotifstatus     00034cfc f   sw_utilityG:sw_utilityG.dll
 0001:00023d0c       ?DWORD2IP@@YAPBGK@Z        00034d0c f   sw_utilityG:sw_utilityG.dll
 0001:00023d1c       ?IP2DWORD@@YAKPBG@Z        00034d1c f   sw_utilityG:sw_utilityG.dll
 0001:00023d2c       GetRilPAParam              00034d2c f   sw_utilityG:sw_utilityG.dll
 0001:00023d3c       ReadPDSMPAParam            00034d3c f   sw_utilityG:sw_utilityG.dll
 0001:00023d4c       SetPDSMPAParam             00034d4c f   sw_utilityG:sw_utilityG.dll
 0001:00023d5c       GetGSMInfo                 00034d5c f   sw_utilityG:sw_utilityG.dll
 0001:00023d6c       ?RelayoutDialog@@YAHPAUHINSTANCE__@@PAUHWND__@@PBG@Z 00034d6c f   sw_utilityG:sw_utilityG.dll
 0001:00023d7c       GetItemnizedUMTSInfo       00034d7c f   sw_utilityG:sw_utilityG.dll
 0001:00023d8c       GetCurrentGSMBandAndList   00034d8c f   sw_utilityG:sw_utilityG.dll
 0001:00023d9c       SelectGSMBand              00034d9c f   sw_utilityG:sw_utilityG.dll
 0001:00023dac       ?GetProductFeatures@@YAHAAK@Z 00034dac f   sw_utilityG:sw_utilityG.dll
 0001:00023dbc       HangUp                     00034dbc f   sw_utilityG:sw_utilityG.dll
 0001:00023dcc       DialEx                     00034dcc f   sw_utilityG:sw_utilityG.dll
 0001:00023ddc       ?LogW@@YAXPBGZZ            00034ddc f   sw_utilityG:sw_utilityG.dll
 0001:00023dec       SetProvisionInfo           00034dec f   sw_utilityG:sw_utilityG.dll
 0001:00023dfc       GetProvisionInfo           00034dfc f   sw_utilityG:sw_utilityG.dll
 0001:00023e0c       GetMDNLengthSupported      00034e0c f   sw_utilityG:sw_utilityG.dll
 0001:00023e1c       GetCallstate               00034e1c f   sw_utilityG:sw_utilityG.dll
 0001:00023e2c       GetProvisionState          00034e2c f   sw_utilityG:sw_utilityG.dll
 0001:00023e3c       GetDMMode                  00034e3c f   sw_utilityG:sw_utilityG.dll
 0001:00023e4c       GetPTMode                  00034e4c f   sw_utilityG:sw_utilityG.dll
 0001:00023e5c       StopPTMode                 00034e5c f   sw_utilityG:sw_utilityG.dll
 0001:00023e6c       StopDMMode                 00034e6c f   sw_utilityG:sw_utilityG.dll
 0001:00023e7c       StartPTMode                00034e7c f   sw_utilityG:sw_utilityG.dll
 0001:00023e8c       StartDMMode                00034e8c f   sw_utilityG:sw_utilityG.dll
 0001:00023e9c       ?GetResolution@@YAHXZ      00034e9c f   sw_utilityG:sw_utilityG.dll
 0001:00023eac       ?GetCarrierIndex@@YAKXZ    00034eac f   sw_utilityG:sw_utilityG.dll
 0001:00023ebc       ?InitLog@@YAXPAUHINSTANCE__@@@Z 00034ebc f   sw_utilityG:sw_utilityG.dll
 0001:00023ecc       GetRilStatus               00034ecc f   sw_utilityG:sw_utilityG.dll
 0001:00023edc       ValidateSpc                00034edc f   sw_utilityG:sw_utilityG.dll
 0001:00023eec       StartDebugMode             00034eec f   sw_utilityG:sw_utilityG.dll
 0001:00023efc       StopDebugMode              00034efc f   sw_utilityG:sw_utilityG.dll
 0001:00023f0c       EnableTechHdrNotifications 00034f0c f   sw_utilityG:sw_utilityG.dll
 0001:00023f1c       GetRilDebugInfo            00034f1c f   sw_utilityG:sw_utilityG.dll
 0001:00023f2c       InitiateHostBoot           00034f2c f   sw_utilityG:sw_utilityG.dll
 0001:00023f3c       RtnReset                   00034f3c f   sw_utilityG:sw_utilityG.dll
 0001:00023f4c       GetSIPNaiPassword          00034f4c f   sw_utilityG:sw_utilityG.dll
 0001:00023f5c       SetSIPNaiPassword          00034f5c f   sw_utilityG:sw_utilityG.dll
 0001:00023f6c       ModGetHDRHybrPrefMode      00034f6c f   sw_utilityG:sw_utilityG.dll
 0001:00023f7c       ModGetSysPrefMode          00034f7c f   sw_utilityG:sw_utilityG.dll
 0001:00023f8c       ModGetRoamingMode          00034f8c f   sw_utilityG:sw_utilityG.dll
 0001:00023f9c       ModSetRoamingMode          00034f9c f   sw_utilityG:sw_utilityG.dll
 0001:00023fac       ModSetSysPrefMode          00034fac f   sw_utilityG:sw_utilityG.dll
 0001:00023fbc       ModSetHDRHybrPrefMode      00034fbc f   sw_utilityG:sw_utilityG.dll
 0001:00023fcc       GetDsMipList               00034fcc f   sw_utilityG:sw_utilityG.dll
 0001:00023fdc       GetDsMipProfile            00034fdc f   sw_utilityG:sw_utilityG.dll
 0001:00023fec       ?THtoT@@YAXPAG0H@Z         00034fec f   sw_utilityG:sw_utilityG.dll
 0001:00023ffc       ?DisplayRawData@@YAXIPAEHPBG@Z 00034ffc f   sw_utilityG:sw_utilityG.dll
 0001:0002400c       ?TtoTH@@YAXPAG0H@Z         0003500c f   sw_utilityG:sw_utilityG.dll
 0001:0002401c       SetHdrNaiPassword          0003501c f   sw_utilityG:sw_utilityG.dll
 0001:0002402c       SetDsMipProfile            0003502c f   sw_utilityG:sw_utilityG.dll
 0001:0002403c       GetVersionInfo             0003503c f   sw_utilityG:sw_utilityG.dll
 0001:0002404c       SetDdtmPreference          0003504c f   GobiApi:GobiApi.dll
 0001:0002405c       GetSysInfo                 0003505c f   GobiApi:GobiApi.dll
 0001:0002406c       GetModelID                 0003506c f   GobiApi:GobiApi.dll
 0001:0002407c       GetFirmwareRevisions       0003507c f   GobiApi:GobiApi.dll
 0001:0002408c       GetHardwareRevision        0003508c f   GobiApi:GobiApi.dll
 0001:0002409c       GetPRLVersion              0003509c f   GobiApi:GobiApi.dll
 0001:000240ac       QCWWANConnect              000350ac f   GobiApi:GobiApi.dll
 0001:000240bc       SwiGetCdmaDominantPn       000350bc f   GobiApi:GobiApi.dll
 0001:000240cc       GetErrRate                 000350cc f   GobiApi:GobiApi.dll
 0001:000240dc       SwiGetSignalStrengthInfo   000350dc f   GobiApi:GobiApi.dll
 0001:000240ec       GetANAAAAuthenticationStatus 000350ec f   GobiApi:GobiApi.dll
 0001:000240fc       SwiGetHrpdStats            000350fc f   GobiApi:GobiApi.dll
 0001:0002410c       GetHdrColorCode            0003510c f   GobiApi:GobiApi.dll
 0001:0002411c       GetRFInfo                  0003511c f   GobiApi:GobiApi.dll
 0001:0002412c       GetTxRxInfo                0003512c f   GobiApi:GobiApi.dll
 0001:0002413c       GetConfig                  0003513c f   GobiApi:GobiApi.dll
 0001:0002414c       SetConfig                  0003514c f   GobiApi:GobiApi.dll
 0001:00024164       WinMainCRTStartup          00035164 f   corelibc:pegwmain.obj
 0001:000241d8       __security_check_cookie    000351d8     corelibc:armsecgs.obj
 0001:000241ec       __gsfailure                000351ec     corelibc:armsecgs.obj
 0001:00024230       GetCurrentProcess          00035230 f i corelibc:crt0dat.obj
 0001:0002426c       _cinit                     0003526c f   corelibc:crt0dat.obj
 0001:000243dc       exit                       000353dc f   corelibc:crt0dat.obj
 0001:000243f4       _exit                      000353f4 f   corelibc:crt0dat.obj
 0001:0002440c       _cexit                     0003540c f   corelibc:crt0dat.obj
 0001:00024428       _c_exit                    00035428 f   corelibc:crt0dat.obj
 0001:00024474       __security_init_cookie     00035474 f   corelibc:seccinit.obj
 0001:000244c4       __GSHandlerCheckCommon     000354c4 f   LIBCMTD:gshandler.obj
 0001:0002450c       __GSHandlerCheck           0003550c f   LIBCMTD:gshandler.obj
 0001:0002453c       _wcsftime_l                0003553c f   LIBCMTD:wcsftime.obj
 0001:00024a10       wcsftime                   00035a10 f   LIBCMTD:wcsftime.obj
 0001:00024a5c       _localtime64_s             00035a5c f   LIBCMTD:loctim64.obj
 0001:000253b4       _invoke_watson_if_error    000363b4 f i LIBCMTD:loctim64.obj
 0001:00025408       _Getdays_l                 00036408 f   LIBCMTD:strftime.obj
 0001:000256c8       _Getdays                   000366c8 f   LIBCMTD:strftime.obj
 0001:00025700       _Getmonths_l               00036700 f   LIBCMTD:strftime.obj
 0001:000259cc       _Getmonths                 000369cc f   LIBCMTD:strftime.obj
 0001:00025a04       _Gettnames_l               00036a04 f   LIBCMTD:strftime.obj
 0001:0002630c       _Gettnames                 0003730c f   LIBCMTD:strftime.obj
 0001:00026344       _Strftime_l                00037344 f   LIBCMTD:strftime.obj
 0001:00029858       _invalid_parameter         0003a858 f   LIBCMTD:invarginternal.obj
 0001:000298a4       _CrtSetReportHookT2        0003a8a4 f   LIBCMTD:dbgrpt.obj
 0001:00029d70       _CrtDbgReportW             0003ad70 f   LIBCMTD:dbgrpt.obj
 0001:00029de8       _CrtDbgReportTV            0003ade8 f i LIBCMTD:dbgrpt.obj
 0001:00029e44       __crtMessageWindowW        0003ae44 f   LIBCMTD:dbgrpt.obj
 0001:0002a524       __tzset                    0003b524 f   LIBCMTD:tzset.obj
 0001:0002a5bc       _tzset                     0003b5bc f   LIBCMTD:tzset.obj
 0001:0002aa08       _set_daylight              0003ba08 f i LIBCMTD:tzset.obj
 0001:0002aa44       _set_dstbias               0003ba44 f i LIBCMTD:tzset.obj
 0001:0002aa80       _set_timezone              0003ba80 f i LIBCMTD:tzset.obj
 0001:0002aac4       _isindst                   0003bac4 f   LIBCMTD:tzset.obj
 0001:0002b630       _gmtime64_s                0003c630 f   LIBCMTD:gmtime64.obj
 0001:0002be54       _get_daylight              0003ce54 f   LIBCMTD:timeset.obj
 0001:0002bf4c       _get_dstbias               0003cf4c f   LIBCMTD:timeset.obj
 0001:0002c044       _get_timezone              0003d044 f   LIBCMTD:timeset.obj
 0001:0002c13c       __daylight                 0003d13c f   LIBCMTD:timeset.obj
 0001:0002c158       __dstbias                  0003d158 f   LIBCMTD:timeset.obj
 0001:0002c174       __timezone                 0003d174 f   LIBCMTD:timeset.obj
 0001:0002c190       __tzname                   0003d190 f   LIBCMTD:timeset.obj
 0001:0002c1ac       _invoke_watson             0003d1ac f   LIBCMTD:invarg.obj
 0001:0002c1e0       strcpy_s                   0003d1e0 f   LIBCMTD:strcpy_s.obj
 0001:0002c634       _mtinitlocks               0003d634 f   LIBCMTD:mlock.obj
 0001:0002c74c       _mtdeletelocks             0003d74c f   LIBCMTD:mlock.obj
 0001:0002c8d0       _mtinitlocknum             0003d8d0 f   LIBCMTD:mlock.obj
 0001:0002ca38       _lock                      0003da38 f   LIBCMTD:mlock.obj
 0001:0002cb34       _unlock                    0003db34 f   LIBCMTD:mlock.obj
 0001:0002cb74       _lockerr_exit              0003db74 f   LIBCMTD:mlock.obj
 0001:0002cb9c       _CrtDbgBreak               0003db9c f   LIBCMTD:dbgrptt.obj
 0001:0002cba4       _CrtSetReportMode          0003dba4 f   LIBCMTD:dbgrptt.obj
 0001:0002cdcc       _CrtSetReportFile          0003ddcc f   LIBCMTD:dbgrptt.obj
 0001:0002cf68       _CrtSetReportHook          0003df68 f   LIBCMTD:dbgrptt.obj
 0001:0002cfac       _CrtGetReportHook          0003dfac f   LIBCMTD:dbgrptt.obj
 0001:0002cfd4       _VCrtDbgReportW            0003dfd4 f   LIBCMTD:dbgrptt.obj
 0001:0002db8c       __crtMessageBoxW           0003eb8c f   LIBCMTD:crtmbox.obj
 0001:0002ddf0       wcsncpy_s                  0003edf0 f   LIBCMTD:wcsncpy_s.obj
 0001:0002e3f0       wcscpy_s                   0003f3f0 f   LIBCMTD:wcscpy_s.obj
 0001:0002e864       _initp_misc_initcrit       0003f864 f   LIBCMTD:initcrit.obj
 0001:0002e890       __crtInitCritSecAndSpinCount 0003f890 f   LIBCMTD:initcrit.obj
 0001:0002e9c0       _amsg_exit                 0003f9c0 f   LIBCMTD:crt0dat.obj
 0001:0002e9ec       __crtExitProcess           0003f9ec f   LIBCMTD:crt0dat.obj
 0001:0002ea34       wcscat_s                   0003fa34 f   LIBCMTD:wcscat_s.obj
 0001:0002f018       _itow_s                    00040018 f   LIBCMTD:xtows.obj
 0001:0002f6a4       _ltow_s                    000406a4 f   LIBCMTD:xtows.obj
 0001:0002f724       _ultow_s                   00040724 f   LIBCMTD:xtows.obj
 0001:0002f778       _encode_pointer            00040778 f   LIBCMTD:tidtable.obj
 0001:0002f7a0       _encoded_null              000407a0 f   LIBCMTD:tidtable.obj
 0001:0002f7d8       _decode_pointer            000407d8 f   LIBCMTD:tidtable.obj
 0001:0002f800       _XcptFilter                00040800 f   coredll:COREDLL.dll
 0001:0002f810       __C_specific_handler       00040810 f   coredll:COREDLL.dll
 0001:0002f820       __report_gsfailure         00040820 f   coredll:COREDLL.dll
 0001:0002f830       LocalFree                  00040830 f   coredll:COREDLL.dll
 0001:0002f840       __security_gen_cookie      00040840 f   coredll:COREDLL.dll
 0001:0002f850       mbstowcs                   00040850 f   coredll:COREDLL.dll
 0001:0002f860       __rt_sdiv64by64            00040860 f   coredll:COREDLL.dll
 0001:0002f870       __rt_srem64by64            00040870 f   coredll:COREDLL.dll
 0001:0002f880       _stricmp                   00040880 f   coredll:COREDLL.dll
 0001:0002f890       GetTimeFormatW             00040890 f   coredll:COREDLL.dll
 0001:0002f8a0       GetDateFormatW             000408a0 f   coredll:COREDLL.dll
 0001:0002f8b0       _snwprintf                 000408b0 f   coredll:COREDLL.dll
 0001:0002f8c0       GetModuleFileNameW         000408c0 f   coredll:COREDLL.dll
 0001:0002f8d0       WideCharToMultiByte        000408d0 f   coredll:COREDLL.dll
 0001:0002f8e0       GetTimeZoneInformation     000408e0 f   coredll:COREDLL.dll
 0001:0002f8f0       RaiseException             000408f0 f   coredll:COREDLL.dll
 0001:0002f900       InterlockedDecrement       00040900 f   coredll:COREDLL.dll
 0001:0002f910       WriteFile                  00040910 f   coredll:COREDLL.dll
 0001:0002f920       _vsnwprintf                00040920 f   coredll:COREDLL.dll
 0001:0002f930       InterlockedIncrement       00040930 f   coredll:COREDLL.dll
 0001:0002f940       GetProcAddressW            00040940 f   coredll:COREDLL.dll
 0001:0002f950       SetLastError               00040950 f   coredll:COREDLL.dll
 0001:0002f960       TerminateProcess           00040960 f   coredll:COREDLL.dll
 0002:00003a8c       ?_Min@?$AtlLimits@H@ATL@@2HB 00049a8c     configdlg.obj
 0002:00003a90       ?_Max@?$AtlLimits@H@ATL@@2HB 00049a90     configdlg.obj
 0002:00003a94       ?_Min@?$AtlLimits@I@ATL@@2IB 00049a94     configdlg.obj
 0002:00003a98       ?_Max@?$AtlLimits@I@ATL@@2IB 00049a98     configdlg.obj
 0002:00003a9c       ?_Min@?$AtlLimits@J@ATL@@2JB 00049a9c     configdlg.obj
 0002:00003aa0       ?_Max@?$AtlLimits@J@ATL@@2JB 00049aa0     configdlg.obj
 0002:00003aa4       ?_Min@?$AtlLimits@K@ATL@@2KB 00049aa4     configdlg.obj
 0002:00003aa8       ?_Max@?$AtlLimits@K@ATL@@2KB 00049aa8     configdlg.obj
 0002:00003ab0       ?_Min@?$AtlLimits@_J@ATL@@2_JB 00049ab0     configdlg.obj
 0002:00003ab8       ?_Max@?$AtlLimits@_J@ATL@@2_JB 00049ab8     configdlg.obj
 0002:00003ac0       ?_Min@?$AtlLimits@_K@ATL@@2_KB 00049ac0     configdlg.obj
 0002:00003ac8       ?_Max@?$AtlLimits@_K@ATL@@2_KB 00049ac8     configdlg.obj
 0002:00003ad0       ?VT@?$CVarTypeInfo@D@ATL@@2GB 00049ad0     configdlg.obj
 0002:00003ad4       ?pmField@?$CVarTypeInfo@D@ATL@@2QQtagVARIANT@@DQ3@ 00049ad4     configdlg.obj
 0002:00003ad8       ?VT@?$CVarTypeInfo@E@ATL@@2GB 00049ad8     configdlg.obj
 0002:00003adc       ?pmField@?$CVarTypeInfo@E@ATL@@2QQtagVARIANT@@EQ3@ 00049adc     configdlg.obj
 0002:00003ae0       ?VT@?$CVarTypeInfo@PAD@ATL@@2GB 00049ae0     configdlg.obj
 0002:00003ae4       ?pmField@?$CVarTypeInfo@PAD@ATL@@2QQtagVARIANT@@PADQ3@ 00049ae4     configdlg.obj
 0002:00003ae8       ?VT@?$CVarTypeInfo@PAE@ATL@@2GB 00049ae8     configdlg.obj
 0002:00003aec       ?pmField@?$CVarTypeInfo@PAE@ATL@@2QQtagVARIANT@@PAEQ3@ 00049aec     configdlg.obj
 0002:00003af0       ?VT@?$CVarTypeInfo@F@ATL@@2GB 00049af0     configdlg.obj
 0002:00003af4       ?pmField@?$CVarTypeInfo@F@ATL@@2QQtagVARIANT@@FQ3@ 00049af4     configdlg.obj
 0002:00003af8       ?VT@?$CVarTypeInfo@PAF@ATL@@2GB 00049af8     configdlg.obj
 0002:00003afc       ?pmField@?$CVarTypeInfo@PAF@ATL@@2QQtagVARIANT@@PAFQ3@ 00049afc     configdlg.obj
 0002:00003b00       ?VT@?$CVarTypeInfo@G@ATL@@2GB 00049b00     configdlg.obj
 0002:00003b04       ?pmField@?$CVarTypeInfo@G@ATL@@2QQtagVARIANT@@GQ3@ 00049b04     configdlg.obj
 0002:00003b08       ?VT@?$CVarTypeInfo@H@ATL@@2GB 00049b08     configdlg.obj
 0002:00003b0c       ?pmField@?$CVarTypeInfo@H@ATL@@2QQtagVARIANT@@HQ3@ 00049b0c     configdlg.obj
 0002:00003b10       ?VT@?$CVarTypeInfo@PAH@ATL@@2GB 00049b10     configdlg.obj
 0002:00003b14       ?pmField@?$CVarTypeInfo@PAH@ATL@@2QQtagVARIANT@@PAHQ3@ 00049b14     configdlg.obj
 0002:00003b18       ?VT@?$CVarTypeInfo@I@ATL@@2GB 00049b18     configdlg.obj
 0002:00003b1c       ?pmField@?$CVarTypeInfo@I@ATL@@2QQtagVARIANT@@IQ3@ 00049b1c     configdlg.obj
 0002:00003b20       ?VT@?$CVarTypeInfo@PAI@ATL@@2GB 00049b20     configdlg.obj
 0002:00003b24       ?pmField@?$CVarTypeInfo@PAI@ATL@@2QQtagVARIANT@@PAIQ3@ 00049b24     configdlg.obj
 0002:00003b28       ?VT@?$CVarTypeInfo@J@ATL@@2GB 00049b28     configdlg.obj
 0002:00003b2c       ?pmField@?$CVarTypeInfo@J@ATL@@2QQtagVARIANT@@JQ3@ 00049b2c     configdlg.obj
 0002:00003b30       ?VT@?$CVarTypeInfo@PAJ@ATL@@2GB 00049b30     configdlg.obj
 0002:00003b34       ?pmField@?$CVarTypeInfo@PAJ@ATL@@2QQtagVARIANT@@PAJQ3@ 00049b34     configdlg.obj
 0002:00003b38       ?VT@?$CVarTypeInfo@K@ATL@@2GB 00049b38     configdlg.obj
 0002:00003b3c       ?pmField@?$CVarTypeInfo@K@ATL@@2QQtagVARIANT@@KQ3@ 00049b3c     configdlg.obj
 0002:00003b40       ?VT@?$CVarTypeInfo@PAK@ATL@@2GB 00049b40     configdlg.obj
 0002:00003b44       ?pmField@?$CVarTypeInfo@PAK@ATL@@2QQtagVARIANT@@PAKQ3@ 00049b44     configdlg.obj
 0002:00003b48       ?VT@?$CVarTypeInfo@M@ATL@@2GB 00049b48     configdlg.obj
 0002:00003b4c       ?pmField@?$CVarTypeInfo@M@ATL@@2QQtagVARIANT@@MQ3@ 00049b4c     configdlg.obj
 0002:00003b50       ?VT@?$CVarTypeInfo@PAM@ATL@@2GB 00049b50     configdlg.obj
 0002:00003b54       ?pmField@?$CVarTypeInfo@PAM@ATL@@2QQtagVARIANT@@PAMQ3@ 00049b54     configdlg.obj
 0002:00003b58       ?VT@?$CVarTypeInfo@N@ATL@@2GB 00049b58     configdlg.obj
 0002:00003b5c       ?pmField@?$CVarTypeInfo@N@ATL@@2QQtagVARIANT@@NQ3@ 00049b5c     configdlg.obj
 0002:00003b60       ?VT@?$CVarTypeInfo@PAN@ATL@@2GB 00049b60     configdlg.obj
 0002:00003b64       ?pmField@?$CVarTypeInfo@PAN@ATL@@2QQtagVARIANT@@PANQ3@ 00049b64     configdlg.obj
 0002:00003b68       ?VT@?$CVarTypeInfo@UtagVARIANT@@@ATL@@2GB 00049b68     configdlg.obj
 0002:00003b6c       ?VT@?$CVarTypeInfo@PAG@ATL@@2GB 00049b6c     configdlg.obj
 0002:00003b70       ?pmField@?$CVarTypeInfo@PAG@ATL@@2QQtagVARIANT@@PAGQ3@ 00049b70     configdlg.obj
 0002:00003b74       ?VT@?$CVarTypeInfo@PAPAG@ATL@@2GB 00049b74     configdlg.obj
 0002:00003b78       ?pmField@?$CVarTypeInfo@PAPAG@ATL@@2QQtagVARIANT@@PAPAGQ3@ 00049b78     configdlg.obj
 0002:00003b7c       ?VT@?$CVarTypeInfo@PAUIUnknown@@@ATL@@2GB 00049b7c     configdlg.obj
 0002:00003b80       ?pmField@?$CVarTypeInfo@PAUIUnknown@@@ATL@@2QQtagVARIANT@@PAUIUnknown@@Q3@ 00049b80     configdlg.obj
 0002:00003b84       ?VT@?$CVarTypeInfo@PAPAUIUnknown@@@ATL@@2GB 00049b84     configdlg.obj
 0002:00003b88       ?pmField@?$CVarTypeInfo@PAPAUIUnknown@@@ATL@@2QQtagVARIANT@@PAPAUIUnknown@@Q3@ 00049b88     configdlg.obj
 0002:00003b8c       ?VT@?$CVarTypeInfo@PAUIDispatch@@@ATL@@2GB 00049b8c     configdlg.obj
 0002:00003b90       ?pmField@?$CVarTypeInfo@PAUIDispatch@@@ATL@@2QQtagVARIANT@@PAUIDispatch@@Q3@ 00049b90     configdlg.obj
 0002:00003b94       ?VT@?$CVarTypeInfo@PAPAUIDispatch@@@ATL@@2GB 00049b94     configdlg.obj
 0002:00003b98       ?pmField@?$CVarTypeInfo@PAPAUIDispatch@@@ATL@@2QQtagVARIANT@@PAPAUIDispatch@@Q3@ 00049b98     configdlg.obj
 0002:00003b9c       ?VT@?$CVarTypeInfo@TtagCY@@@ATL@@2GB 00049b9c     configdlg.obj
 0002:00003ba0       ?pmField@?$CVarTypeInfo@TtagCY@@@ATL@@2QQtagVARIANT@@TtagCY@@Q3@ 00049ba0     configdlg.obj
 0002:00003ba4       ?VT@?$CVarTypeInfo@PATtagCY@@@ATL@@2GB 00049ba4     configdlg.obj
 0002:00003ba8       ?pmField@?$CVarTypeInfo@PATtagCY@@@ATL@@2QQtagVARIANT@@PATtagCY@@Q3@ 00049ba8     configdlg.obj
 0002:00003bac       ?c_bIsMFCDLLTraits@?$_MFCDLLTraitsCheck@DV?$StrTraitATL@DV?$ChTraitsOS@D@ATL@@@ATL@@@_CSTRING_IMPL_@ATL@@2_NB 00049bac     configdlg.obj
 0002:00003bad       ?c_bIsMFCDLLTraits@?$_MFCDLLTraitsCheck@GV?$StrTraitATL@GV?$ChTraitsOS@G@ATL@@@ATL@@@_CSTRING_IMPL_@ATL@@2_NB 00049bad     configdlg.obj
 0002:00003bb0       ?generic@CArchiveException@@2HB 00049bb0     configdlg.obj
 0002:00003bb4       ?c_bIsMFCDLLTraits@?$_MFCDLLTraitsCheck@GV?$StrTraitMFC@GV?$ChTraitsOS@G@ATL@@@@@_CSTRING_IMPL_@ATL@@2_NB 00049bb4     configdlg.obj
 0002:00003bb8       ?generic@CFileException@@2HB 00049bb8     configdlg.obj
 0002:00003bc0       ?Millisecond@CFileTime@ATL@@2_KB 00049bc0     configdlg.obj
 0002:00003bc8       ?Second@CFileTime@ATL@@2_KB 00049bc8     configdlg.obj
 0002:00003bd0       ?Minute@CFileTime@ATL@@2_KB 00049bd0     configdlg.obj
 0002:00003bd8       ?Hour@CFileTime@ATL@@2_KB  00049bd8     configdlg.obj
 0002:00003be0       ?Day@CFileTime@ATL@@2_KB   00049be0     configdlg.obj
 0002:00003be8       ?Week@CFileTime@ATL@@2_KB  00049be8     configdlg.obj
 0002:00003bf0       ?szInvalidDateTime@ATL@@3QBGB 00049bf0     configdlg.obj
 0002:00003bf4       ?szInvalidDateTimeSpan@ATL@@3QBGB 00049bf4     configdlg.obj
 0002:000103f4       ??_C@_1BM@FEGPDFAG@?$AAS?$AAy?$AAs?$AAL?$AAi?$AAs?$AAt?$AAV?$AAi?$AAe?$AAw?$AA3?$AA2?$AA?$AA@ 000563f4     listview.obj
 0002:00010410       ??_C@_1GA@OPNDGMGH@?$AAC?$AAr?$AAe?$AAa?$AAt?$AAe?$AAE?$AAR?$AAI?$AAW?$AAi?$AAn?$AAd?$AAo?$AAw?$AA?5?$AA?5?$AAF?$AAa?$AAi?$AAl?$AAe?$AAd?$AA?5?$AAt?$AAo?$AA?5?$AAG?$AAe?$AAt?$AA?5?$AAP@ 00056410     listview.obj
 0002:00010470       ??_C@_1FM@NFCFLKBP@?$AA?3?$AAI?$AAn?$AAi?$AAt?$AAi?$AAa?$AAl?$AAi?$AAz?$AAe?$AAL?$AAi?$AAs?$AAt?$AA?5?$AAn?$AAC?$AAa?$AAr?$AAr?$AAi?$AAe?$AAr?$AA?$DN?$AA?$CF?$AAd?$AA?5?$AA?0?$AAd?$AAw?$AAA@ 00056470     listview.obj
 0002:000104cc       ??_C@_1BO@CKMBKLHM@?$AA?4?$AA?2?$AAl?$AAi?$AAs?$AAt?$AAv?$AAi?$AAe?$AAw?$AA?4?$AAc?$AAp?$AAp?$AA?$AA@ 000564cc     listview.obj
 0002:000104ec       ??_C@_1DC@EBFLAGON@?$AAC?$AAa?$AAn?$AA?5?$AAn?$AAo?$AAt?$AA?5?$AAc?$AAr?$AAe?$AAa?$AAt?$AAe?$AA?5?$AAd?$AAi?$AAa?$AAl?$AAo?$AAg?$AA?5?$AA?$CF?$AAd?$AA?$AA@ 000564ec     listview.obj
 0002:00010520       ??_C@_1M@IDCMGJNH@?$AAC?$AAL?$AAE?$AAA?$AAR?$AA?$AA@ 00056520     listview.obj
 0002:0001989c       ??_C@_1CI@MHCAEBKF@?$AA?$CI?$AA?5?$AAw?$AAf?$AAo?$AAr?$AAm?$AAa?$AAt?$AA?5?$AA?$CB?$AA?$DN?$AA?5?$AAN?$AAU?$AAL?$AAL?$AA?5?$AA?$CJ?$AA?$AA@ 0005f89c     LIBCMTD:wcsftime.obj
 0002:000198c4       ??_C@_1CC@IHEJKGMG@?$AA?$CI?$AA?5?$AAm?$AAa?$AAx?$AAs?$AAi?$AAz?$AAe?$AA?5?$AA?$CB?$AA?$DN?$AA?5?$AA0?$AA?5?$AA?$CJ?$AA?$AA@ 0005f8c4     LIBCMTD:wcsftime.obj
 0002:000198e8       ??_C@_1CC@GIGDCKGO@?$AA_?$AAw?$AAc?$AAs?$AAf?$AAt?$AAi?$AAm?$AAe?$AA_?$AAl?$AA_?$AAs?$AAt?$AAa?$AAt?$AA?$AA@ 0005f8e8     LIBCMTD:wcsftime.obj
 0002:00019910       ??_C@_1FG@JFIEMGOH@?$AAf?$AA?3?$AA?2?$AAs?$AAp?$AA?2?$AAv?$AAc?$AAt?$AAo?$AAo?$AAl?$AAs?$AA?2?$AAc?$AAr?$AAt?$AAc?$AAe?$AA?2?$AAc?$AAr?$AAt?$AAw?$AA3?$AA2?$AA?2?$AAt?$AAi?$AAm?$AAe?$AA?2@ 0005f910     LIBCMTD:wcsftime.obj
 0002:00019968       ??_C@_1CI@MPAHGLBB@?$AA?$CI?$AA?5?$AAw?$AAs?$AAt?$AAr?$AAi?$AAn?$AAg?$AA?5?$AA?$CB?$AA?$DN?$AA?5?$AAN?$AAU?$AAL?$AAL?$AA?5?$AA?$CJ?$AA?$AA@ 0005f968     LIBCMTD:wcsftime.obj
 0002:00019990       ??_C@_1DC@CMKCHHFC@?$AA_?$AAg?$AAe?$AAt?$AA_?$AAt?$AAi?$AAm?$AAe?$AAz?$AAo?$AAn?$AAe?$AA?$CI?$AA?$CG?$AAt?$AAi?$AAm?$AAe?$AAz?$AAo?$AAn?$AAe?$AA?$CJ?$AA?$AA@ 0005f990     LIBCMTD:loctim64.obj
 0002:000199c4       ??_C@_1CO@IMMOMMCB@?$AA_?$AAg?$AAe?$AAt?$AA_?$AAd?$AAs?$AAt?$AAb?$AAi?$AAa?$AAs?$AA?$CI?$AA?$CG?$AAd?$AAs?$AAt?$AAb?$AAi?$AAa?$AAs?$AA?$CJ?$AA?$AA@ 0005f9c4     LIBCMTD:loctim64.obj
 0002:000199f4       ??_C@_1DC@MEHEMOPB@?$AA_?$AAg?$AAe?$AAt?$AA_?$AAd?$AAa?$AAy?$AAl?$AAi?$AAg?$AAh?$AAt?$AA?$CI?$AA?$CG?$AAd?$AAa?$AAy?$AAl?$AAi?$AAg?$AAh?$AAt?$AA?$CJ?$AA?$AA@ 0005f9f4     LIBCMTD:loctim64.obj
 0002:00019a28       ??_C@_1DG@DHJKDLHN@?$AA?$CI?$AA?$CK?$AAp?$AAt?$AAi?$AAm?$AAe?$AA?5?$AA?$DM?$AA?$DN?$AA?5?$AA_?$AAM?$AAA?$AAX?$AA_?$AA_?$AAT?$AAI?$AAM?$AAE?$AA6?$AA4?$AA_?$AAT?$AA?$CJ?$AA?$AA@ 0005fa28     LIBCMTD:loctim64.obj
 0002:00019a60       ??_C@_1CE@EHHPAMNN@?$AA?$CI?$AA?5?$AAp?$AAt?$AAi?$AAm?$AAe?$AA?5?$AA?$CB?$AA?$DN?$AA?5?$AAN?$AAU?$AAL?$AAL?$AA?5?$AA?$CJ?$AA?$AA@ 0005fa60     LIBCMTD:loctim64.obj
 0002:00019a84       ??_C@_1BO@OIBEEOEM@?$AA_?$AAl?$AAo?$AAc?$AAa?$AAl?$AAt?$AAi?$AAm?$AAe?$AA6?$AA4?$AA_?$AAs?$AA?$AA@ 0005fa84     LIBCMTD:loctim64.obj
 0002:00019aa8       ??_C@_1FG@CKGMIEEH@?$AAf?$AA?3?$AA?2?$AAs?$AAp?$AA?2?$AAv?$AAc?$AAt?$AAo?$AAo?$AAl?$AAs?$AA?2?$AAc?$AAr?$AAt?$AAc?$AAe?$AA?2?$AAc?$AAr?$AAt?$AAw?$AA3?$AA2?$AA?2?$AAt?$AAi?$AAm?$AAe?$AA?2@ 0005faa8     LIBCMTD:loctim64.obj
 0002:00019b00       ??_C@_1CA@NJFECEIO@?$AA?$CI?$AA?5?$AAp?$AAt?$AAm?$AA?5?$AA?$CB?$AA?$DN?$AA?5?$AAN?$AAU?$AAL?$AAL?$AA?5?$AA?$CJ?$AA?$AA@ 0005fb00     LIBCMTD:loctim64.obj
 0002:00019b20       ??_C@_08JCCMCCIL@HH?3mm?3ss?$AA@ 0005fb20     LIBCMTD:strftime.obj
 0002:00019b2c       ??_C@_0BE@CKGJFCPC@dddd?0?5MMMM?5dd?0?5yyyy?$AA@ 0005fb2c     LIBCMTD:strftime.obj
 0002:00019b40       ??_C@_08BPBNCDIB@MM?1dd?1yy?$AA@ 0005fb40     LIBCMTD:strftime.obj
 0002:00019b4c       ??_C@_02CJNFDJBF@PM?$AA@   0005fb4c     LIBCMTD:strftime.obj
 0002:00019b50       ??_C@_02DEDBPAFC@AM?$AA@   0005fb50     LIBCMTD:strftime.obj
 0002:00019b54       ??_C@_08EDHMEBNP@December?$AA@ 0005fb54     LIBCMTD:strftime.obj
 0002:00019b60       ??_C@_08HCHEGEOA@November?$AA@ 0005fb60     LIBCMTD:strftime.obj
 0002:00019b6c       ??_C@_07JJNFCEND@October?$AA@ 0005fb6c     LIBCMTD:strftime.obj
 0002:00019b74       ??_C@_09BHHEALKD@September?$AA@ 0005fb74     LIBCMTD:strftime.obj
 0002:00019b80       ??_C@_06LBBHFDDG@August?$AA@ 0005fb80     LIBCMTD:strftime.obj
 0002:00019b88       ??_C@_04MIEPOIFP@July?$AA@ 0005fb88     LIBCMTD:strftime.obj
 0002:00019b90       ??_C@_04CNLMGBGM@June?$AA@ 0005fb90     LIBCMTD:strftime.obj
 0002:00019b98       ??_C@_05DMJDNLEJ@April?$AA@ 0005fb98     LIBCMTD:strftime.obj
 0002:00019ba0       ??_C@_05HPCKOFNC@March?$AA@ 0005fba0     LIBCMTD:strftime.obj
 0002:00019ba8       ??_C@_08GNJGEPFN@February?$AA@ 0005fba8     LIBCMTD:strftime.obj
 0002:00019bb4       ??_C@_07CGJPFGJA@January?$AA@ 0005fbb4     LIBCMTD:strftime.obj
 0002:00019bbc       ??_C@_03MKABNOCG@Dec?$AA@  0005fbbc     LIBCMTD:strftime.obj
 0002:00019bc0       ??_C@_03JPJOFNIA@Nov?$AA@  0005fbc0     LIBCMTD:strftime.obj
 0002:00019bc4       ??_C@_03BMAOKBAD@Oct?$AA@  0005fbc4     LIBCMTD:strftime.obj
 0002:00019bc8       ??_C@_03GGCAPAJC@Sep?$AA@  0005fbc8     LIBCMTD:strftime.obj
 0002:00019bcc       ??_C@_03IFJFEIGA@Aug?$AA@  0005fbcc     LIBCMTD:strftime.obj
 0002:00019bd0       ??_C@_03LBGABGKK@Jul?$AA@  0005fbd0     LIBCMTD:strftime.obj
 0002:00019bd4       ??_C@_03IDFGHECI@Jun?$AA@  0005fbd4     LIBCMTD:strftime.obj
 0002:00019bd8       ??_C@_03CNMDKL@May?$AA@    0005fbd8     LIBCMTD:strftime.obj
 0002:00019bdc       ??_C@_03LEOLGMJP@Apr?$AA@  0005fbdc     LIBCMTD:strftime.obj
 0002:00019be0       ??_C@_03ODNJBKGA@Mar?$AA@  0005fbe0     LIBCMTD:strftime.obj
 0002:00019be4       ??_C@_03HJBDCHOM@Feb?$AA@  0005fbe4     LIBCMTD:strftime.obj
 0002:00019be8       ??_C@_03JIHJHPIE@Jan?$AA@  0005fbe8     LIBCMTD:strftime.obj
 0002:00019bec       ??_C@_08INBOOONO@Saturday?$AA@ 0005fbec     LIBCMTD:strftime.obj
 0002:00019bf8       ??_C@_06JECMNKMI@Friday?$AA@ 0005fbf8     LIBCMTD:strftime.obj
 0002:00019c00       ??_C@_08HACCIKIA@Thursday?$AA@ 0005fc00     LIBCMTD:strftime.obj
 0002:00019c0c       ??_C@_09DLIGFAKA@Wednesday?$AA@ 0005fc0c     LIBCMTD:strftime.obj
 0002:00019c18       ??_C@_07BAAGCFCM@Tuesday?$AA@ 0005fc18     LIBCMTD:strftime.obj
 0002:00019c20       ??_C@_06JLEDEDGH@Monday?$AA@ 0005fc20     LIBCMTD:strftime.obj
 0002:00019c28       ??_C@_06OOPIFAJ@Sunday?$AA@ 0005fc28     LIBCMTD:strftime.obj
 0002:00019c30       ??_C@_03FEFJNEK@Sat?$AA@   0005fc30     LIBCMTD:strftime.obj
 0002:00019c34       ??_C@_03IDIOELNC@Fri?$AA@  0005fc34     LIBCMTD:strftime.obj
 0002:00019c38       ??_C@_03IOFIKPDN@Thu?$AA@  0005fc38     LIBCMTD:strftime.obj
 0002:00019c3c       ??_C@_03MHOMLAJA@Wed?$AA@  0005fc3c     LIBCMTD:strftime.obj
 0002:00019c40       ??_C@_03NAGEINEP@Tue?$AA@  0005fc40     LIBCMTD:strftime.obj
 0002:00019c44       ??_C@_03PDAGKDH@Mon?$AA@   0005fc44     LIBCMTD:strftime.obj
 0002:00019c48       ??_C@_03KOEHGMDN@Sun?$AA@  0005fc48     LIBCMTD:strftime.obj
 0002:00019c50       ??_C@_1FM@LPEPDBJF@?$AAs?$AAt?$AAr?$AAc?$AAp?$AAy?$AA_?$AAs?$AA?$CI?$AAs?$AA?0?$AA?5?$AA?$CI?$AAl?$AAe?$AAn?$AA?5?$AA?$CL?$AA?5?$AA1?$AA?$CJ?$AA?5?$AA?9?$AA?5?$AA?$CI?$AAs?$AA?5?$AA?9?$AA?5?$AAp?$AA?$CJ?$AA?0@ 0005fc50     LIBCMTD:strftime.obj
 0002:00019cb0       ??_C@_1GG@NAGHPCAA@?$AAs?$AAt?$AAr?$AAc?$AAp?$AAy?$AA_?$AAs?$AA?$CI?$AAs?$AA?0?$AA?5?$AA?$CI?$AAl?$AAe?$AAn?$AA?5?$AA?$CL?$AA?5?$AA1?$AA?$CJ?$AA?5?$AA?9?$AA?5?$AA?$CI?$AAs?$AA?5?$AA?9?$AA?5?$AAp?$AA?$CJ?$AA?0@ 0005fcb0     LIBCMTD:strftime.obj
 0002:00019d18       ??_C@_1BG@LGACIFJI@?$AA_?$AAG?$AAe?$AAt?$AAd?$AAa?$AAy?$AAs?$AA_?$AAl?$AA?$AA@ 0005fd18     LIBCMTD:strftime.obj
 0002:00019d30       ??_C@_1FG@CHPFOOLA@?$AAf?$AA?3?$AA?2?$AAs?$AAp?$AA?2?$AAv?$AAc?$AAt?$AAo?$AAo?$AAl?$AAs?$AA?2?$AAc?$AAr?$AAt?$AAc?$AAe?$AA?2?$AAc?$AAr?$AAt?$AAw?$AA3?$AA2?$AA?2?$AAt?$AAi?$AAm?$AAe?$AA?2@ 0005fd30     LIBCMTD:strftime.obj
 0002:00019d88       ??_C@_1FO@IFFKPIEL@?$AAs?$AAt?$AAr?$AAc?$AAp?$AAy?$AA_?$AAs?$AA?$CI?$AAs?$AA?0?$AA?5?$AA?$CI?$AAl?$AAe?$AAn?$AA?5?$AA?$CL?$AA?5?$AA1?$AA?$CJ?$AA?5?$AA?9?$AA?5?$AA?$CI?$AAs?$AA?5?$AA?9?$AA?5?$AAp?$AA?$CJ?$AA?0@ 0005fd88     LIBCMTD:strftime.obj
 0002:00019de8       ??_C@_1GI@LNJDDNLK@?$AAs?$AAt?$AAr?$AAc?$AAp?$AAy?$AA_?$AAs?$AA?$CI?$AAs?$AA?0?$AA?5?$AA?$CI?$AAl?$AAe?$AAn?$AA?5?$AA?$CL?$AA?5?$AA1?$AA?$CJ?$AA?5?$AA?9?$AA?5?$AA?$CI?$AAs?$AA?5?$AA?9?$AA?5?$AAp?$AA?$CJ?$AA?0@ 0005fde8     LIBCMTD:strftime.obj
 0002:00019e50       ??_C@_1BK@IDMELNCB@?$AA_?$AAG?$AAe?$AAt?$AAm?$AAo?$AAn?$AAt?$AAh?$AAs?$AA_?$AAl?$AA?$AA@ 0005fe50     LIBCMTD:strftime.obj
 0002:00019e70       ??_C@_1FG@CJBIADLJ@?$AAs?$AAt?$AAr?$AAc?$AAp?$AAy?$AA_?$AAs?$AA?$CI?$AAs?$AA?0?$AA?5?$AAl?$AAe?$AAn?$AA?5?$AA?9?$AA?5?$AA?$CI?$AAs?$AA?5?$AA?9?$AA?5?$AAp?$AA?$CJ?$AA?0?$AA?5?$AAp?$AAt?$AA?9?$AA?$DO?$AAw@ 0005fe70     LIBCMTD:strftime.obj
 0002:00019ec8       ??_C@_1FI@PPIHCJGH@?$AAs?$AAt?$AAr?$AAc?$AAp?$AAy?$AA_?$AAs?$AA?$CI?$AAs?$AA?0?$AA?5?$AAl?$AAe?$AAn?$AA?5?$AA?9?$AA?5?$AA?$CI?$AAs?$AA?5?$AA?9?$AA?5?$AAp?$AA?$CJ?$AA?0?$AA?5?$AAp?$AAt?$AA?9?$AA?$DO?$AAw@ 0005fec8     LIBCMTD:strftime.obj
 0002:00019f20       ??_C@_1FI@GDNOPCGD@?$AAs?$AAt?$AAr?$AAc?$AAp?$AAy?$AA_?$AAs?$AA?$CI?$AAs?$AA?0?$AA?5?$AAl?$AAe?$AAn?$AA?5?$AA?9?$AA?5?$AA?$CI?$AAs?$AA?5?$AA?9?$AA?5?$AAp?$AA?$CJ?$AA?0?$AA?5?$AAp?$AAt?$AA?9?$AA?$DO?$AAw@ 0005ff20     LIBCMTD:strftime.obj
 0002:00019f78       ??_C@_1FA@MEHIJEIL@?$AAs?$AAt?$AAr?$AAc?$AAp?$AAy?$AA_?$AAs?$AA?$CI?$AAs?$AA?0?$AA?5?$AAl?$AAe?$AAn?$AA?5?$AA?9?$AA?5?$AA?$CI?$AAs?$AA?5?$AA?9?$AA?5?$AAp?$AA?$CJ?$AA?0?$AA?5?$AAp?$AAt?$AA?9?$AA?$DO?$AAa@ 0005ff78     LIBCMTD:strftime.obj
 0002:00019fc8       ??_C@_1FA@INCJEBF@?$AAs?$AAt?$AAr?$AAc?$AAp?$AAy?$AA_?$AAs?$AA?$CI?$AAs?$AA?0?$AA?5?$AAl?$AAe?$AAn?$AA?5?$AA?9?$AA?5?$AA?$CI?$AAs?$AA?5?$AA?9?$AA?5?$AAp?$AA?$CJ?$AA?0?$AA?5?$AAp?$AAt?$AA?9?$AA?$DO?$AAa@ 0005ffc8     LIBCMTD:strftime.obj
 0002:0001a018       ??_C@_1FC@BEAPAEGE@?$AAs?$AAt?$AAr?$AAc?$AAp?$AAy?$AA_?$AAs?$AA?$CI?$AAs?$AA?0?$AA?5?$AAl?$AAe?$AAn?$AA?5?$AA?9?$AA?5?$AA?$CI?$AAs?$AA?5?$AA?9?$AA?5?$AAp?$AA?$CJ?$AA?0?$AA?5?$AAp?$AAt?$AA?9?$AA?$DO?$AAm@ 00060018     LIBCMTD:strftime.obj
 0002:0001a070       ??_C@_1FM@CHHONFED@?$AAs?$AAt?$AAr?$AAc?$AAp?$AAy?$AA_?$AAs?$AA?$CI?$AAs?$AA?0?$AA?5?$AAl?$AAe?$AAn?$AA?5?$AA?9?$AA?5?$AA?$CI?$AAs?$AA?5?$AA?9?$AA?5?$AAp?$AA?$CJ?$AA?0?$AA?5?$AAp?$AAt?$AA?9?$AA?$DO?$AAm@ 00060070     LIBCMTD:strftime.obj
 0002:0001a0d0       ??_C@_1FA@EBHJJADL@?$AAs?$AAt?$AAr?$AAc?$AAp?$AAy?$AA_?$AAs?$AA?$CI?$AAs?$AA?0?$AA?5?$AAl?$AAe?$AAn?$AA?5?$AA?9?$AA?5?$AA?$CI?$AAs?$AA?5?$AA?9?$AA?5?$AAp?$AA?$CJ?$AA?0?$AA?5?$AAp?$AAt?$AA?9?$AA?$DO?$AAw@ 000600d0     LIBCMTD:strftime.obj
 0002:0001a120       ??_C@_1FK@ODMKEFLD@?$AAs?$AAt?$AAr?$AAc?$AAp?$AAy?$AA_?$AAs?$AA?$CI?$AAs?$AA?0?$AA?5?$AAl?$AAe?$AAn?$AA?5?$AA?9?$AA?5?$AA?$CI?$AAs?$AA?5?$AA?9?$AA?5?$AAp?$AA?$CJ?$AA?0?$AA?5?$AAp?$AAt?$AA?9?$AA?$DO?$AAw@ 00060120     LIBCMTD:strftime.obj
 0002:0001a17c       ??_C@_1BK@MJNHIAGO@?$AA_?$AAG?$AAe?$AAt?$AAt?$AAn?$AAa?$AAm?$AAe?$AAs?$AA_?$AAl?$AA?$AA@ 0006017c     LIBCMTD:strftime.obj
 0002:0001a198       ??_C@_1M@HCOOECOK@?$AAF?$AAA?$AAL?$AAS?$AAE?$AA?$AA@ 00060198     LIBCMTD:strftime.obj
 0002:0001a1a8       ??_C@_1HC@JGDOBCNK@?$AA?$CI?$AA?$CC?$AAI?$AAn?$AAv?$AAa?$AAl?$AAi?$AAd?$AA?5?$AAM?$AAB?$AAC?$AAS?$AA?5?$AAc?$AAh?$AAa?$AAr?$AAa?$AAc?$AAt?$AAe?$AAr?$AA?5?$AAs?$AAe?$AAq?$AAu?$AAe?$AAn?$AAc@ 000601a8     LIBCMTD:strftime.obj
 0002:0001a21c       ??_C@_1BG@CCBNLOOI@?$AAt?$AAi?$AAm?$AAe?$AAp?$AAt?$AAr?$AA?$CB?$AA?$DN?$AA0?$AA?$AA@ 0006021c     LIBCMTD:strftime.obj
 0002:0001a234       ??_C@_1CG@MHIOFJLE@?$AA?$CI?$AA?5?$AAf?$AAo?$AAr?$AAm?$AAa?$AAt?$AA?5?$AA?$CB?$AA?$DN?$AA?5?$AAN?$AAU?$AAL?$AAL?$AA?5?$AA?$CJ?$AA?$AA@ 00060234     LIBCMTD:strftime.obj
 0002:0001a25c       ??_C@_1BI@ONBMGNNA@?$AA_?$AAS?$AAt?$AAr?$AAf?$AAt?$AAi?$AAm?$AAe?$AA_?$AAl?$AA?$AA@ 0006025c     LIBCMTD:strftime.obj
 0002:0001a274       ??_C@_1CG@MPKJHDAA@?$AA?$CI?$AA?5?$AAs?$AAt?$AAr?$AAi?$AAn?$AAg?$AA?5?$AA?$CB?$AA?$DN?$AA?5?$AAN?$AAU?$AAL?$AAL?$AA?5?$AA?$CJ?$AA?$AA@ 00060274     LIBCMTD:strftime.obj
 0002:0001a2a0       ??_C@_1EG@JNJKHKFI@?$AA?$CI?$AA?5?$AA?$CC?$AAI?$AAn?$AAv?$AAa?$AAl?$AAi?$AAd?$AA?5?$AAf?$AAo?$AAr?$AAm?$AAa?$AAt?$AA?5?$AAd?$AAi?$AAr?$AAe?$AAc?$AAt?$AAi?$AAv?$AAe?$AA?$CC?$AA?5?$AA?0?$AA?5?$AA0@ 000602a0     LIBCMTD:strftime.obj
 0002:0001a2e8       ??_C@_1DC@NMCFBMJP@?$AA?$CI?$AA?5?$AAt?$AAi?$AAm?$AAe?$AAp?$AAt?$AAr?$AA?9?$AA?$DO?$AAt?$AAm?$AA_?$AAy?$AAe?$AAa?$AAr?$AA?5?$AA?$DO?$AA?$DN?$AA0?$AA?5?$AA?$CJ?$AA?$AA@ 000602e8     LIBCMTD:strftime.obj
 0002:0001a320       ??_C@_1HC@HLKHIKOB@?$AA?$CI?$AA?5?$AA?$CI?$AA?5?$AAt?$AAi?$AAm?$AAe?$AAp?$AAt?$AAr?$AA?9?$AA?$DO?$AAt?$AAm?$AA_?$AAs?$AAe?$AAc?$AA?5?$AA?$DO?$AA?$DN?$AA0?$AA?5?$AA?$CJ?$AA?5?$AA?$CG?$AA?$CG?$AA?5?$AA?$CI?$AA?5?$AAt@ 00060320     LIBCMTD:strftime.obj
 0002:0001a398       ??_C@_1HC@IGKDPPHL@?$AA?$CI?$AA?5?$AA?$CI?$AA?5?$AAt?$AAi?$AAm?$AAe?$AAp?$AAt?$AAr?$AA?9?$AA?$DO?$AAt?$AAm?$AA_?$AAm?$AAi?$AAn?$AA?5?$AA?$DO?$AA?$DN?$AA0?$AA?5?$AA?$CJ?$AA?5?$AA?$CG?$AA?$CG?$AA?5?$AA?$CI?$AA?5?$AAt@ 00060398     LIBCMTD:strftime.obj
 0002:0001a410       ??_C@_1HI@HHCJCPE@?$AA?$CI?$AA?5?$AA?$CI?$AA?5?$AAt?$AAi?$AAm?$AAe?$AAp?$AAt?$AAr?$AA?9?$AA?$DO?$AAt?$AAm?$AA_?$AAy?$AAd?$AAa?$AAy?$AA?5?$AA?$DO?$AA?$DN?$AA0?$AA?5?$AA?$CJ?$AA?5?$AA?$CG?$AA?$CG?$AA?5?$AA?$CI?$AA?5@ 00060410     LIBCMTD:strftime.obj
 0002:0001a488       ??_C@_1HG@KCGGFLNI@?$AA?$CI?$AA?5?$AA?$CI?$AA?5?$AAt?$AAi?$AAm?$AAe?$AAp?$AAt?$AAr?$AA?9?$AA?$DO?$AAt?$AAm?$AA_?$AAh?$AAo?$AAu?$AAr?$AA?5?$AA?$DO?$AA?$DN?$AA0?$AA?5?$AA?$CJ?$AA?5?$AA?$CG?$AA?$CG?$AA?5?$AA?$CI?$AA?5@ 00060488     LIBCMTD:strftime.obj
 0002:0001a500       ??_C@_1HG@NFHHOAD@?$AA?$CI?$AA?5?$AA?$CI?$AA?5?$AAt?$AAi?$AAm?$AAe?$AAp?$AAt?$AAr?$AA?9?$AA?$DO?$AAt?$AAm?$AA_?$AAm?$AAd?$AAa?$AAy?$AA?5?$AA?$DO?$AA?$DN?$AA1?$AA?5?$AA?$CJ?$AA?5?$AA?$CG?$AA?$CG?$AA?5?$AA?$CI?$AA?5@ 00060500     LIBCMTD:strftime.obj
 0002:0001a578       ??_C@_1HC@OOAMILFB@?$AA?$CI?$AA?5?$AA?$CI?$AA?5?$AAt?$AAi?$AAm?$AAe?$AAp?$AAt?$AAr?$AA?9?$AA?$DO?$AAt?$AAm?$AA_?$AAm?$AAo?$AAn?$AA?5?$AA?$DO?$AA?$DN?$AA0?$AA?5?$AA?$CJ?$AA?5?$AA?$CG?$AA?$CG?$AA?5?$AA?$CI?$AA?5?$AAt@ 00060578     LIBCMTD:strftime.obj
 0002:0001a5ec       ??_C@_1BI@HBKPAJH@?$AA_?$AAe?$AAx?$AAp?$AAa?$AAn?$AAd?$AAt?$AAi?$AAm?$AAe?$AA?$AA@ 000605ec     LIBCMTD:strftime.obj
 0002:0001a608       ??_C@_1HE@BFLEOKFO@?$AA?$CI?$AA?5?$AA?$CI?$AA?5?$AAt?$AAi?$AAm?$AAe?$AAp?$AAt?$AAr?$AA?9?$AA?$DO?$AAt?$AAm?$AA_?$AAw?$AAd?$AAa?$AAy?$AA?5?$AA?$DO?$AA?$DN?$AA0?$AA?5?$AA?$CJ?$AA?5?$AA?$CG?$AA?$CG?$AA?5?$AA?$CI?$AA?5@ 00060608     LIBCMTD:strftime.obj
 0002:0001a680       ??_C@_1HG@PAEENAPO@?$AA?$CI?$AA?$CC?$AAI?$AAn?$AAv?$AAa?$AAl?$AAi?$AAd?$AA?5?$AAM?$AAB?$AAC?$AAS?$AA?5?$AAc?$AAh?$AAa?$AAr?$AAa?$AAc?$AAt?$AAe?$AAr?$AA?5?$AAs?$AAe?$AAq?$AAu?$AAe?$AAn?$AAc@ 00060680     LIBCMTD:strftime.obj
 0002:0001a6f8       ??_C@_1IE@EIDABBDG@?$AA?$CI?$AA?$CC?$AAI?$AAn?$AAv?$AAa?$AAl?$AAi?$AAd?$AA?5?$AAM?$AAB?$AAC?$AAS?$AA?5?$AAc?$AAh?$AAa?$AAr?$AAa?$AAc?$AAt?$AAe?$AAr?$AA?5?$AAs?$AAe?$AAq?$AAu?$AAe?$AAn?$AAc@ 000606f8     LIBCMTD:strftime.obj
 0002:0001a77c       ??_C@_03EBAPMIKO@a?1p?$AA@ 0006077c     LIBCMTD:strftime.obj
 0002:0001a780       ??_C@_05JAMEPDIN@am?1pm?$AA@ 00060780     LIBCMTD:strftime.obj
 0002:0001a788       ??_C@_1BKC@GNMHAJKJ@?$AA?$CI?$AA?5?$AA?$CI?$AA?5?$AAt?$AAm?$AAp?$AAt?$AAr?$AA?9?$AA?$DO?$AAt?$AAm?$AA_?$AAm?$AAd?$AAa?$AAy?$AA?5?$AA?$DO?$AA?$DN?$AA?5?$AA1?$AA?5?$AA?$CJ?$AA?5?$AA?$CG?$AA?$CG?$AA?5?$AA?$CI?$AA?5?$AA?$CI@ 00060788     LIBCMTD:strftime.obj
 0002:0001a930       ??_C@_1GM@ODJADGLF@?$AA?$CI?$AA?5?$AA?$CI?$AA?5?$AAt?$AAm?$AAp?$AAt?$AAr?$AA?9?$AA?$DO?$AAt?$AAm?$AA_?$AAs?$AAe?$AAc?$AA?5?$AA?$DO?$AA?$DN?$AA?5?$AA0?$AA?5?$AA?$CJ?$AA?5?$AA?$CG?$AA?$CG?$AA?5?$AA?$CI?$AA?5?$AAt?$AAm@ 00060930     LIBCMTD:strftime.obj
 0002:0001a9a0       ??_C@_1GM@LGPAHFOJ@?$AA?$CI?$AA?5?$AA?$CI?$AA?5?$AAt?$AAm?$AAp?$AAt?$AAr?$AA?9?$AA?$DO?$AAt?$AAm?$AA_?$AAm?$AAi?$AAn?$AA?5?$AA?$DO?$AA?$DN?$AA?5?$AA0?$AA?5?$AA?$CJ?$AA?5?$AA?$CG?$AA?$CG?$AA?5?$AA?$CI?$AA?5?$AAt?$AAm@ 000609a0     LIBCMTD:strftime.obj
 0002:0001aa10       ??_C@_1HA@HFAMHJOB@?$AA?$CI?$AA?5?$AA?$CI?$AA?5?$AAt?$AAm?$AAp?$AAt?$AAr?$AA?9?$AA?$DO?$AAt?$AAm?$AA_?$AAh?$AAo?$AAu?$AAr?$AA?5?$AA?$DO?$AA?$DN?$AA?5?$AA0?$AA?5?$AA?$CJ?$AA?5?$AA?$CG?$AA?$CG?$AA?5?$AA?$CI?$AA?5?$AAt@ 00060a10     LIBCMTD:strftime.obj
 0002:0001aa80       ??_C@_1GM@PGNHCPKA@?$AA?$CI?$AA?5?$AA?$CI?$AA?5?$AAt?$AAm?$AAp?$AAt?$AAr?$AA?9?$AA?$DO?$AAt?$AAm?$AA_?$AAm?$AAo?$AAn?$AA?5?$AA?$DO?$AA?$DN?$AA?5?$AA0?$AA?5?$AA?$CJ?$AA?5?$AA?$CG?$AA?$CG?$AA?5?$AA?$CI?$AA?5?$AAt?$AAm@ 00060a80     LIBCMTD:strftime.obj
 0002:0001aaec       ??_C@_1BO@CFDLGFLB@?$AA_?$AAs?$AAt?$AAo?$AAr?$AAe?$AA_?$AAw?$AAi?$AAn?$AAw?$AAo?$AAr?$AAd?$AA?$AA@ 00060aec     LIBCMTD:strftime.obj
 0002:0001ab0c       ??_C@_1DA@DFCEAJHI@?$AA?$CI?$AA?5?$AAt?$AAm?$AAp?$AAt?$AAr?$AA?9?$AA?$DO?$AAt?$AAm?$AA_?$AAy?$AAe?$AAa?$AAr?$AA?5?$AA?$DO?$AA?$DN?$AA?5?$AA0?$AA?5?$AA?$CJ?$AA?$AA@ 00060b0c     LIBCMTD:strftime.obj
 0002:0001ab3c       ??_C@_17LGKOMLJ@?$AA?4?$AA?4?$AA?4?$AA?$AA@ 00060b3c     LIBCMTD:dbgrpt.obj
 0002:0001ab44       ??_C@_1CC@CGHMNGDG@?$AAA?$AAs?$AAs?$AAe?$AAr?$AAt?$AAi?$AAo?$AAn?$AA?5?$AAF?$AAa?$AAi?$AAl?$AAe?$AAd?$AA?$AA@ 00060b44     LIBCMTD:dbgrpt.obj
 0002:0001ab68       ??_C@_1M@ILHOPKA@?$AAE?$AAr?$AAr?$AAo?$AAr?$AA?$AA@ 00060b68     LIBCMTD:dbgrpt.obj
 0002:0001ab74       ??_C@_1BA@GLMCNLEM@?$AAW?$AAa?$AAr?$AAn?$AAi?$AAn?$AAg?$AA?$AA@ 00060b74     LIBCMTD:dbgrpt.obj
 0002:0001ab88       ??_C@_1FI@PHIAFFHM@?$AA?$CI?$AA?$CC?$AAT?$AAh?$AAe?$AA?5?$AAh?$AAo?$AAo?$AAk?$AA?5?$AAf?$AAu?$AAn?$AAc?$AAt?$AAi?$AAo?$AAn?$AA?5?$AAi?$AAs?$AA?5?$AAn?$AAo?$AAt?$AA?5?$AAi?$AAn?$AA?5?$AAt?$AAh@ 00060b88     LIBCMTD:dbgrpt.obj
 0002:0001abe0       ??_C@_1CG@JBJEFOCM@?$AAp?$AAf?$AAn?$AAN?$AAe?$AAw?$AAH?$AAo?$AAo?$AAk?$AA?5?$AA?$CB?$AA?$DN?$AA?5?$AAN?$AAU?$AAL?$AAL?$AA?$AA@ 00060be0     LIBCMTD:dbgrpt.obj
 0002:0001ac08       ??_C@_1CI@OOAHIOG@?$AA_?$AAC?$AAr?$AAt?$AAS?$AAe?$AAt?$AAR?$AAe?$AAp?$AAo?$AAr?$AAt?$AAH?$AAo?$AAo?$AAk?$AAT?$AA2?$AA?$AA@ 00060c08     LIBCMTD:dbgrpt.obj
 0002:0001ac30       ??_C@_1FC@DDJKODKC@?$AAf?$AA?3?$AA?2?$AAs?$AAp?$AA?2?$AAv?$AAc?$AAt?$AAo?$AAo?$AAl?$AAs?$AA?2?$AAc?$AAr?$AAt?$AAc?$AAe?$AA?2?$AAc?$AAr?$AAt?$AAw?$AA3?$AA2?$AA?2?$AAm?$AAi?$AAs?$AAc?$AA?2@ 00060c30     LIBCMTD:dbgrpt.obj
 0002:0001ac88       ??_C@_1HI@OFEHGPPC@?$AAm?$AAo?$AAd?$AAe?$AA?5?$AA?$DN?$AA?$DN?$AA?5?$AA_?$AAC?$AAR?$AAT?$AA_?$AAR?$AAP?$AAT?$AAH?$AAO?$AAO?$AAK?$AA_?$AAI?$AAN?$AAS?$AAT?$AAA?$AAL?$AAL?$AA?5?$AA?$HM?$AA?$HM?$AA?5@ 00060c88     LIBCMTD:dbgrpt.obj
 0002:0001ad00       ??_C@_1EG@PEOEAKBB@?$AAM?$AAi?$AAc?$AAr?$AAo?$AAs?$AAo?$AAf?$AAt?$AA?5?$AAV?$AAi?$AAs?$AAu?$AAa?$AAl?$AA?5?$AAC?$AA?$CL?$AA?$CL?$AA?5?$AAD?$AAe?$AAb?$AAu?$AAg?$AA?5?$AAL?$AAi?$AAb?$AAr?$AAa@ 00060d00     LIBCMTD:dbgrpt.obj
 0002:0001ad48       ??_C@_1JI@EACPGHID@?$AAw?$AAc?$AAs?$AAc?$AAp?$AAy?$AA_?$AAs?$AA?$CI?$AAs?$AAz?$AAO?$AAu?$AAt?$AAM?$AAe?$AAs?$AAs?$AAa?$AAg?$AAe?$AA?0?$AA?5?$AA4?$AA0?$AA9?$AA6?$AA?0?$AA?5?$AAL?$AA?$CC?$AA_@ 00060d48     LIBCMTD:dbgrpt.obj
 0002:0001ade0       ??_C@_1FG@BBOLDHGF@?$AA_?$AAC?$AAr?$AAt?$AAD?$AAb?$AAg?$AAR?$AAe?$AAp?$AAo?$AAr?$AAt?$AA?3?$AA?5?$AAS?$AAt?$AAr?$AAi?$AAn?$AAg?$AA?5?$AAt?$AAo?$AAo?$AA?5?$AAl?$AAo?$AAn?$AAg?$AA?5?$AAo@ 00060de0     LIBCMTD:dbgrpt.obj
 0002:0001ae38       ??_C@_1KG@MFHGLLO@?$AAD?$AAe?$AAb?$AAu?$AAg?$AA?5?$AA?$CF?$AAs?$AA?$CB?$AA?6?$AA?6?$AAP?$AAr?$AAo?$AAg?$AAr?$AAa?$AAm?$AA?3?$AA?5?$AA?$CF?$AAs?$AA?$CF?$AAs?$AA?$CF?$AAs?$AA?$CF?$AAs?$AA?$CF?$AAs?$AA?$CF?$AAs@ 00060e38     LIBCMTD:dbgrpt.obj
 0002:0001aee0       ??_C@_1BE@CGCJKGHI@?$AA?6?$AAM?$AAo?$AAd?$AAu?$AAl?$AAe?$AA?3?$AA?5?$AA?$AA@ 00060ee0     LIBCMTD:dbgrpt.obj
 0002:0001aef4       ??_C@_1BA@LNHECFIM@?$AA?6?$AAF?$AAi?$AAl?$AAe?$AA?3?$AA?5?$AA?$AA@ 00060ef4     LIBCMTD:dbgrpt.obj
 0002:0001af04       ??_C@_1BA@GLLGCPCK@?$AA?6?$AAL?$AAi?$AAn?$AAe?$AA?3?$AA?5?$AA?$AA@ 00060f04     LIBCMTD:dbgrpt.obj
 0002:0001af14       ??_C@_13LBAGMAIH@?$AA?6?$AA?$AA@ 00060f14     LIBCMTD:dbgrpt.obj
 0002:0001af18       ??_C@_1BK@PEDCIPMA@?$AAE?$AAx?$AAp?$AAr?$AAe?$AAs?$AAs?$AAi?$AAo?$AAn?$AA?3?$AA?5?$AA?$AA@ 00060f18     LIBCMTD:dbgrpt.obj
 0002:0001af34       ??_C@_11LOCGONAA@?$AA?$AA@ 00060f34     LIBCMTD:dbgrpt.obj
 0002:0001af38       ??_C@_1JM@GKDPCMEA@?$AAw?$AAc?$AAs?$AAn?$AAc?$AAp?$AAy?$AA_?$AAs?$AA?$CI?$AAs?$AAz?$AAS?$AAh?$AAo?$AAr?$AAt?$AAP?$AAr?$AAo?$AAg?$AAN?$AAa?$AAm?$AAe?$AA?0?$AA?5?$AA2?$AA6?$AA0?$AA?5?$AA?9@ 00060f38     LIBCMTD:dbgrpt.obj
 0002:0001afd8       ??_C@_1GI@DEDNNLCI@?$AAw?$AAc?$AAs?$AAc?$AAp?$AAy?$AA_?$AAs?$AA?$CI?$AAs?$AAz?$AAE?$AAx?$AAe?$AAN?$AAa?$AAm?$AAe?$AA?0?$AA?5?$AA2?$AA6?$AA0?$AA?0?$AA?5?$AAL?$AA?$CC?$AA?$DM?$AAp?$AAr?$AAo?$AAg@ 00060fd8     LIBCMTD:dbgrpt.obj
 0002:0001b040       ??_C@_1CI@PGJIFDEK@?$AA_?$AA_?$AAc?$AAr?$AAt?$AAM?$AAe?$AAs?$AAs?$AAa?$AAg?$AAe?$AAW?$AAi?$AAn?$AAd?$AAo?$AAw?$AAW?$AA?$AA@ 00061040     LIBCMTD:dbgrpt.obj
 0002:0001b068       ??_C@_1CO@EAEJAADC@?$AA?$DM?$AAp?$AAr?$AAo?$AAg?$AAr?$AAa?$AAm?$AA?5?$AAn?$AAa?$AAm?$AAe?$AA?5?$AAu?$AAn?$AAk?$AAn?$AAo?$AAw?$AAn?$AA?$DO?$AA?$AA@ 00061068     LIBCMTD:dbgrpt.obj
 0002:0001b098       ??_C@_1BM@IIODHMJC@?$AA_?$AAt?$AAz?$AAs?$AAe?$AAt?$AA_?$AAn?$AAo?$AAl?$AAo?$AAc?$AAk?$AA?$AA@ 00061098     LIBCMTD:tzset.obj
 0002:0001b0b8       ??_C@_1FA@HOEHGBHN@?$AAf?$AA?3?$AA?2?$AAs?$AAp?$AA?2?$AAv?$AAc?$AAt?$AAo?$AAo?$AAl?$AAs?$AA?2?$AAc?$AAr?$AAt?$AAc?$AAe?$AA?2?$AAc?$AAr?$AAt?$AAw?$AA3?$AA2?$AA?2?$AAt?$AAi?$AAm?$AAe?$AA?2@ 000610b8     LIBCMTD:tzset.obj
 0002:0001b108       ??_C@_1CA@GOLIIEDM@?$AA_?$AAi?$AAs?$AAi?$AAn?$AAd?$AAs?$AAt?$AA_?$AAn?$AAo?$AAl?$AAo?$AAc?$AAk?$AA?$AA@ 00061108     LIBCMTD:tzset.obj
 0002:0001b128       ??_C@_1BA@GOCKIDGO@?$AAc?$AAv?$AAt?$AAd?$AAa?$AAt?$AAe?$AA?$AA@ 00061128     LIBCMTD:tzset.obj
 0002:0001b138       ??_C@_1DK@DBNCAPPN@?$AA?$CI?$AA?5?$AAc?$AAa?$AAl?$AAt?$AAi?$AAm?$AA?5?$AA?$DM?$AA?$DN?$AA?5?$AA_?$AAM?$AAA?$AAX?$AA_?$AA_?$AAT?$AAI?$AAM?$AAE?$AA6?$AA4?$AA_?$AAT?$AA?5?$AA?$CJ?$AA?$AA@ 00061138     LIBCMTD:gmtime64.obj
 0002:0001b174       ??_C@_1CC@FPMHPAM@?$AA?$CI?$AA?5?$AAt?$AAi?$AAm?$AAp?$AA?5?$AA?$CB?$AA?$DN?$AA?5?$AAN?$AAU?$AAL?$AAL?$AA?5?$AA?$CJ?$AA?$AA@ 00061174     LIBCMTD:gmtime64.obj
 0002:0001b198       ??_C@_1BI@BFNFPMLP@?$AA_?$AAg?$AAm?$AAt?$AAi?$AAm?$AAe?$AA6?$AA4?$AA_?$AAs?$AA?$AA@ 00061198     LIBCMTD:gmtime64.obj
 0002:0001b1b0       ??_C@_1FG@FPNJKKNF@?$AAf?$AA?3?$AA?2?$AAs?$AAp?$AA?2?$AAv?$AAc?$AAt?$AAo?$AAo?$AAl?$AAs?$AA?2?$AAc?$AAr?$AAt?$AAc?$AAe?$AA?2?$AAc?$AAr?$AAt?$AAw?$AA3?$AA2?$AA?2?$AAt?$AAi?$AAm?$AAe?$AA?2@ 000611b0     LIBCMTD:gmtime64.obj
 0002:0001b208       __dnames                   00061208     LIBCMTD:timeset.obj
 0002:0001b220       __mnames                   00061220     LIBCMTD:timeset.obj
 0002:0001b248       ??_C@_1BM@FIMHBHEB@?$AA_?$AAg?$AAe?$AAt?$AA_?$AAd?$AAa?$AAy?$AAl?$AAi?$AAg?$AAh?$AAt?$AA?$AA@ 00061248     LIBCMTD:timeset.obj
 0002:0001b268       ??_C@_1FE@KKMMAEKB@?$AAf?$AA?3?$AA?2?$AAs?$AAp?$AA?2?$AAv?$AAc?$AAt?$AAo?$AAo?$AAl?$AAs?$AA?2?$AAc?$AAr?$AAt?$AAc?$AAe?$AA?2?$AAc?$AAr?$AAt?$AAw?$AA3?$AA2?$AA?2?$AAt?$AAi?$AAm?$AAe?$AA?2@ 00061268     LIBCMTD:timeset.obj
 0002:0001b2bc       ??_C@_1CI@MKJEHFPG@?$AA?$CI?$AA_?$AAD?$AAa?$AAy?$AAl?$AAi?$AAg?$AAh?$AAt?$AA?5?$AA?$CB?$AA?$DN?$AA?5?$AAN?$AAU?$AAL?$AAL?$AA?$CJ?$AA?$AA@ 000612bc     LIBCMTD:timeset.obj
 0002:0001b2e4       ??_C@_1BK@EMODDHEE@?$AA_?$AAg?$AAe?$AAt?$AA_?$AAd?$AAs?$AAt?$AAb?$AAi?$AAa?$AAs?$AA?$AA@ 000612e4     LIBCMTD:timeset.obj
 0002:0001b300       ??_C@_1EC@PKDJPAAB@?$AA?$CI?$AA_?$AAD?$AAa?$AAy?$AAl?$AAi?$AAg?$AAh?$AAt?$AA_?$AAs?$AAa?$AAv?$AAi?$AAn?$AAg?$AAs?$AA_?$AAb?$AAi?$AAa?$AAs?$AA?5?$AA?$CB?$AA?$DN?$AA?5?$AAN?$AAU?$AAL?$AAL?$AA?$CJ@ 00061300     LIBCMTD:timeset.obj
 0002:0001b344       ??_C@_1BM@MGEAKPEJ@?$AA_?$AAg?$AAe?$AAt?$AA_?$AAt?$AAi?$AAm?$AAe?$AAz?$AAo?$AAn?$AAe?$AA?$AA@ 00061344     LIBCMTD:timeset.obj
 0002:0001b360       ??_C@_1CI@PODJJGAL@?$AA?$CI?$AA_?$AAT?$AAi?$AAm?$AAe?$AAz?$AAo?$AAn?$AAe?$AA?5?$AA?$CB?$AA?$DN?$AA?5?$AAN?$AAU?$AAL?$AAL?$AA?$CJ?$AA?$AA@ 00061360     LIBCMTD:timeset.obj
 0002:0001b388       ??_C@_1DM@MADKGDLO@?$AA?$CI?$AAL?$AA?$CC?$AAB?$AAu?$AAf?$AAf?$AAe?$AAr?$AA?5?$AAi?$AAs?$AA?5?$AAt?$AAo?$AAo?$AA?5?$AAs?$AAm?$AAa?$AAl?$AAl?$AA?$CC?$AA?5?$AA?$CG?$AA?$CG?$AA?5?$AA0?$AA?$CJ?$AA?$AA@ 00061388     LIBCMTD:strcpy_s.obj
 0002:0001b3c4       ??_C@_1CI@HCPHDDLE@?$AAB?$AAu?$AAf?$AAf?$AAe?$AAr?$AA?5?$AAi?$AAs?$AA?5?$AAt?$AAo?$AAo?$AA?5?$AAs?$AAm?$AAa?$AAl?$AAl?$AA?$AA@ 000613c4     LIBCMTD:strcpy_s.obj
 0002:0001b3ec       ??_C@_1CG@OFBJMIGJ@?$AA?$CI?$AA?$CI?$AA?$CI?$AA_?$AAS?$AAr?$AAc?$AA?$CJ?$AA?$CJ?$AA?$CJ?$AA?5?$AA?$CB?$AA?$DN?$AA?5?$AAN?$AAU?$AAL?$AAL?$AA?$AA@ 000613ec     LIBCMTD:strcpy_s.obj
 0002:0001b414       ??_C@_1BC@CFJEPFGF@?$AAs?$AAt?$AAr?$AAc?$AAp?$AAy?$AA_?$AAs?$AA?$AA@ 00061414     LIBCMTD:strcpy_s.obj
 0002:0001b428       ??_C@_1FE@IPADLOPJ@?$AAf?$AA?3?$AA?2?$AAs?$AAp?$AA?2?$AAv?$AAc?$AAt?$AAo?$AAo?$AAl?$AAs?$AA?2?$AAc?$AAr?$AAt?$AAc?$AAe?$AA?2?$AAc?$AAr?$AAt?$AAw?$AA3?$AA2?$AA?2?$AAh?$AA?2?$AAt?$AAc?$AAs@ 00061428     LIBCMTD:strcpy_s.obj
 0002:0001b480       ??_C@_1FC@NCPEPIBI@?$AA?$CI?$AA?$CI?$AA_?$AAD?$AAs?$AAt?$AA?$CJ?$AA?$CJ?$AA?5?$AA?$CB?$AA?$DN?$AA?5?$AAN?$AAU?$AAL?$AAL?$AA?5?$AA?$CG?$AA?$CG?$AA?5?$AA?$CI?$AA?$CI?$AA_?$AAS?$AAi?$AAz?$AAe?$AAI?$AAn?$AAB?$AAy?$AAt@ 00061480     LIBCMTD:strcpy_s.obj
 0002:0001b4d4       ??_C@_0BJ@IPHDMCNM@fatal?5error?5in?5_lock?5?$CD0?6?$AA@ 000614d4     LIBCMTD:mlock.obj
 0002:0001b4f0       ??_C@_1NK@LOFHIHFC@?$AAf?$AAM?$AAo?$AAd?$AAe?$AA?5?$AA?$DN?$AA?$DN?$AA?5?$AA_?$AAC?$AAR?$AAT?$AAD?$AAB?$AAG?$AA_?$AAR?$AAE?$AAP?$AAO?$AAR?$AAT?$AA_?$AAM?$AAO?$AAD?$AAE?$AA?5?$AA?$HM?$AA?$HM?$AA?5@ 000614f0     LIBCMTD:dbgrptt.obj
 0002:0001b5cc       ??_C@_1CE@FIHIECNJ@?$AA_?$AAC?$AAr?$AAt?$AAS?$AAe?$AAt?$AAR?$AAe?$AAp?$AAo?$AAr?$AAt?$AAM?$AAo?$AAd?$AAe?$AA?$AA@ 000615cc     LIBCMTD:dbgrptt.obj
 0002:0001b5f0       ??_C@_1FE@PLIBPAGC@?$AAf?$AA?3?$AA?2?$AAs?$AAp?$AA?2?$AAv?$AAc?$AAt?$AAo?$AAo?$AAl?$AAs?$AA?2?$AAc?$AAr?$AAt?$AAc?$AAe?$AA?2?$AAc?$AAr?$AAt?$AAw?$AA3?$AA2?$AA?2?$AAm?$AAi?$AAs?$AAc?$AA?2@ 000615f0     LIBCMTD:dbgrptt.obj
 0002:0001b648       ??_C@_1FA@IFFFOLDJ@?$AAn?$AAR?$AAp?$AAt?$AAT?$AAy?$AAp?$AAe?$AA?5?$AA?$DO?$AA?$DN?$AA?5?$AA0?$AA?5?$AA?$CG?$AA?$CG?$AA?5?$AAn?$AAR?$AAp?$AAt?$AAT?$AAy?$AAp?$AAe?$AA?5?$AA?$DM?$AA?5?$AA_?$AAC?$AAR?$AAT@ 00061648     LIBCMTD:dbgrptt.obj
 0002:0001b698       ??_C@_1CE@IKKEDCME@?$AA_?$AAC?$AAr?$AAt?$AAS?$AAe?$AAt?$AAR?$AAe?$AAp?$AAo?$AAr?$AAt?$AAF?$AAi?$AAl?$AAe?$AA?$AA@ 00061698     LIBCMTD:dbgrptt.obj
 0002:0001b6c0       ??_C@_1MA@LBAMNNOB@?$AAs?$AAt?$AAr?$AAc?$AAp?$AAy?$AA_?$AAs?$AA?$CI?$AAs?$AAz?$AAO?$AAu?$AAt?$AAM?$AAe?$AAs?$AAs?$AAa?$AAg?$AAe?$AA2?$AA?0?$AA?5?$AA4?$AA0?$AA9?$AA6?$AA?0?$AA?5?$AA?$CC?$AA_@ 000616c0     LIBCMTD:dbgrptt.obj
 0002:0001b780       ??_C@_0DP@GNPEPHJD@_CrtDbgReport?3?5String?5too?5long?5o@ 00061780     LIBCMTD:dbgrptt.obj
 0002:0001b7c0       ??_C@_1FI@DBAIJPJE@?$AAw?$AAc?$AAs?$AAc?$AAp?$AAy?$AA_?$AAs?$AA?$CI?$AAs?$AAz?$AAO?$AAu?$AAt?$AAM?$AAe?$AAs?$AAs?$AAa?$AAg?$AAe?$AA?0?$AA?5?$AA4?$AA0?$AA9?$AA6?$AA?0?$AA?5?$AAs?$AAz?$AAL@ 000617c0     LIBCMTD:dbgrptt.obj
 0002:0001b818       ??_C@_1BI@JIDBEPIG@?$AA?$CF?$AAs?$AA?$CI?$AA?$CF?$AAd?$AA?$CJ?$AA?5?$AA?3?$AA?5?$AA?$CF?$AAs?$AA?$AA@ 00061818     LIBCMTD:dbgrptt.obj
 0002:0001b830       ??_C@_1EK@PHCBEDKB@?$AAw?$AAc?$AAs?$AAc?$AAa?$AAt?$AA_?$AAs?$AA?$CI?$AAs?$AAz?$AAL?$AAi?$AAn?$AAe?$AAM?$AAe?$AAs?$AAs?$AAa?$AAg?$AAe?$AA?0?$AA?5?$AA4?$AA0?$AA9?$AA6?$AA?0?$AA?5?$AAL?$AA?$CC@ 00061830     LIBCMTD:dbgrptt.obj
 0002:0001b880       ??_C@_1EK@NMDFGHMF@?$AAw?$AAc?$AAs?$AAc?$AAa?$AAt?$AA_?$AAs?$AA?$CI?$AAs?$AAz?$AAL?$AAi?$AAn?$AAe?$AAM?$AAe?$AAs?$AAs?$AAa?$AAg?$AAe?$AA?0?$AA?5?$AA4?$AA0?$AA9?$AA6?$AA?0?$AA?5?$AAL?$AA?$CC@ 00061880     LIBCMTD:dbgrptt.obj
 0002:0001b8cc       ??_C@_13CMNBPIDO@?$AA?$AN?$AA?$AA@ 000618cc     LIBCMTD:dbgrptt.obj
 0002:0001b8d0       ??_C@_1FK@HPADHBBD@?$AAw?$AAc?$AAs?$AAc?$AAa?$AAt?$AA_?$AAs?$AA?$CI?$AAs?$AAz?$AAL?$AAi?$AAn?$AAe?$AAM?$AAe?$AAs?$AAs?$AAa?$AAg?$AAe?$AA?0?$AA?5?$AA4?$AA0?$AA9?$AA6?$AA?0?$AA?5?$AAs?$AAz@ 000618d0     LIBCMTD:dbgrptt.obj
 0002:0001b930       ??_C@_1KO@DGAHENCH@?$AAw?$AAc?$AAs?$AAc?$AAp?$AAy?$AA_?$AAs?$AA?$CI?$AAs?$AAz?$AAL?$AAi?$AAn?$AAe?$AAM?$AAe?$AAs?$AAs?$AAa?$AAg?$AAe?$AA?0?$AA?5?$AA4?$AA0?$AA9?$AA6?$AA?0?$AA?5?$AAs?$AAz@ 00061930     LIBCMTD:dbgrptt.obj
 0002:0001b9e0       ??_C@_1CE@OJBNHDMO@?$AAA?$AAs?$AAs?$AAe?$AAr?$AAt?$AAi?$AAo?$AAn?$AA?5?$AAf?$AAa?$AAi?$AAl?$AAe?$AAd?$AA?$CB?$AA?$AA@ 000619e0     LIBCMTD:dbgrptt.obj
 0002:0001ba04       ??_C@_1CG@FFFGGODN@?$AAA?$AAs?$AAs?$AAe?$AAr?$AAt?$AAi?$AAo?$AAn?$AA?5?$AAf?$AAa?$AAi?$AAl?$AAe?$AAd?$AA?3?$AA?5?$AA?$AA@ 00061a04     LIBCMTD:dbgrptt.obj
 0002:0001ba30       ??_C@_1JK@KHFABAEO@?$AAw?$AAc?$AAs?$AAc?$AAp?$AAy?$AA_?$AAs?$AA?$CI?$AAs?$AAz?$AAU?$AAs?$AAe?$AAr?$AAM?$AAe?$AAs?$AAs?$AAa?$AAg?$AAe?$AA?0?$AA?5?$AA4?$AA0?$AA9?$AA6?$AA?0?$AA?5?$AAL?$AA?$CC@ 00061a30     LIBCMTD:dbgrptt.obj
 0002:0001bacc       ??_C@_1BA@ELMMDCFC@?$AA?0?$AA?5?$AAL?$AAi?$AAn?$AAe?$AA?5?$AA?$AA@ 00061acc     LIBCMTD:dbgrptt.obj
 0002:0001badc       ??_C@_1BO@OCHMLCAG@?$AA?$DM?$AAf?$AAi?$AAl?$AAe?$AA?5?$AAu?$AAn?$AAk?$AAn?$AAo?$AAw?$AAn?$AA?$DO?$AA?$AA@ 00061adc     LIBCMTD:dbgrptt.obj
 0002:0001bb00       ??_C@_1EM@MJFLEDMB@?$AAS?$AAe?$AAc?$AAo?$AAn?$AAd?$AA?5?$AAC?$AAh?$AAa?$AAn?$AAc?$AAe?$AA?5?$AAA?$AAs?$AAs?$AAe?$AAr?$AAt?$AAi?$AAo?$AAn?$AA?5?$AAF?$AAa?$AAi?$AAl?$AAe?$AAd?$AA?3?$AA?5@ 00061b00     LIBCMTD:dbgrptt.obj
 0002:0001bb50       ??_C@_1FA@CNLLOMHI@?$AA_?$AAi?$AAt?$AAo?$AAw?$AA_?$AAs?$AA?$CI?$AAn?$AAL?$AAi?$AAn?$AAe?$AA?0?$AA?5?$AAs?$AAz?$AAL?$AAi?$AAn?$AAe?$AAM?$AAe?$AAs?$AAs?$AAa?$AAg?$AAe?$AA?0?$AA?5?$AA4?$AA0@ 00061b50     LIBCMTD:dbgrptt.obj
 0002:0001bba0       ??_C@_1CA@HPALHDOD@?$AA_?$AAV?$AAC?$AAr?$AAt?$AAD?$AAb?$AAg?$AAR?$AAe?$AAp?$AAo?$AAr?$AAt?$AAW?$AA?$AA@ 00061ba0     LIBCMTD:dbgrptt.obj
 0002:0001bbc0       ??_C@_1CG@MKBKDNCP@?$AAG?$AAe?$AAt?$AAL?$AAa?$AAs?$AAt?$AAA?$AAc?$AAt?$AAi?$AAv?$AAe?$AAP?$AAo?$AAp?$AAu?$AAp?$AA?$AA@ 00061bc0     LIBCMTD:crtmbox.obj
 0002:0001bbe8       ??_C@_1CA@HNKPMKAN@?$AAG?$AAe?$AAt?$AAA?$AAc?$AAt?$AAi?$AAv?$AAe?$AAW?$AAi?$AAn?$AAd?$AAo?$AAw?$AA?$AA@ 00061be8     LIBCMTD:crtmbox.obj
 0002:0001bc08       ??_C@_1BI@OGPGOOGK@?$AAM?$AAe?$AAs?$AAs?$AAa?$AAg?$AAe?$AAB?$AAo?$AAx?$AAW?$AA?$AA@ 00061c08     LIBCMTD:crtmbox.obj
 0002:0001bc20       ??_C@_1BI@IENOMFML@?$AAC?$AAO?$AAR?$AAE?$AAD?$AAL?$AAL?$AA?4?$AAD?$AAL?$AAL?$AA?$AA@ 00061c20     LIBCMTD:crtmbox.obj
 0002:0001bc38       ??_C@_1BE@PMMBFFCC@?$AAw?$AAc?$AAs?$AAn?$AAc?$AAp?$AAy?$AA_?$AAs?$AA?$AA@ 00061c38     LIBCMTD:wcsncpy_s.obj
 0002:0001bc50       ??_C@_1FG@OHHBDIEA@?$AAf?$AA?3?$AA?2?$AAs?$AAp?$AA?2?$AAv?$AAc?$AAt?$AAo?$AAo?$AAl?$AAs?$AA?2?$AAc?$AAr?$AAt?$AAc?$AAe?$AA?2?$AAc?$AAr?$AAt?$AAw?$AA3?$AA2?$AA?2?$AAh?$AA?2?$AAt?$AAc?$AAs@ 00061c50     LIBCMTD:wcsncpy_s.obj
 0002:0001bca8       ??_C@_1FC@PFMLEHKI@?$AA?$CI?$AA?$CI?$AA_?$AAD?$AAs?$AAt?$AA?$CJ?$AA?$CJ?$AA?5?$AA?$CB?$AA?$DN?$AA?5?$AAN?$AAU?$AAL?$AAL?$AA?5?$AA?$CG?$AA?$CG?$AA?5?$AA?$CI?$AA?$CI?$AA_?$AAS?$AAi?$AAz?$AAe?$AAI?$AAn?$AAW?$AAo?$AAr@ 00061ca8     LIBCMTD:wcsncpy_s.obj
 0002:0001bcfc       ??_C@_1BC@KIONAFPO@?$AAw?$AAc?$AAs?$AAc?$AAp?$AAy?$AA_?$AAs?$AA?$AA@ 00061cfc     LIBCMTD:wcscpy_s.obj
 0002:0001bd10       __newctype                 00061d10     LIBCMTD:ctype.obj
 0002:0001c010       _wctype                    00062010     LIBCMTD:ctype.obj
 0002:0001c218       ??_C@_1FA@MJKDNFFB@?$AA?$CI?$AAL?$AA?$CC?$AAS?$AAt?$AAr?$AAi?$AAn?$AAg?$AA?5?$AAi?$AAs?$AA?5?$AAn?$AAo?$AAt?$AA?5?$AAn?$AAu?$AAl?$AAl?$AA?5?$AAt?$AAe?$AAr?$AAm?$AAi?$AAn?$AAa?$AAt?$AAe?$AAd@ 00062218     LIBCMTD:wcscat_s.obj
 0002:0001c268       ??_C@_1DM@FHLMIEG@?$AAS?$AAt?$AAr?$AAi?$AAn?$AAg?$AA?5?$AAi?$AAs?$AA?5?$AAn?$AAo?$AAt?$AA?5?$AAn?$AAu?$AAl?$AAl?$AA?5?$AAt?$AAe?$AAr?$AAm?$AAi?$AAn?$AAa?$AAt?$AAe?$AAd?$AA?$AA@ 00062268     LIBCMTD:wcscat_s.obj
 0002:0001c2a4       ??_C@_1BC@PLIEPKPJ@?$AAw?$AAc?$AAs?$AAc?$AAa?$AAt?$AA_?$AAs?$AA?$AA@ 000622a4     LIBCMTD:wcscat_s.obj
 0002:0001c2b8       ??_C@_1FE@EHLIBGFJ@?$AAf?$AA?3?$AA?2?$AAs?$AAp?$AA?2?$AAv?$AAc?$AAt?$AAo?$AAo?$AAl?$AAs?$AA?2?$AAc?$AAr?$AAt?$AAc?$AAe?$AA?2?$AAc?$AAr?$AAt?$AAw?$AA3?$AA2?$AA?2?$AAh?$AA?2?$AAt?$AAc?$AAs@ 000622b8     LIBCMTD:wcscat_s.obj
 0002:0001c30c       ??_C@_1CM@HABGDNLJ@?$AAl?$AAe?$AAn?$AAg?$AAt?$AAh?$AA?5?$AA?$DM?$AA?5?$AAs?$AAi?$AAz?$AAe?$AAI?$AAn?$AAT?$AAC?$AAh?$AAa?$AAr?$AAs?$AA?$AA@ 0006230c     LIBCMTD:xtows.obj
 0002:0001c338       ??_C@_1DE@PCJGDBBD@?$AA2?$AA?5?$AA?$DM?$AA?$DN?$AA?5?$AAr?$AAa?$AAd?$AAi?$AAx?$AA?5?$AA?$CG?$AA?$CG?$AA?5?$AAr?$AAa?$AAd?$AAi?$AAx?$AA?5?$AA?$DM?$AA?$DN?$AA?5?$AA3?$AA6?$AA?$AA@ 00062338     LIBCMTD:xtows.obj
 0002:0001c370       ??_C@_1FA@MKGGAGEI@?$AAs?$AAi?$AAz?$AAe?$AAI?$AAn?$AAT?$AAC?$AAh?$AAa?$AAr?$AAs?$AA?5?$AA?$DO?$AA?5?$AA?$CI?$AAs?$AAi?$AAz?$AAe?$AA_?$AAt?$AA?$CJ?$AA?$CI?$AAi?$AAs?$AA_?$AAn?$AAe?$AAg?$AA?5?$AA?$DP@ 00062370     LIBCMTD:xtows.obj
 0002:0001c3c0       ??_C@_1CC@JNJFIMGE@?$AAs?$AAi?$AAz?$AAe?$AAI?$AAn?$AAT?$AAC?$AAh?$AAa?$AAr?$AAs?$AA?5?$AA?$DO?$AA?5?$AA0?$AA?$AA@ 000623c0     LIBCMTD:xtows.obj
 0002:0001c3e4       ??_C@_1O@NCBFODOE@?$AAx?$AAt?$AAo?$AAw?$AA_?$AAs?$AA?$AA@ 000623e4     LIBCMTD:xtows.obj
 0002:0001c3f8       ??_C@_1FE@LAGNOOBA@?$AAf?$AA?3?$AA?2?$AAs?$AAp?$AA?2?$AAv?$AAc?$AAt?$AAo?$AAo?$AAl?$AAs?$AA?2?$AAc?$AAr?$AAt?$AAc?$AAe?$AA?2?$AAc?$AAr?$AAt?$AAw?$AA3?$AA2?$AA?2?$AAc?$AAo?$AAn?$AAv?$AAe@ 000623f8     LIBCMTD:xtows.obj
 0002:0001c44c       ??_C@_1BI@ICGGMGLK@?$AAb?$AAu?$AAf?$AA?5?$AA?$CB?$AA?$DN?$AA?5?$AAN?$AAU?$AAL?$AAL?$AA?$AA@ 0006244c     LIBCMTD:xtows.obj
 0002:0001c760       __IMPORT_DESCRIPTOR_COREDLL 00062760     coredll:COREDLL.dll
 0002:0001c774       __IMPORT_DESCRIPTOR_AYGSHELL 00062774     aygshell:AYGSHELL.dll
 0002:0001c788       __IMPORT_DESCRIPTOR_sw_utilityG 00062788     sw_utilityG:sw_utilityG.dll
 0002:0001c79c       __IMPORT_DESCRIPTOR_GobiApi 0006279c     GobiApi:GobiApi.dll
 0002:0001c7b0       __NULL_IMPORT_DESCRIPTOR   000627b0     coredll:COREDLL.dll
 0003:00000000       __imp_SHInitDialog         00064000     aygshell:AYGSHELL.dll
 0003:00000004       __imp_SHCreateMenuBar      00064004     aygshell:AYGSHELL.dll
 0003:00000008       \177AYGSHELL_NULL_THUNK_DATA 00064008     aygshell:AYGSHELL.dll
 0003:0000000c       __imp_LoadStringW          0006400c     coredll:COREDLL.dll
 0003:00000010       __imp_GetWindowTextW       00064010     coredll:COREDLL.dll
 0003:00000014       __imp_wcsncpy              00064014     coredll:COREDLL.dll
 0003:00000018       __imp_memset               00064018     coredll:COREDLL.dll
 0003:0000001c       __imp_wcscpy               0006401c     coredll:COREDLL.dll
 0003:00000020       __imp_Sleep                00064020     coredll:COREDLL.dll
 0003:00000024       __imp_swprintf             00064024     coredll:COREDLL.dll
 0003:00000028       __imp_SetWindowTextW       00064028     coredll:COREDLL.dll
 0003:0000002c       __imp_GetDlgItem           0006402c     coredll:COREDLL.dll
 0003:00000030       __imp_SetDlgItemInt        00064030     coredll:COREDLL.dll
 0003:00000034       __imp_SetDlgItemTextW      00064034     coredll:COREDLL.dll
 0003:00000038       __imp_EndDialog            00064038     coredll:COREDLL.dll
 0003:0000003c       __imp_MessageBoxW          0006403c     coredll:COREDLL.dll
 0003:00000040       __imp_SetFocus             00064040     coredll:COREDLL.dll
 0003:00000044       __imp_DialogBoxIndirectParamW 00064044     coredll:COREDLL.dll
 0003:00000048       __imp_LoadResource         00064048     coredll:COREDLL.dll
 0003:0000004c       __imp_FindResourceW        0006404c     coredll:COREDLL.dll
 0003:00000050       __imp_GetLastError         00064050     coredll:COREDLL.dll
 0003:00000054       __imp_RegisterClassW       00064054     coredll:COREDLL.dll
 0003:00000058       __imp_GetStockObject       00064058     coredll:COREDLL.dll
 0003:0000005c       __imp_RegisterWindowMessageW 0006405c     coredll:COREDLL.dll
 0003:00000060       __imp_EnableMenuItem       00064060     coredll:COREDLL.dll
 0003:00000064       __imp_wcslen               00064064     coredll:COREDLL.dll
 0003:00000068       __imp_EnableWindow         00064068     coredll:COREDLL.dll
 0003:0000006c       __imp_ShowWindow           0006406c     coredll:COREDLL.dll
 0003:00000070       __imp__wtol                00064070     coredll:COREDLL.dll
 0003:00000074       __imp_PostMessageW         00064074     coredll:COREDLL.dll
 0003:00000078       __imp_PostQuitMessage      00064078     coredll:COREDLL.dll
 0003:0000007c       __imp___rt_sdiv            0006407c     coredll:COREDLL.dll
 0003:00000080       __imp___utos               00064080     coredll:COREDLL.dll
 0003:00000084       __imp___gts                00064084     coredll:COREDLL.dll
 0003:00000088       __imp___ges                00064088     coredll:COREDLL.dll
 0003:0000008c       __imp___les                0006408c     coredll:COREDLL.dll
 0003:00000090       __imp___muls               00064090     coredll:COREDLL.dll
 0003:00000094       __imp___eqs                00064094     coredll:COREDLL.dll
 0003:00000098       __imp___itos               00064098     coredll:COREDLL.dll
 0003:0000009c       __imp___stou               0006409c     coredll:COREDLL.dll
 0003:000000a0       __imp___rt_udiv            000640a0     coredll:COREDLL.dll
 0003:000000a4       __imp___dtos               000640a4     coredll:COREDLL.dll
 0003:000000a8       __imp___utod               000640a8     coredll:COREDLL.dll
 0003:000000ac       __imp___muld               000640ac     coredll:COREDLL.dll
 0003:000000b0       __imp___dtou               000640b0     coredll:COREDLL.dll
 0003:000000b4       __imp___stod               000640b4     coredll:COREDLL.dll
 0003:000000b8       __imp_TerminateThread      000640b8     coredll:COREDLL.dll
 0003:000000bc       __imp_WaitForSingleObject  000640bc     coredll:COREDLL.dll
 0003:000000c0       __imp_CreateThread         000640c0     coredll:COREDLL.dll
 0003:000000c4       __imp_KillTimer            000640c4     coredll:COREDLL.dll
 0003:000000c8       __imp_SetTimer             000640c8     coredll:COREDLL.dll
 0003:000000cc       __imp_MultiByteToWideChar  000640cc     coredll:COREDLL.dll
 0003:000000d0       __imp_SetWindowPos         000640d0     coredll:COREDLL.dll
 0003:000000d4       __imp__wcsicmp             000640d4     coredll:COREDLL.dll
 0003:000000d8       __imp_LeaveCriticalSection 000640d8     coredll:COREDLL.dll
 0003:000000dc       __imp_memcpy               000640dc     coredll:COREDLL.dll
 0003:000000e0       __imp_EnterCriticalSection 000640e0     coredll:COREDLL.dll
 0003:000000e4       __imp___divd               000640e4     coredll:COREDLL.dll
 0003:000000e8       __imp_DeleteCriticalSection 000640e8     coredll:COREDLL.dll
 0003:000000ec       __imp_InitializeCriticalSection 000640ec     coredll:COREDLL.dll
 0003:000000f0       __imp___itod               000640f0     coredll:COREDLL.dll
 0003:000000f4       __imp___ltd                000640f4     coredll:COREDLL.dll
 0003:000000f8       __imp___negd               000640f8     coredll:COREDLL.dll
 0003:000000fc       __imp___dtoi               000640fc     coredll:COREDLL.dll
 0003:00000100       __imp___subd               00064100     coredll:COREDLL.dll
 0003:00000104       __imp_free                 00064104     coredll:COREDLL.dll
 0003:00000108       __imp_strlen               00064108     coredll:COREDLL.dll
 0003:0000010c       __imp_wcstombs             0006410c     coredll:COREDLL.dll
 0003:00000110       __imp_malloc               00064110     coredll:COREDLL.dll
 0003:00000114       __imp_sscanf               00064114     coredll:COREDLL.dll
 0003:00000118       __imp_HideCaret            00064118     coredll:COREDLL.dll
 0003:0000011c       __imp_GetWindowLongW       0006411c     coredll:COREDLL.dll
 0003:00000120       __imp_??2@YAPAXI@Z         00064120     coredll:COREDLL.dll
 0003:00000124       __imp_SetWindowLongW       00064124     coredll:COREDLL.dll
 0003:00000128       __imp_GetParent            00064128     coredll:COREDLL.dll
 0003:0000012c       __imp_CreateWindowExW      0006412c     coredll:COREDLL.dll
 0003:00000130       __imp_DestroyWindow        00064130     coredll:COREDLL.dll
 0003:00000134       __imp_IsWindow             00064134     coredll:COREDLL.dll
 0003:00000138       __imp_wcscmp               00064138     coredll:COREDLL.dll
 0003:0000013c       __imp_wcscat               0006413c     coredll:COREDLL.dll
 0003:00000140       __imp_MessageBeep          00064140     coredll:COREDLL.dll
 0003:00000144       __imp_iswctype             00064144     coredll:COREDLL.dll
 0003:00000148       __imp_OutputDebugStringW   00064148     coredll:COREDLL.dll
 0003:0000014c       __imp_DefWindowProcW       0006414c     coredll:COREDLL.dll
 0003:00000150       __imp_UpdateWindow         00064150     coredll:COREDLL.dll
 0003:00000154       __imp_GetWindowTextLengthW 00064154     coredll:COREDLL.dll
 0003:00000158       __imp_abs                  00064158     coredll:COREDLL.dll
 0003:0000015c       __imp___addd               0006415c     coredll:COREDLL.dll
 0003:00000160       __imp_LoadBitmapW          00064160     coredll:COREDLL.dll
 0003:00000164       __imp_NKDbgPrintfW         00064164     coredll:COREDLL.dll
 0003:00000168       __imp_CloseHandle          00064168     coredll:COREDLL.dll
 0003:0000016c       __imp_SetForegroundWindow  0006416c     coredll:COREDLL.dll
 0003:00000170       __imp_FindWindowW          00064170     coredll:COREDLL.dll
 0003:00000174       __imp_DispatchMessageW     00064174     coredll:COREDLL.dll
 0003:00000178       __imp_TranslateMessage     00064178     coredll:COREDLL.dll
 0003:0000017c       __imp_GetMessageW          0006417c     coredll:COREDLL.dll
 0003:00000180       __imp_CreateMutexW         00064180     coredll:COREDLL.dll
 0003:00000184       __imp_LoadLibraryW         00064184     coredll:COREDLL.dll
 0003:00000188       __imp__wcsupr              00064188     coredll:COREDLL.dll
 0003:0000018c       __imp__isctype             0006418c     coredll:COREDLL.dll
 0003:00000190       __imp_SendDlgItemMessageW  00064190     coredll:COREDLL.dll
 0003:00000194       __imp__wtoll               00064194     coredll:COREDLL.dll
 0003:00000198       __imp_wsprintfW            00064198     coredll:COREDLL.dll
 0003:0000019c       __imp_SetActiveWindow      0006419c     coredll:COREDLL.dll
 0003:000001a0       __imp_??3@YAXPAX@Z         000641a0     coredll:COREDLL.dll
 0003:000001a4       __imp_GetClientRect        000641a4     coredll:COREDLL.dll
 0003:000001a8       __imp_SendMessageW         000641a8     coredll:COREDLL.dll
 0003:000001ac       __imp_SetLastError         000641ac     coredll:COREDLL.dll
 0003:000001b0       __imp_GetProcAddressW      000641b0     coredll:COREDLL.dll
 0003:000001b4       __imp_InterlockedIncrement 000641b4     coredll:COREDLL.dll
 0003:000001b8       __imp_TerminateProcess     000641b8     coredll:COREDLL.dll
 0003:000001bc       __imp__vsnwprintf          000641bc     coredll:COREDLL.dll
 0003:000001c0       __imp_WriteFile            000641c0     coredll:COREDLL.dll
 0003:000001c4       __imp_InterlockedDecrement 000641c4     coredll:COREDLL.dll
 0003:000001c8       __imp_RaiseException       000641c8     coredll:COREDLL.dll
 0003:000001cc       __imp_GetTimeZoneInformation 000641cc     coredll:COREDLL.dll
 0003:000001d0       __imp_WideCharToMultiByte  000641d0     coredll:COREDLL.dll
 0003:000001d4       __imp_GetModuleFileNameW   000641d4     coredll:COREDLL.dll
 0003:000001d8       __imp__snwprintf           000641d8     coredll:COREDLL.dll
 0003:000001dc       __imp_GetDateFormatW       000641dc     coredll:COREDLL.dll
 0003:000001e0       __imp_GetTimeFormatW       000641e0     coredll:COREDLL.dll
 0003:000001e4       __imp__stricmp             000641e4     coredll:COREDLL.dll
 0003:000001e8       __imp___rt_srem64by64      000641e8     coredll:COREDLL.dll
 0003:000001ec       __imp___rt_sdiv64by64      000641ec     coredll:COREDLL.dll
 0003:000001f0       __imp_mbstowcs             000641f0     coredll:COREDLL.dll
 0003:000001f4       __imp___security_gen_cookie 000641f4     coredll:COREDLL.dll
 0003:000001f8       __imp_LocalFree            000641f8     coredll:COREDLL.dll
 0003:000001fc       __imp___report_gsfailure   000641fc     coredll:COREDLL.dll
 0003:00000200       __imp___C_specific_handler 00064200     coredll:COREDLL.dll
 0003:00000204       __imp__XcptFilter          00064204     coredll:COREDLL.dll
 0003:00000208       \177COREDLL_NULL_THUNK_DATA 00064208     coredll:COREDLL.dll
 0003:0000020c       __imp_GetConfig            0006420c     GobiApi:GobiApi.dll
 0003:00000210       __imp_GetTxRxInfo          00064210     GobiApi:GobiApi.dll
 0003:00000214       __imp_GetRFInfo            00064214     GobiApi:GobiApi.dll
 0003:00000218       __imp_GetHdrColorCode      00064218     GobiApi:GobiApi.dll
 0003:0000021c       __imp_SwiGetHrpdStats      0006421c     GobiApi:GobiApi.dll
 0003:00000220       __imp_GetANAAAAuthenticationStatus 00064220     GobiApi:GobiApi.dll
 0003:00000224       __imp_SwiGetSignalStrengthInfo 00064224     GobiApi:GobiApi.dll
 0003:00000228       __imp_GetErrRate           00064228     GobiApi:GobiApi.dll
 0003:0000022c       __imp_SwiGetCdmaDominantPn 0006422c     GobiApi:GobiApi.dll
 0003:00000230       __imp_QCWWANConnect        00064230     GobiApi:GobiApi.dll
 0003:00000234       __imp_GetPRLVersion        00064234     GobiApi:GobiApi.dll
 0003:00000238       __imp_GetHardwareRevision  00064238     GobiApi:GobiApi.dll
 0003:0000023c       __imp_GetFirmwareRevisions 0006423c     GobiApi:GobiApi.dll
 0003:00000240       __imp_GetModelID           00064240     GobiApi:GobiApi.dll
 0003:00000244       __imp_GetSysInfo           00064244     GobiApi:GobiApi.dll
 0003:00000248       __imp_SetDdtmPreference    00064248     GobiApi:GobiApi.dll
 0003:0000024c       __imp_SetConfig            0006424c     GobiApi:GobiApi.dll
 0003:00000250       \177GobiApi_NULL_THUNK_DATA 00064250     GobiApi:GobiApi.dll
 0003:00000254       __imp_GetPTMode            00064254     sw_utilityG:sw_utilityG.dll
 0003:00000258       __imp_StopPTMode           00064258     sw_utilityG:sw_utilityG.dll
 0003:0000025c       __imp_StopDMMode           0006425c     sw_utilityG:sw_utilityG.dll
 0003:00000260       __imp_StartPTMode          00064260     sw_utilityG:sw_utilityG.dll
 0003:00000264       __imp_StartDMMode          00064264     sw_utilityG:sw_utilityG.dll
 0003:00000268       __imp_?GetResolution@@YAHXZ 00064268     sw_utilityG:sw_utilityG.dll
 0003:0000026c       __imp_?GetCarrierIndex@@YAKXZ 0006426c     sw_utilityG:sw_utilityG.dll
 0003:00000270       __imp_?InitLog@@YAXPAUHINSTANCE__@@@Z 00064270     sw_utilityG:sw_utilityG.dll
 0003:00000274       __imp_GetRilStatus         00064274     sw_utilityG:sw_utilityG.dll
 0003:00000278       __imp_ValidateSpc          00064278     sw_utilityG:sw_utilityG.dll
 0003:0000027c       __imp_StartDebugMode       0006427c     sw_utilityG:sw_utilityG.dll
 0003:00000280       __imp_StopDebugMode        00064280     sw_utilityG:sw_utilityG.dll
 0003:00000284       __imp_EnableTechHdrNotifications 00064284     sw_utilityG:sw_utilityG.dll
 0003:00000288       __imp_GetRilDebugInfo      00064288     sw_utilityG:sw_utilityG.dll
 0003:0000028c       __imp_InitiateHostBoot     0006428c     sw_utilityG:sw_utilityG.dll
 0003:00000290       __imp_RtnReset             00064290     sw_utilityG:sw_utilityG.dll
 0003:00000294       __imp_GetDMMode            00064294     sw_utilityG:sw_utilityG.dll
 0003:00000298       __imp_SetSIPNaiPassword    00064298     sw_utilityG:sw_utilityG.dll
 0003:0000029c       __imp_ModGetHDRHybrPrefMode 0006429c     sw_utilityG:sw_utilityG.dll
 0003:000002a0       __imp_ModGetSysPrefMode    000642a0     sw_utilityG:sw_utilityG.dll
 0003:000002a4       __imp_ModGetRoamingMode    000642a4     sw_utilityG:sw_utilityG.dll
 0003:000002a8       __imp_ModSetRoamingMode    000642a8     sw_utilityG:sw_utilityG.dll
 0003:000002ac       __imp_ModSetSysPrefMode    000642ac     sw_utilityG:sw_utilityG.dll
 0003:000002b0       __imp_ModSetHDRHybrPrefMode 000642b0     sw_utilityG:sw_utilityG.dll
 0003:000002b4       __imp_GetDsMipList         000642b4     sw_utilityG:sw_utilityG.dll
 0003:000002b8       __imp_GetDsMipProfile      000642b8     sw_utilityG:sw_utilityG.dll
 0003:000002bc       __imp_?THtoT@@YAXPAG0H@Z   000642bc     sw_utilityG:sw_utilityG.dll
 0003:000002c0       __imp_?DisplayRawData@@YAXIPAEHPBG@Z 000642c0     sw_utilityG:sw_utilityG.dll
 0003:000002c4       __imp_?TtoTH@@YAXPAG0H@Z   000642c4     sw_utilityG:sw_utilityG.dll
 0003:000002c8       __imp_SetHdrNaiPassword    000642c8     sw_utilityG:sw_utilityG.dll
 0003:000002cc       __imp_SetDsMipProfile      000642cc     sw_utilityG:sw_utilityG.dll
 0003:000002d0       __imp_GetVersionInfo       000642d0     sw_utilityG:sw_utilityG.dll
 0003:000002d4       __imp_GetProvisionState    000642d4     sw_utilityG:sw_utilityG.dll
 0003:000002d8       __imp_GetCallstate         000642d8     sw_utilityG:sw_utilityG.dll
 0003:000002dc       __imp_GetMDNLengthSupported 000642dc     sw_utilityG:sw_utilityG.dll
 0003:000002e0       __imp_GetProvisionInfo     000642e0     sw_utilityG:sw_utilityG.dll
 0003:000002e4       __imp_SetProvisionInfo     000642e4     sw_utilityG:sw_utilityG.dll
 0003:000002e8       __imp_?LogW@@YAXPBGZZ      000642e8     sw_utilityG:sw_utilityG.dll
 0003:000002ec       __imp_DialEx               000642ec     sw_utilityG:sw_utilityG.dll
 0003:000002f0       __imp_HangUp               000642f0     sw_utilityG:sw_utilityG.dll
 0003:000002f4       __imp_?GetProductFeatures@@YAHAAK@Z 000642f4     sw_utilityG:sw_utilityG.dll
 0003:000002f8       __imp_SelectGSMBand        000642f8     sw_utilityG:sw_utilityG.dll
 0003:000002fc       __imp_GetCurrentGSMBandAndList 000642fc     sw_utilityG:sw_utilityG.dll
 0003:00000300       __imp_GetItemnizedUMTSInfo 00064300     sw_utilityG:sw_utilityG.dll
 0003:00000304       __imp_?RelayoutDialog@@YAHPAUHINSTANCE__@@PAUHWND__@@PBG@Z 00064304     sw_utilityG:sw_utilityG.dll
 0003:00000308       __imp_GetGSMInfo           00064308     sw_utilityG:sw_utilityG.dll
 0003:0000030c       __imp_SetPDSMPAParam       0006430c     sw_utilityG:sw_utilityG.dll
 0003:00000310       __imp_ReadPDSMPAParam      00064310     sw_utilityG:sw_utilityG.dll
 0003:00000314       __imp_GetSIPNaiPassword    00064314     sw_utilityG:sw_utilityG.dll
 0003:00000318       __imp_GetRilPAParam        00064318     sw_utilityG:sw_utilityG.dll
 0003:0000031c       __imp_?IP2DWORD@@YAKPBG@Z  0006431c     sw_utilityG:sw_utilityG.dll
 0003:00000320       __imp_?DWORD2IP@@YAPBGK@Z  00064320     sw_utilityG:sw_utilityG.dll
 0003:00000324       __imp_StopPDSMLocNotifstatus 00064324     sw_utilityG:sw_utilityG.dll
 0003:00000328       __imp_StopPDSMDldNotifstatus 00064328     sw_utilityG:sw_utilityG.dll
 0003:0000032c       __imp_StartPDSMLocNotifstatus 0006432c     sw_utilityG:sw_utilityG.dll
 0003:00000330       __imp_StartPDSMDldNotifstatus 00064330     sw_utilityG:sw_utilityG.dll
 0003:00000334       __imp_StartLBTrackSession  00064334     sw_utilityG:sw_utilityG.dll
 0003:00000338       __imp_EndLBTrackSession    00064338     sw_utilityG:sw_utilityG.dll
 0003:0000033c       __imp_ReadPDSMPAData       0006433c     sw_utilityG:sw_utilityG.dll
 0003:00000340       __imp_GetRilPDData         00064340     sw_utilityG:sw_utilityG.dll
 0003:00000344       __imp_?InWideMode@@YAHXZ   00064344     sw_utilityG:sw_utilityG.dll
 0003:00000348       __imp_GetByteCounter       00064348     sw_utilityG:sw_utilityG.dll
 0003:0000034c       __imp_?WriteLog@@YAXKPBGZZ 0006434c     sw_utilityG:sw_utilityG.dll
 0003:00000350       __imp_SaveAkey             00064350     sw_utilityG:sw_utilityG.dll
 0003:00000354       __imp_?SetLimitText@@YAJPAUHWND__@@H@Z 00064354     sw_utilityG:sw_utilityG.dll
 0003:00000358       __imp_GetAdvancedMenuInfo  00064358     sw_utilityG:sw_utilityG.dll
 0003:0000035c       __imp_SetEquipmentState    0006435c     sw_utilityG:sw_utilityG.dll
 0003:00000360       __imp_?SetWaitCursor@@YAXXZ 00064360     sw_utilityG:sw_utilityG.dll
 0003:00000364       __imp_ReadNv               00064364     sw_utilityG:sw_utilityG.dll
 0003:00000368       __imp_WriteNv              00064368     sw_utilityG:sw_utilityG.dll
 0003:0000036c       __imp_?LogStoreFileLine@@YAXPAGH@Z 0006436c     sw_utilityG:sw_utilityG.dll
 0003:00000370       __imp_?LogC@@YAXPBGZZ      00064370     sw_utilityG:sw_utilityG.dll
 0003:00000374       __imp_?SetNormalCursor@@YAXXZ 00064374     sw_utilityG:sw_utilityG.dll
 0003:00000378       \177sw_utilityG_NULL_THUNK_DATA 00064378     sw_utilityG:sw_utilityG.dll
 0003:0000037c       __xc_a                     0006437c     corelibc:crt0init.obj
 0003:000009b4       __xc_z                     000649b4     corelibc:crt0init.obj
 0003:000009b8       __xi_a                     000649b8     corelibc:crt0init.obj
 0003:000009bc       __xi_z                     000649bc     corelibc:crt0init.obj
 0003:000009c0       __xp_a                     000649c0     corelibc:crt0init.obj
 0003:000009c4       __xp_z                     000649c4     corelibc:crt0init.obj
 0003:000009c8       __xt_a                     000649c8     corelibc:crt0init.obj
 0003:000009cc       __xt_z                     000649cc     corelibc:crt0init.obj
 0003:000009d0       ?g_szAdvanceClass@@3PAGA   000649d0     advanceddlg.obj
 0003:000009d4       ?g_szAuthKeyClass@@3PAGA   000649d4     authkey.obj
 0003:000009d8       ?g_szBrowserDlgClass@@3PAGA 000649d8     browserdlg.obj
 0003:000009dc       ?g_szBWMeterClass@@3PAGA   000649dc     bwmeterdlg.obj
 0003:000009e0       ?g_fTxDiv@@3MA             000649e0     bwmeterdlg.obj
 0003:000009e4       ?g_fRxDiv@@3MA             000649e4     bwmeterdlg.obj
 0003:000009e8       ?szBWMList@@3PAPBGA        000649e8     bwmeterdlg.obj
 0003:000009fc       ?g_szConfigClass@@3PAGA    000649fc     configdlg.obj
 0003:00000a00       ?g_szEVDODlgClass@@3PAGA   00064a00     evdo.obj
 0003:00000a04       ?g_szFingerClass@@3PAGA    00064a04     finger.obj
 0003:00000a08       ?g_szGPSDataClass@@3PAGA   00064a08     gpsdatadlg.obj
 0003:00000a0c       ?g_dwMaxDelay@@3KA         00064a0c     gpsdatadlg.obj
 0003:00000a10       ?g_dwEditFixCount@@3KA     00064a10     gpsdatadlg.obj
 0003:00000a14       ?g_dwFixType@@3KA          00064a14     gpsdatadlg.obj
 0003:00000a18       ?g_bStart@@3HA             00064a18     gpsdatadlg.obj
 0003:00000a1c       ?g_szGPSSettingsClass@@3PAGA 00064a1c     gpssettingsdlg.obj
 0003:00000a20       ?g_szGSM2GClass@@3PAGA     00064a20     gsm2G.obj
 0003:00000a24       ?g_szGSM3GClass@@3PAGA     00064a24     gsm3G.obj
 0003:00000a28       ?g_szGSM3GItemnizeClass@@3PAGA 00064a28     gsm3G.obj
 0003:00000a2c       ?g_szGSMBandClass@@3PAGA   00064a2c     gsmband.obj
 0003:00000a30       ?g_szIOTAClass@@3PAGA      00064a30     iota.obj
 0003:00000a34       ?g_szLoopBackDlgClass@@3PAGA 00064a34     loopbackdlg.obj
 0003:00000a38       ?g_szMslClass@@3PAGA       00064a38     msldlg.obj
 0003:00000a3c       ?g_szNetworkClass@@3PAGA   00064a3c     network.obj
 0003:00000a40       ?g_szOtkslClass@@3PAGA     00064a40     otksldlg.obj
 0003:00000a44       ?g_szPassThruClass@@3PAGA  00064a44     passthrudlg.obj
 0003:00000a48       ?g_bPasstruStart@@3HA      00064a48     passthrudlg.obj
 0003:00000a4c       ?g_szAppWndClass@@3PBGB    00064a4c     PhoneUtility.obj
 0003:00000a50       ?g_szRTNClass@@3PAGA       00064a50     rtndlg.obj
 0003:00000a54       ?g_szSimpleIPClass@@3PAGA  00064a54     simpleipdlg.obj
 0003:00000a58       ?g_dwPreference@@3KA       00064a58     simpleipdlg.obj
 0003:00000a5c       ?szSimpleIPList@@3PAPBGA   00064a5c     simpleipdlg.obj
 0003:00000a68       ?g_szSipDlgClass@@3PAGA    00064a68     sipdlg.obj
 0003:00000a6c       ?g_szSPCValidationClass@@3PAGA 00064a6c     spcvalidation.obj
 0003:00000a70       ?g_szSystemDlgClass@@3PAGA 00064a70     systemdlg.obj
 0003:00000a74       ?g_szUsernameClass@@3PAGA  00064a74     usernamedlg.obj
 0003:00000a7c       ?g_szVersionInfoDlgClass@@3PAGA 00064a7c     versioninfo.obj
 0003:00000a80       ?g_szVocoderDlgClass@@3PAGA 00064a80     vocoderdlg.obj
 0003:00000a84       ?g_wHomePageVoiceSO@@3GA   00064a84     vocoderdlg.obj
 0003:00000a88       ?g_wHomeOrigVoiceSO@@3GA   00064a88     vocoderdlg.obj
 0003:00000a8c       ?g_wRoamOrigVoiceSO@@3GA   00064a8c     vocoderdlg.obj
 0003:00000a90       __security_cookie_complement 00064a90     corelibc:seccook.obj
 0003:00000a94       __security_cookie          00064a94     corelibc:seccook.obj
 0003:00000a98       __lc_time_c                00064a98     LIBCMTD:strftime.obj
 0003:00000b50       __lc_time_curr             00064b50     LIBCMTD:strftime.obj
 0003:00000b80       _timezone                  00064b80     LIBCMTD:timeset.obj
 0003:00000b84       _daylight                  00064b84     LIBCMTD:timeset.obj
 0003:00000b88       _dstbias                   00064b88     LIBCMTD:timeset.obj
 0003:00000c10       _tzname                    00064c10     LIBCMTD:timeset.obj
 0003:00000c18       __clocalestr               00064c18     LIBCMTD:nlsdata2.obj
 0003:00000c20       __initiallocinfo           00064c20     LIBCMTD:nlsdata2.obj
 0003:00000cf0       __ptlocinfo                00064cf0     LIBCMTD:nlsdata2.obj
 0003:00000cf4       __lc_clike                 00064cf4     LIBCMTD:nlsdata2.obj
 0003:00000cf8       _lpdays                    00064cf8     LIBCMTD:days.obj
 0003:00000d2c       _days                      00064d2c     LIBCMTD:days.obj
 0003:00000e80       _crtAssertBusy             00064e80     LIBCMTD:dbgrptt.obj
 0003:00000e84       _CrtDbgMode                00064e84     LIBCMTD:dbgrptt.obj
 0003:00000e90       _CrtDbgFile                00064e90     LIBCMTD:dbgrptt.obj
 0003:00000e9c       _pctype                    00064e9c     LIBCMTD:ctype.obj
 0003:00000ea0       _pwctype                   00064ea0     LIBCMTD:ctype.obj
 0003:00000ea4       __lconv_static_decimal     00064ea4     LIBCMTD:lconv.obj
 0003:00000ea8       __lconv_c                  00064ea8     LIBCMTD:lconv.obj
 0003:00000ed8       _aexit_rtn                 00064ed8     LIBCMTD:crt0dat.obj
 0003:00000ee0       ?g_szLockCode@@3PAGA       00064ee0     advanceddlg.obj
 0003:000010e0       ?g_hWndLBOrg@@3PAUHWND__@@A 000650e0     advanceddlg.obj
 0003:000010e4       ?g_hWndLBSID@@3PAUHWND__@@A 000650e4     advanceddlg.obj
 0003:000010e8       ?g_hWndLBNID@@3PAUHWND__@@A 000650e8     advanceddlg.obj
 0003:000010ec       ?g_hWndLBHSys@@3PAUHWND__@@A 000650ec     advanceddlg.obj
 0003:000010f0       ?g_hWndCAIRev@@3PAUHWND__@@A 000650f0     advanceddlg.obj
 0003:000010f4       ?g_hWndSCM@@3PAUHWND__@@A  000650f4     advanceddlg.obj
 0003:000010f8       ?g_hWndCameraUrl@@3PAUHWND__@@A 000650f8     advanceddlg.obj
 0003:000010fc       ?g_hWndLockCode@@3PAUHWND__@@A 000650fc     advanceddlg.obj
 0003:00001100       ?g_hWndNIDUPDOWN@@3PAUHWND__@@A 00065100     advanceddlg.obj
 0003:00001104       ?g_hWndSIDUPDOWN@@3PAUHWND__@@A 00065104     advanceddlg.obj
 0003:00001108       ?g_hWndHSYSUPDOWN@@3PAUHWND__@@A 00065108     advanceddlg.obj
 0003:0000110c       ?g_hWndORGUPDOWN@@3PAUHWND__@@A 0006510c     advanceddlg.obj
 0003:00001110       ?g_hListDDTM@@3PAUHWND__@@A 00065110     advanceddlg.obj
 0003:00001114       ?g_dwAdvCAIRev@@3KA        00065114     advanceddlg.obj
 0003:00001118       ?g_dwHomeOrg@@3KA          00065118     advanceddlg.obj
 0003:0000111c       ?g_dwFNID@@3HA             0006511c     advanceddlg.obj
 0003:00001120       ?g_dwFSID@@3HA             00065120     advanceddlg.obj
 0003:00001124       ?g_dwHSYSReg@@3HA          00065124     advanceddlg.obj
 0003:00001128       ?g_dwSCM@@3KA              00065128     advanceddlg.obj
 0003:00001130       ?g_dwSaveResult@@3KA       00065130     authkey.obj
 0003:00001134       ?g_bMNCode@@3HA            00065134     authkey.obj
 0003:00001138       ?g_bAkey@@3HA              00065138     authkey.obj
 0003:0000113c       ?g_hAkeyMenu@@3PAUHWND__@@A 0006513c     authkey.obj
 0003:0000114c       ?g_stRilByteCounterInfo@@3Urilbytecounter_tag@@A 0006514c     bwmeterdlg.obj
 0003:00001160       ?g_stCallType@@3KA         00065160     bwmeterdlg.obj
 0003:00001164       ?g_hWndLBMaxRX@@3PAUHWND__@@A 00065164     bwmeterdlg.obj
 0003:00001168       ?g_hWndLBMaxTX@@3PAUHWND__@@A 00065168     bwmeterdlg.obj
 0003:0000116c       ?g_hThread@@3PAXA          0006516c     bwmeterdlg.obj
 0003:00001170       ?g_dwRxNow@@3KA            00065170     bwmeterdlg.obj
 0003:00001174       ?g_dwTxNow@@3KA            00065174     bwmeterdlg.obj
 0003:00001178       ?g_dwCurrentHighRxCur@@3KA 00065178     bwmeterdlg.obj
 0003:0000117c       ?g_dwCurrentHighTxCur@@3KA 0006517c     bwmeterdlg.obj
 0003:00001180       ?g_dwRxCount@@3KA          00065180     bwmeterdlg.obj
 0003:00001184       ?g_dwTxCount@@3KA          00065184     bwmeterdlg.obj
 0003:00001188       ?g_dwHighTxAvg@@3KA        00065188     bwmeterdlg.obj
 0003:0000118c       ?g_dwHighRxAvg@@3KA        0006518c     bwmeterdlg.obj
 0003:00001190       ?g_hWndStatMaxTX@@3PAUHWND__@@A 00065190     bwmeterdlg.obj
 0003:00001194       ?g_hWndStatMaxRX@@3PAUHWND__@@A 00065194     bwmeterdlg.obj
 0003:00001198       ?g_hProgressTxAvg@@3PAUHWND__@@A 00065198     bwmeterdlg.obj
 0003:0000119c       ?g_hProgressRxAvg@@3PAUHWND__@@A 0006519c     bwmeterdlg.obj
 0003:000011a0       ?g_hProgressTx@@3PAUHWND__@@A 000651a0     bwmeterdlg.obj
 0003:000011a4       ?g_hProgressRx@@3PAUHWND__@@A 000651a4     bwmeterdlg.obj
 0003:000011a8       ?g_hStaticTxVal@@3PAUHWND__@@A 000651a8     bwmeterdlg.obj
 0003:000011ac       ?g_hStaticRxVal@@3PAUHWND__@@A 000651ac     bwmeterdlg.obj
 0003:000011b0       ?g_hStaticTxAvg@@3PAUHWND__@@A 000651b0     bwmeterdlg.obj
 0003:000011b4       ?g_hStaticRxAvg@@3PAUHWND__@@A 000651b4     bwmeterdlg.obj
 0003:000011b8       ?g_hStaticHighTxCur@@3PAUHWND__@@A 000651b8     bwmeterdlg.obj
 0003:000011bc       ?g_hStaticHighTxAvg@@3PAUHWND__@@A 000651bc     bwmeterdlg.obj
 0003:000011c0       ?g_hStaticHighRxCur@@3PAUHWND__@@A 000651c0     bwmeterdlg.obj
 0003:000011c4       ?g_hStaticHighRxAvg@@3PAUHWND__@@A 000651c4     bwmeterdlg.obj
 0003:000011c8       ?g_hStaticTxBytes@@3PAUHWND__@@A 000651c8     bwmeterdlg.obj
 0003:000011cc       ?g_hStaticRxBytes@@3PAUHWND__@@A 000651cc     bwmeterdlg.obj
 0003:000011d0       ?g_fRxAvg@@3MA             000651d0     bwmeterdlg.obj
 0003:000011d4       ?g_fTxAvg@@3MA             000651d4     bwmeterdlg.obj
 0003:000011d8       ?g_bExitThread@@3_NA       000651d8     bwmeterdlg.obj
 0003:000011dc       ?g_dwRxBytes@@3KA          000651dc     bwmeterdlg.obj
 0003:000011e0       ?g_dwTxBytes@@3KA          000651e0     bwmeterdlg.obj
 0003:000011e8       ?m_bInitFailed@CAtlBaseModule@ATL@@2_NA 000651e8     configdlg.obj
 0003:000011ec       ?s_pLog@CFixedStringMgr@ATL@@2PAVIFixedStringLog@2@A 000651ec     configdlg.obj
 0003:000012e0       ?g_PhUpdateEvdo@@3UCRITICAL_SECTION@@A 000652e0     evdo.obj
 0003:000012f4       ?g_hWndEvdoList@@3PAUHWND__@@A 000652f4     evdo.obj
 0003:000012fc       ?g_hFingerList@@3PAUHWND__@@A 000652fc     finger.obj
 0003:00001300       ?g_hActivestList@@3PAUHWND__@@A 00065300     finger.obj
 0003:00001310       ?g_szEditEndReason@@3PAGA  00065310     gpsdatadlg.obj
 0003:000017c0       ?g_szEditSessionStatus@@3PAGA 000657c0     gpsdatadlg.obj
 0003:00001c70       ?g_szEditLongitude@@3PAGA  00065c70     gpsdatadlg.obj
 0003:00002120       ?g_szEditLatitude@@3PAGA   00066120     gpsdatadlg.obj
 0003:000025d0       ?g_szEditLocTime@@3PAGA    000665d0     gpsdatadlg.obj
 0003:00002a80       ?g_PDSMPDEndSession@@3UtagRILPDSMPDEndSession@@A 00066a80     gpsdatadlg.obj
 0003:00002a88       ?g_PDSMPDTrack@@3UtagRILPDSMPATrack@@A 00066a88     gpsdatadlg.obj
 0003:00002aa0       ?g_PDSMPDData@@3UtagRILGETPAData@@A 00066aa0     gpsdatadlg.obj
 0003:00002adc       ?g_hEditStatus@@3PAUHWND__@@A 00066adc     gpsdatadlg.obj
 0003:00002ae0       ?g_hEditEndReason@@3PAUHWND__@@A 00066ae0     gpsdatadlg.obj
 0003:00002ae4       ?g_hEditTime@@3PAUHWND__@@A 00066ae4     gpsdatadlg.obj
 0003:00002ae8       ?g_hEditLatitude@@3PAUHWND__@@A 00066ae8     gpsdatadlg.obj
 0003:00002aec       ?g_hEditLongitude@@3PAUHWND__@@A 00066aec     gpsdatadlg.obj
 0003:00002af0       ?g_hFixType@@3PAUHWND__@@A 00066af0     gpsdatadlg.obj
 0003:00002af4       ?g_hFixTypeUpDn@@3PAUHWND__@@A 00066af4     gpsdatadlg.obj
 0003:00002af8       ?g_hEditMaxDelay@@3PAUHWND__@@A 00066af8     gpsdatadlg.obj
 0003:00002afc       ?g_hEDTMaxErrs@@3PAUHWND__@@A 00066afc     gpsdatadlg.obj
 0003:00002b00       ?g_hEDTFixRate@@3PAUHWND__@@A 00066b00     gpsdatadlg.obj
 0003:00002b04       ?g_hEDTFixCt@@3PAUHWND__@@A 00066b04     gpsdatadlg.obj
 0003:00002b08       ?g_dwMaxError@@3KA         00066b08     gpsdatadlg.obj
 0003:00002b0c       ?g_dwEditFixRate@@3KA      00066b0c     gpsdatadlg.obj
 0003:00002b24       ?g_stGetPDSMPAParam@@3UtagRILSETGETPAParam@@A 00066b24     gpssettingsdlg.obj
 0003:00002b48       ?g_hLBGPSLock@@3PAUHWND__@@A 00066b48     gpssettingsdlg.obj
 0003:00002b4c       ?g_hLBTMech@@3PAUHWND__@@A 00066b4c     gpssettingsdlg.obj
 0003:00002b50       ?g_hLBPrivacy@@3PAUHWND__@@A 00066b50     gpssettingsdlg.obj
 0003:00002b54       ?g_hLBNTACCSLVL@@3PAUHWND__@@A 00066b54     gpssettingsdlg.obj
 0003:00002b58       ?g_hLBGPSLockUPDN@@3PAUHWND__@@A 00066b58     gpssettingsdlg.obj
 0003:00002b5c       ?g_hLBTMechUPDN@@3PAUHWND__@@A 00066b5c     gpssettingsdlg.obj
 0003:00002b60       ?g_hLBPrivacyUPDN@@3PAUHWND__@@A 00066b60     gpssettingsdlg.obj
 0003:00002b64       ?g_hLBNTACCSLVLUPDN@@3PAUHWND__@@A 00066b64     gpssettingsdlg.obj
 0003:00002b68       ?g_hEDTIP@@3PAUHWND__@@A   00066b68     gpssettingsdlg.obj
 0003:00002b6c       ?g_hEDTPort@@3PAUHWND__@@A 00066b6c     gpssettingsdlg.obj
 0003:00002b70       ?g_hFixRate@@3PAUHWND__@@A 00066b70     gpssettingsdlg.obj
 0003:00002b74       ?g_hAutoTrack@@3PAUHWND__@@A 00066b74     gpssettingsdlg.obj
 0003:00002b78       ?g_hFixMode@@3PAUHWND__@@A 00066b78     gpssettingsdlg.obj
 0003:00002b7c       ?g_u2GTimer@@3IA           00066b7c     gsm2G.obj
 0003:00002c70       ?g_u3GTimer@@3IA           00066c70     gsm3G.obj
 0003:00002c74       ?g_lIndex@@3JA             00066c74     gsm3G.obj
 0003:00002e5c       ?m_hMenuConnect@@3PAUHWND__@@A 00066e5c     loopbackdlg.obj
 0003:00002e60       ?m_hMenuDisConnect@@3PAUHWND__@@A 00066e60     loopbackdlg.obj
 0003:00002e64       ?g_hstatMsg@@3PAUHWND__@@A 00066e64     loopbackdlg.obj
 0003:00002e68       ?g_dwServiceOption@@3KA    00066e68     loopbackdlg.obj
 0003:00002e70       ?g_hActiveWindow@@3PAUHWND__@@A 00066e70     mainfrm.obj
 0003:00002e88       ?g_bNidOK@@3HA             00066e88     msldlg.obj
 0003:00002e8c       ?g_bMCCOK@@3HA             00066e8c     msldlg.obj
 0003:00002e90       ?g_bMNCOK@@3HA             00066e90     msldlg.obj
 0003:00002e94       ?g_bSidOK@@3HA             00066e94     msldlg.obj
 0003:00002e98       ?g_bMsidOK@@3HA            00066e98     msldlg.obj
 0003:00002e9c       ?g_bMDNOK@@3HA             00066e9c     msldlg.obj
 0003:00002ea0       ?g_pMslInfo@@3UtagRILMSLINFO@@A 00066ea0     msldlg.obj
 0003:00002f1c       ?g_nPhoneNumLen@@3KA       00066f1c     msldlg.obj
 0003:00002f20       ?g_hMSLSaveMenu@@3PAUHWND__@@A 00066f20     msldlg.obj
 0003:00002f2c       ?g_hWndNetworkList@@3PAUHWND__@@A 00066f2c     network.obj
 0003:00002f38       ?g_bMsid@@3HA              00066f38     otksldlg.obj
 0003:00002f3c       ?g_bMDN@@3HA               00066f3c     otksldlg.obj
 0003:00002f40       ?g_pmslInfo@@3UtagRILMSLINFO@@A 00066f40     otksldlg.obj
 0003:00002fbc       ?g_nphoneNumLen@@3KA       00066fbc     otksldlg.obj
 0003:00002fc0       ?g_hOTKSLSaveMenu@@3PAUHWND__@@A 00066fc0     otksldlg.obj
 0003:00002fd0       ?g_stRilTechHdrInfo@@3USW_RILTECHHDRINFO@@A 00066fd0     PhoneUtility.obj
 0003:00003068       ?g_stRilDbgInfo@@3UtagRILMODEMDEBUGINFO@@A 00067068     PhoneUtility.obj
 0003:00003144       ?g_NoAAMResponseId@@3IA    00067144     PhoneUtility.obj
 0003:00003148       ?g_Err@@3UtagErrorInfo@@A  00067148     PhoneUtility.obj
 0003:00003350       ?g_bGrp@@3HA               00067350     PhoneUtility.obj
 0003:00003354       ?g_bSPCValidated@@3HA      00067354     PhoneUtility.obj
 0003:00003358       ?g_dwSPC@@3KA              00067358     PhoneUtility.obj
 0003:0000335c       ?g_dwActiveTab@@3KA        0006735c     PhoneUtility.obj
 0003:00003360       ?g_stRilStatus@@3USW_RILStatus@@A 00067360     PhoneUtility.obj
 0003:000033a0       ?g_strMSL@@3PAGA           000673a0     PhoneUtility.obj
 0003:00003850       ?g_szCmdLine@@3PAGA        00067850     PhoneUtility.obj
 0003:00003d00       ?g_szMessage@@3PAGA        00067d00     PhoneUtility.obj
 0003:000041b0       ?g_pszTitle@@3PAGA         000681b0     PhoneUtility.obj
 0003:00004660       ?g_pszAppName@@3PAGA       00068660     PhoneUtility.obj
 0003:00004b10       ?g_hWndMain@@3PAUHWND__@@A 00068b10     PhoneUtility.obj
 0003:00004b14       ?g_dwSpMode@@3KA           00068b14     PhoneUtility.obj
 0003:00004b18       ?g_nCarrier@@3KA           00068b18     PhoneUtility.obj
 0003:00004b1c       ?g_hResInst@@3PAUHINSTANCE__@@A 00068b1c     PhoneUtility.obj
 0003:00004b20       ?g_hInst@@3PAUHINSTANCE__@@A 00068b20     PhoneUtility.obj
 0003:00004b24       ?g_hWndListView@@3PAUHWND__@@A 00068b24     PhoneUtility.obj
 0003:00004b28       ?g_bDbgMode@@3HA           00068b28     PhoneUtility.obj
 0003:00004b2c       ?g_dwRtnOrClear@@3KA       00068b2c     PhoneUtility.obj
 0003:00004b38       ?g_szPass@@3PAGA           00068b38     simpleipdlg.obj
 0003:00004fe8       ?g_szUname@@3PAGA          00068fe8     simpleipdlg.obj
 0003:000054a0       ?g_hSpcMenu@@3PAUHWND__@@A 000694a0     spcvalidation.obj
 0003:0000559c       ?g_dwCAIRev@@3KA           0006959c     systemdlg.obj
 0003:000055a0       ?g_dwRoamMode@@3KA         000695a0     systemdlg.obj
 0003:000055a8       ?g_szHdrPass@@3PAGA        000695a8     usernamedlg.obj
 0003:00005a58       ?g_szHdrUname@@3PAGA       00069a58     usernamedlg.obj
 0003:00005f08       ?g_stPDPList@@3UtagRILPDPLIST@@A 00069f08     usernamedlg.obj
 0003:00005f28       ?g_stPDPPayload@@3UtagRILPDPPAYLOAD@@A 00069f28     usernamedlg.obj
 0003:00006028       ?g_stcurrentPDP@@3UtagRILGETORSETPDP@@A 0006a028     usernamedlg.obj
 0003:00006128       ?g_nNumOfProfiles@@3HA     0006a128     usernamedlg.obj
 0003:0000612c       ?g_bChk@@3HA               0006a12c     usernamedlg.obj
 0003:00006130       ?g_hWndSPIMNAA@@3PAUHWND__@@A 0006a130     usernamedlg.obj
 0003:00006134       ?g_hWndSPIMNHA@@3PAUHWND__@@A 0006a134     usernamedlg.obj
 0003:00006138       ?g_hWndMNASSecret@@3PAUHWND__@@A 0006a138     usernamedlg.obj
 0003:0000613c       ?g_hWndMNHASSecret@@3PAUHWND__@@A 0006a13c     usernamedlg.obj
 0003:00006140       ?g_hWndUNai@@3PAUHWND__@@A 0006a140     usernamedlg.obj
 0003:00006144       ?g_hWndRTunnel@@3PAUHWND__@@A 0006a144     usernamedlg.obj
 0003:00006148       ?g_hWndSHomeAgent@@3PAUHWND__@@A 0006a148     usernamedlg.obj
 0003:0000614c       ?g_hWndPHomeAgent@@3PAUHWND__@@A 0006a14c     usernamedlg.obj
 0003:00006150       ?g_hWndHomeAgent@@3PAUHWND__@@A 0006a150     usernamedlg.obj
 0003:00006154       ?g_hWndChkHex@@3PAUHWND__@@A 0006a154     usernamedlg.obj
 0003:00006158       ?g_hWndPDPList@@3PAUHWND__@@A 0006a158     usernamedlg.obj
 0003:0000615c       ?g_hWndActivePDP@@3PAUHWND__@@A 0006a15c     usernamedlg.obj
 0003:00006160       ?g_hWndHdrAAASSecret@@3PAUHWND__@@A 0006a160     usernamedlg.obj
 0003:00006164       ?g_hWndHdrNai@@3PAUHWND__@@A 0006a164     usernamedlg.obj
 0003:00006170       ?g_VersionInfo@@3UtagRILVERNOINFO@@A 0006a170     versioninfo.obj
 0003:00006e70       ?m_hMenuVocoder@@3PAUHWND__@@A 0006ae70     vocoderdlg.obj
 0003:00006e74       ?g_namID@@3EA              0006ae74     vocoderdlg.obj
 0003:00006e78       ?g_bEvrcEnabled@@3HA       0006ae78     vocoderdlg.obj
 0003:00006f40       __lc_handle                0006af40     LIBCMTD:nlsdata2.obj
 0003:00006f58       __lc_codepage              0006af58     LIBCMTD:nlsdata2.obj
 0003:00006f5c       __lc_collate_cp            0006af5c     LIBCMTD:nlsdata2.obj
 0003:000070a4       __lconv_static_null        0006b0a4     LIBCMTD:lconv.obj
 0003:000070ac       __onexitend                0006b0ac     <common>
 0003:000070b0       __onexitbegin              0006b0b0     <common>
 0003:000070b4       _exitflag                  0006b0b4     <common>
 0003:000070b8       _pfnReportHook             0006b0b8     <common>
 0003:000070bc       _pReportHookListW          0006b0bc     <common>
 0003:000070c0       _pReportHookList           0006b0c0     <common>

 entry point at        0001:00024164

 Static symbols

 0001:00024238       _initterm                  00035238 f   corelibc:crt0dat.obj
 0001:000242d8       doexit                     000352d8 f   corelibc:crt0dat.obj
 0001:00024588       _wcsftime_l_stat           00035588 f   LIBCMTD:wcsftime.obj
 0001:00026918       _expandtime                00037918 f   LIBCMTD:strftime.obj
 0001:00028190       _store_str                 00039190 f   LIBCMTD:strftime.obj
 0001:00028210       _store_num                 00039210 f   LIBCMTD:strftime.obj
 0001:00028344       _store_number              00039344 f   LIBCMTD:strftime.obj
 0001:00028478       _store_winword             00039478 f   LIBCMTD:strftime.obj
 0001:0002a614       _tzset_nolock              0003b614 f   LIBCMTD:tzset.obj
 0001:0002ab44       _isindst_nolock            0003bb44 f   LIBCMTD:tzset.obj
 0001:0002b0e0       cvtdate                    0003c0e0 f   LIBCMTD:tzset.obj
 0001:0002e984       __crtInitCritSecNoSpinCount 0003f984 f   LIBCMTD:initcrit.obj
 0001:0002f0c8       xtow_s                     000400c8 f   LIBCMTD:xtows.obj
 0001:0002f970       ??__ERIL_STATUS_CHANGED@@YAXXZ 00040970 f   advanceddlg.obj
 0001:0002f9a0       ??__EPHONEUTILS_END_MESSAGE@@YAXXZ 000409a0 f   authkey.obj
 0001:0002f9d0       ??__ERIL_STATUS_CHANGED@@YAXXZ 000409d0 f   authkey.obj
 0001:0002fa00       ??__ERIL_STATUS_CHANGED@@YAXXZ 00040a00 f   browserdlg.obj
 0001:0002fa30       ??__ERIL_STATUS_CHANGED@@YAXXZ 00040a30 f   bwmeterdlg.obj
 0001:0002fa60       ??__EPOWER_ON@@YAXXZ       00040a60 f   configdlg.obj
 0001:0002fa90       ??__EPOWER_OFF@@YAXXZ      00040a90 f   configdlg.obj
 0001:0002fac0       ??__EIOTA_BEGIN_MESSAGE@@YAXXZ 00040ac0 f   configdlg.obj
 0001:0002faf0       ??__EIOTA_END_MESSAGE@@YAXXZ 00040af0 f   configdlg.obj
 0001:0002fb20       ??__EIOTA_BEGIN_ACK@@YAXXZ 00040b20 f   configdlg.obj
 0001:0002fb50       ??__EIOTA_BEGIN_NACK@@YAXXZ 00040b50 f   configdlg.obj
 0001:0002fb80       ??__EIOTA_END_ACK@@YAXXZ   00040b80 f   configdlg.obj
 0001:0002fbb0       ??__EIOTA_EXIT_MESSAGE@@YAXXZ 00040bb0 f   configdlg.obj
 0001:0002fbe0       ??__EIOTA_ALIVE_MESSAGE@@YAXXZ 00040be0 f   configdlg.obj
 0001:0002fc10       ??__EIOTA_PING_MESSAGE@@YAXXZ 00040c10 f   configdlg.obj
 0001:0002fc40       ??__EIOTA_PING_ACK@@YAXXZ  00040c40 f   configdlg.obj
 0001:0002fc70       ??__EIOTA_CRITICAL_ERROR@@YAXXZ 00040c70 f   configdlg.obj
 0001:0002fca0       ??__EIOTA_NON_CRITICAL_ERROR@@YAXXZ 00040ca0 f   configdlg.obj
 0001:0002fcd0       ??__EIOTA_KILL_ME@@YAXXZ   00040cd0 f   configdlg.obj
 0001:0002fd00       ??__EIOTA_UPDATE_STATUS@@YAXXZ 00040d00 f   configdlg.obj
 0001:0002fd30       ??__EIOTA_DATAPORT_INUSE@@YAXXZ 00040d30 f   configdlg.obj
 0001:0002fd60       ??__EIOTA_DONE@@YAXXZ      00040d60 f   configdlg.obj
 0001:0002fd90       ??__EIOTA_DIAL@@YAXXZ      00040d90 f   configdlg.obj
 0001:0002fdc0       ??__EIOTA_1012_MIP_ERR@@YAXXZ 00040dc0 f   configdlg.obj
 0001:0002fdf0       ??__EPHONEUTILS_BEGIN_MESSAGE@@YAXXZ 00040df0 f   configdlg.obj
 0001:0002fe20       ??__EPHONEUTILS_END_MESSAGE@@YAXXZ 00040e20 f   configdlg.obj
 0001:0002fe50       ??__EPHONEUTILS_BEGIN_ACK@@YAXXZ 00040e50 f   configdlg.obj
 0001:0002fe80       ??__EPHONEUTILS_BEGIN_NACK@@YAXXZ 00040e80 f   configdlg.obj
 0001:0002feb0       ??__EPHONEUTILS_END_ACK@@YAXXZ 00040eb0 f   configdlg.obj
 0001:0002fee0       ??__EPHONEUTILS_EXIT_MESSAGE@@YAXXZ 00040ee0 f   configdlg.obj
 0001:0002ff10       ??__EPHONEUTILS_ALIVE_MESSAGE@@YAXXZ 00040f10 f   configdlg.obj
 0001:0002ff40       ??__EPHONEUTILS_PING_MESSAGE@@YAXXZ 00040f40 f   configdlg.obj
 0001:0002ff70       ??__EPHONEUTILS_PING_ACK@@YAXXZ 00040f70 f   configdlg.obj
 0001:0002ffa0       ??__EAW_BEGIN_MESSAGE@@YAXXZ 00040fa0 f   configdlg.obj
 0001:0002ffd0       ??__EAW_END_MESSAGE@@YAXXZ 00040fd0 f   configdlg.obj
 0001:00030000       ??__EAW_BEGIN_ACK@@YAXXZ   00041000 f   configdlg.obj
 0001:00030030       ??__EAW_BEGIN_NACK@@YAXXZ  00041030 f   configdlg.obj
 0001:00030060       ??__EAW_END_ACK@@YAXXZ     00041060 f   configdlg.obj
 0001:00030090       ??__EAW_EXIT_MESSAGE@@YAXXZ 00041090 f   configdlg.obj
 0001:000300c0       ??__EAW_ALIVE_MESSAGE@@YAXXZ 000410c0 f   configdlg.obj
 0001:000300f0       ??__EAW_PING_MESSAGE@@YAXXZ 000410f0 f   configdlg.obj
 0001:00030120       ??__EAW_PING_ACK@@YAXXZ    00041120 f   configdlg.obj
 0001:00030150       ??__EUPDATER_BEGIN@@YAXXZ  00041150 f   configdlg.obj
 0001:00030180       ??__EUPDATER_END@@YAXXZ    00041180 f   configdlg.obj
 0001:000301b0       ??__EUPDATER_BEGIN_ACK@@YAXXZ 000411b0 f   configdlg.obj
 0001:000301e0       ??__EUPDATER_BEGIN_NACK@@YAXXZ 000411e0 f   configdlg.obj
 0001:00030210       ??__EUPDATER_END_ACK@@YAXXZ 00041210 f   configdlg.obj
 0001:00030240       ??__EUPDATER_END_NACK@@YAXXZ 00041240 f   configdlg.obj
 0001:00030270       ??__ERIL_STATUS_CHANGED@@YAXXZ 00041270 f   configdlg.obj
 0001:000302a0       ??__ERIL_DBG_NOTIFY@@YAXXZ 000412a0 f   configdlg.obj
 0001:000302d0       ??__ERIL_TECHHDR_NOTIFY@@YAXXZ 000412d0 f   configdlg.obj
 0001:00030300       ??__ERIL_IOTA_STATUS_CHANGED@@YAXXZ 00041300 f   configdlg.obj
 0001:00030330       ??__ERIL_IOTA_WAP_URI@@YAXXZ 00041330 f   configdlg.obj
 0001:00030360       ??__ERIL_PDSM_PD_DATA@@YAXXZ 00041360 f   configdlg.obj
 0001:00030390       ??__ERIL_PDSM_PD_DONE@@YAXXZ 00041390 f   configdlg.obj
 0001:000303c0       ??__ERIL_PDSM_PD_END@@YAXXZ 000413c0 f   configdlg.obj
 0001:000303f0       ??__ERIL_PDSM_PD_BEGIN@@YAXXZ 000413f0 f   configdlg.obj
 0001:00030420       ??__ERIL_PDSM_PD_UPDATE_FAILURE@@YAXXZ 00041420 f   configdlg.obj
 0001:00030450       ??__ERIL_PDSM_PD_DLD_DATA@@YAXXZ 00041450 f   configdlg.obj
 0001:00030480       ??__ERIL_PDSM_PD_DLD_DONE@@YAXXZ 00041480 f   configdlg.obj
 0001:000304b0       ??__ERIL_PDSM_PD_DLD_END@@YAXXZ 000414b0 f   configdlg.obj
 0001:000304e0       ??__ERIL_PDSM_PD_DLD_BEGIN@@YAXXZ 000414e0 f   configdlg.obj
 0001:00030510       ??__ERIL_PDSM_PA_PARAM@@YAXXZ 00041510 f   configdlg.obj
 0001:00030540       ??__ERIL_CALL_BYTE_CTR@@YAXXZ 00041540 f   configdlg.obj
 0001:00030570       ??__ERIL_CREATE_MAIN_LIST@@YAXXZ 00041570 f   configdlg.obj
 0001:000305a0       ??__ERIL_STATUS_CHANGED@@YAXXZ 000415a0 f   evdo.obj
 0001:000305d0       ??__ERIL_STATUS_CHANGED@@YAXXZ 000415d0 f   finger.obj
 0001:00030600       ??__ERIL_DBG_NOTIFY@@YAXXZ 00041600 f   finger.obj
 0001:00030630       ??__ERIL_PDSM_PD_DATA@@YAXXZ 00041630 f   gpsdatadlg.obj
 0001:00030660       ??__ERIL_PDSM_PD_DONE@@YAXXZ 00041660 f   gpsdatadlg.obj
 0001:00030690       ??__ERIL_PDSM_PD_END@@YAXXZ 00041690 f   gpsdatadlg.obj
 0001:000306c0       ??__ERIL_PDSM_PD_BEGIN@@YAXXZ 000416c0 f   gpsdatadlg.obj
 0001:000306f0       ??__ERIL_PDSM_PD_UPDATE_FAILURE@@YAXXZ 000416f0 f   gpsdatadlg.obj
 0001:00030720       ??__EPOWER_ON@@YAXXZ       00041720 f   gsm2G.obj
 0001:00030750       ??__EPOWER_OFF@@YAXXZ      00041750 f   gsm2G.obj
 0001:00030780       ??__EIOTA_BEGIN_MESSAGE@@YAXXZ 00041780 f   gsm2G.obj
 0001:000307b0       ??__EIOTA_END_MESSAGE@@YAXXZ 000417b0 f   gsm2G.obj
 0001:000307e0       ??__EIOTA_BEGIN_ACK@@YAXXZ 000417e0 f   gsm2G.obj
 0001:00030810       ??__EIOTA_BEGIN_NACK@@YAXXZ 00041810 f   gsm2G.obj
 0001:00030840       ??__EIOTA_END_ACK@@YAXXZ   00041840 f   gsm2G.obj
 0001:00030870       ??__EIOTA_EXIT_MESSAGE@@YAXXZ 00041870 f   gsm2G.obj
 0001:000308a0       ??__EIOTA_ALIVE_MESSAGE@@YAXXZ 000418a0 f   gsm2G.obj
 0001:000308d0       ??__EIOTA_PING_MESSAGE@@YAXXZ 000418d0 f   gsm2G.obj
 0001:00030900       ??__EIOTA_PING_ACK@@YAXXZ  00041900 f   gsm2G.obj
 0001:00030930       ??__EIOTA_CRITICAL_ERROR@@YAXXZ 00041930 f   gsm2G.obj
 0001:00030960       ??__EIOTA_NON_CRITICAL_ERROR@@YAXXZ 00041960 f   gsm2G.obj
 0001:00030990       ??__EIOTA_KILL_ME@@YAXXZ   00041990 f   gsm2G.obj
 0001:000309c0       ??__EIOTA_UPDATE_STATUS@@YAXXZ 000419c0 f   gsm2G.obj
 0001:000309f0       ??__EIOTA_DATAPORT_INUSE@@YAXXZ 000419f0 f   gsm2G.obj
 0001:00030a20       ??__EIOTA_DONE@@YAXXZ      00041a20 f   gsm2G.obj
 0001:00030a50       ??__EIOTA_DIAL@@YAXXZ      00041a50 f   gsm2G.obj
 0001:00030a80       ??__EIOTA_1012_MIP_ERR@@YAXXZ 00041a80 f   gsm2G.obj
 0001:00030ab0       ??__EPHONEUTILS_BEGIN_MESSAGE@@YAXXZ 00041ab0 f   gsm2G.obj
 0001:00030ae0       ??__EPHONEUTILS_END_MESSAGE@@YAXXZ 00041ae0 f   gsm2G.obj
 0001:00030b10       ??__EPHONEUTILS_BEGIN_ACK@@YAXXZ 00041b10 f   gsm2G.obj
 0001:00030b40       ??__EPHONEUTILS_BEGIN_NACK@@YAXXZ 00041b40 f   gsm2G.obj
 0001:00030b70       ??__EPHONEUTILS_END_ACK@@YAXXZ 00041b70 f   gsm2G.obj
 0001:00030ba0       ??__EPHONEUTILS_EXIT_MESSAGE@@YAXXZ 00041ba0 f   gsm2G.obj
 0001:00030bd0       ??__EPHONEUTILS_ALIVE_MESSAGE@@YAXXZ 00041bd0 f   gsm2G.obj
 0001:00030c00       ??__EPHONEUTILS_PING_MESSAGE@@YAXXZ 00041c00 f   gsm2G.obj
 0001:00030c30       ??__EPHONEUTILS_PING_ACK@@YAXXZ 00041c30 f   gsm2G.obj
 0001:00030c60       ??__EAW_BEGIN_MESSAGE@@YAXXZ 00041c60 f   gsm2G.obj
 0001:00030c90       ??__EAW_END_MESSAGE@@YAXXZ 00041c90 f   gsm2G.obj
 0001:00030cc0       ??__EAW_BEGIN_ACK@@YAXXZ   00041cc0 f   gsm2G.obj
 0001:00030cf0       ??__EAW_BEGIN_NACK@@YAXXZ  00041cf0 f   gsm2G.obj
 0001:00030d20       ??__EAW_END_ACK@@YAXXZ     00041d20 f   gsm2G.obj
 0001:00030d50       ??__EAW_EXIT_MESSAGE@@YAXXZ 00041d50 f   gsm2G.obj
 0001:00030d80       ??__EAW_ALIVE_MESSAGE@@YAXXZ 00041d80 f   gsm2G.obj
 0001:00030db0       ??__EAW_PING_MESSAGE@@YAXXZ 00041db0 f   gsm2G.obj
 0001:00030de0       ??__EAW_PING_ACK@@YAXXZ    00041de0 f   gsm2G.obj
 0001:00030e10       ??__EUPDATER_BEGIN@@YAXXZ  00041e10 f   gsm2G.obj
 0001:00030e40       ??__EUPDATER_END@@YAXXZ    00041e40 f   gsm2G.obj
 0001:00030e70       ??__EUPDATER_BEGIN_ACK@@YAXXZ 00041e70 f   gsm2G.obj
 0001:00030ea0       ??__EUPDATER_BEGIN_NACK@@YAXXZ 00041ea0 f   gsm2G.obj
 0001:00030ed0       ??__EUPDATER_END_ACK@@YAXXZ 00041ed0 f   gsm2G.obj
 0001:00030f00       ??__EUPDATER_END_NACK@@YAXXZ 00041f00 f   gsm2G.obj
 0001:00030f30       ??__ERIL_STATUS_CHANGED@@YAXXZ 00041f30 f   gsm2G.obj
 0001:00030f60       ??__ERIL_DBG_NOTIFY@@YAXXZ 00041f60 f   gsm2G.obj
 0001:00030f90       ??__ERIL_TECHHDR_NOTIFY@@YAXXZ 00041f90 f   gsm2G.obj
 0001:00030fc0       ??__ERIL_IOTA_STATUS_CHANGED@@YAXXZ 00041fc0 f   gsm2G.obj
 0001:00030ff0       ??__ERIL_IOTA_WAP_URI@@YAXXZ 00041ff0 f   gsm2G.obj
 0001:00031020       ??__ERIL_PDSM_PD_DATA@@YAXXZ 00042020 f   gsm2G.obj
 0001:00031050       ??__ERIL_PDSM_PD_DONE@@YAXXZ 00042050 f   gsm2G.obj
 0001:00031080       ??__ERIL_PDSM_PD_END@@YAXXZ 00042080 f   gsm2G.obj
 0001:000310b0       ??__ERIL_PDSM_PD_BEGIN@@YAXXZ 000420b0 f   gsm2G.obj
 0001:000310e0       ??__ERIL_PDSM_PD_UPDATE_FAILURE@@YAXXZ 000420e0 f   gsm2G.obj
 0001:00031110       ??__ERIL_PDSM_PD_DLD_DATA@@YAXXZ 00042110 f   gsm2G.obj
 0001:00031140       ??__ERIL_PDSM_PD_DLD_DONE@@YAXXZ 00042140 f   gsm2G.obj
 0001:00031170       ??__ERIL_PDSM_PD_DLD_END@@YAXXZ 00042170 f   gsm2G.obj
 0001:000311a0       ??__ERIL_PDSM_PD_DLD_BEGIN@@YAXXZ 000421a0 f   gsm2G.obj
 0001:000311d0       ??__ERIL_PDSM_PA_PARAM@@YAXXZ 000421d0 f   gsm2G.obj
 0001:00031200       ??__ERIL_CALL_BYTE_CTR@@YAXXZ 00042200 f   gsm2G.obj
 0001:00031230       ??__ERIL_CREATE_MAIN_LIST@@YAXXZ 00042230 f   gsm2G.obj
 0001:00031260       ??__EPOWER_ON@@YAXXZ       00042260 f   gsm3G.obj
 0001:00031290       ??__EPOWER_OFF@@YAXXZ      00042290 f   gsm3G.obj
 0001:000312c0       ??__EIOTA_BEGIN_MESSAGE@@YAXXZ 000422c0 f   gsm3G.obj
 0001:000312f0       ??__EIOTA_END_MESSAGE@@YAXXZ 000422f0 f   gsm3G.obj
 0001:00031320       ??__EIOTA_BEGIN_ACK@@YAXXZ 00042320 f   gsm3G.obj
 0001:00031350       ??__EIOTA_BEGIN_NACK@@YAXXZ 00042350 f   gsm3G.obj
 0001:00031380       ??__EIOTA_END_ACK@@YAXXZ   00042380 f   gsm3G.obj
 0001:000313b0       ??__EIOTA_EXIT_MESSAGE@@YAXXZ 000423b0 f   gsm3G.obj
 0001:000313e0       ??__EIOTA_ALIVE_MESSAGE@@YAXXZ 000423e0 f   gsm3G.obj
 0001:00031410       ??__EIOTA_PING_MESSAGE@@YAXXZ 00042410 f   gsm3G.obj
 0001:00031440       ??__EIOTA_PING_ACK@@YAXXZ  00042440 f   gsm3G.obj
 0001:00031470       ??__EIOTA_CRITICAL_ERROR@@YAXXZ 00042470 f   gsm3G.obj
 0001:000314a0       ??__EIOTA_NON_CRITICAL_ERROR@@YAXXZ 000424a0 f   gsm3G.obj
 0001:000314d0       ??__EIOTA_KILL_ME@@YAXXZ   000424d0 f   gsm3G.obj
 0001:00031500       ??__EIOTA_UPDATE_STATUS@@YAXXZ 00042500 f   gsm3G.obj
 0001:00031530       ??__EIOTA_DATAPORT_INUSE@@YAXXZ 00042530 f   gsm3G.obj
 0001:00031560       ??__EIOTA_DONE@@YAXXZ      00042560 f   gsm3G.obj
 0001:00031590       ??__EIOTA_DIAL@@YAXXZ      00042590 f   gsm3G.obj
 0001:000315c0       ??__EIOTA_1012_MIP_ERR@@YAXXZ 000425c0 f   gsm3G.obj
 0001:000315f0       ??__EPHONEUTILS_BEGIN_MESSAGE@@YAXXZ 000425f0 f   gsm3G.obj
 0001:00031620       ??__EPHONEUTILS_END_MESSAGE@@YAXXZ 00042620 f   gsm3G.obj
 0001:00031650       ??__EPHONEUTILS_BEGIN_ACK@@YAXXZ 00042650 f   gsm3G.obj
 0001:00031680       ??__EPHONEUTILS_BEGIN_NACK@@YAXXZ 00042680 f   gsm3G.obj
 0001:000316b0       ??__EPHONEUTILS_END_ACK@@YAXXZ 000426b0 f   gsm3G.obj
 0001:000316e0       ??__EPHONEUTILS_EXIT_MESSAGE@@YAXXZ 000426e0 f   gsm3G.obj
 0001:00031710       ??__EPHONEUTILS_ALIVE_MESSAGE@@YAXXZ 00042710 f   gsm3G.obj
 0001:00031740       ??__EPHONEUTILS_PING_MESSAGE@@YAXXZ 00042740 f   gsm3G.obj
 0001:00031770       ??__EPHONEUTILS_PING_ACK@@YAXXZ 00042770 f   gsm3G.obj
 0001:000317a0       ??__EAW_BEGIN_MESSAGE@@YAXXZ 000427a0 f   gsm3G.obj
 0001:000317d0       ??__EAW_END_MESSAGE@@YAXXZ 000427d0 f   gsm3G.obj
 0001:00031800       ??__EAW_BEGIN_ACK@@YAXXZ   00042800 f   gsm3G.obj
 0001:00031830       ??__EAW_BEGIN_NACK@@YAXXZ  00042830 f   gsm3G.obj
 0001:00031860       ??__EAW_END_ACK@@YAXXZ     00042860 f   gsm3G.obj
 0001:00031890       ??__EAW_EXIT_MESSAGE@@YAXXZ 00042890 f   gsm3G.obj
 0001:000318c0       ??__EAW_ALIVE_MESSAGE@@YAXXZ 000428c0 f   gsm3G.obj
 0001:000318f0       ??__EAW_PING_MESSAGE@@YAXXZ 000428f0 f   gsm3G.obj
 0001:00031920       ??__EAW_PING_ACK@@YAXXZ    00042920 f   gsm3G.obj
 0001:00031950       ??__EUPDATER_BEGIN@@YAXXZ  00042950 f   gsm3G.obj
 0001:00031980       ??__EUPDATER_END@@YAXXZ    00042980 f   gsm3G.obj
 0001:000319b0       ??__EUPDATER_BEGIN_ACK@@YAXXZ 000429b0 f   gsm3G.obj
 0001:000319e0       ??__EUPDATER_BEGIN_NACK@@YAXXZ 000429e0 f   gsm3G.obj
 0001:00031a10       ??__EUPDATER_END_ACK@@YAXXZ 00042a10 f   gsm3G.obj
 0001:00031a40       ??__EUPDATER_END_NACK@@YAXXZ 00042a40 f   gsm3G.obj
 0001:00031a70       ??__ERIL_STATUS_CHANGED@@YAXXZ 00042a70 f   gsm3G.obj
 0001:00031aa0       ??__ERIL_DBG_NOTIFY@@YAXXZ 00042aa0 f   gsm3G.obj
 0001:00031ad0       ??__ERIL_TECHHDR_NOTIFY@@YAXXZ 00042ad0 f   gsm3G.obj
 0001:00031b00       ??__ERIL_IOTA_STATUS_CHANGED@@YAXXZ 00042b00 f   gsm3G.obj
 0001:00031b30       ??__ERIL_IOTA_WAP_URI@@YAXXZ 00042b30 f   gsm3G.obj
 0001:00031b60       ??__ERIL_PDSM_PD_DATA@@YAXXZ 00042b60 f   gsm3G.obj
 0001:00031b90       ??__ERIL_PDSM_PD_DONE@@YAXXZ 00042b90 f   gsm3G.obj
 0001:00031bc0       ??__ERIL_PDSM_PD_END@@YAXXZ 00042bc0 f   gsm3G.obj
 0001:00031bf0       ??__ERIL_PDSM_PD_BEGIN@@YAXXZ 00042bf0 f   gsm3G.obj
 0001:00031c20       ??__ERIL_PDSM_PD_UPDATE_FAILURE@@YAXXZ 00042c20 f   gsm3G.obj
 0001:00031c50       ??__ERIL_PDSM_PD_DLD_DATA@@YAXXZ 00042c50 f   gsm3G.obj
 0001:00031c80       ??__ERIL_PDSM_PD_DLD_DONE@@YAXXZ 00042c80 f   gsm3G.obj
 0001:00031cb0       ??__ERIL_PDSM_PD_DLD_END@@YAXXZ 00042cb0 f   gsm3G.obj
 0001:00031ce0       ??__ERIL_PDSM_PD_DLD_BEGIN@@YAXXZ 00042ce0 f   gsm3G.obj
 0001:00031d10       ??__ERIL_PDSM_PA_PARAM@@YAXXZ 00042d10 f   gsm3G.obj
 0001:00031d40       ??__ERIL_CALL_BYTE_CTR@@YAXXZ 00042d40 f   gsm3G.obj
 0001:00031d70       ??__ERIL_CREATE_MAIN_LIST@@YAXXZ 00042d70 f   gsm3G.obj
 0001:00031da0       ??__EPOWER_ON@@YAXXZ       00042da0 f   gsmband.obj
 0001:00031dd0       ??__EPOWER_OFF@@YAXXZ      00042dd0 f   gsmband.obj
 0001:00031e00       ??__EIOTA_BEGIN_MESSAGE@@YAXXZ 00042e00 f   gsmband.obj
 0001:00031e30       ??__EIOTA_END_MESSAGE@@YAXXZ 00042e30 f   gsmband.obj
 0001:00031e60       ??__EIOTA_BEGIN_ACK@@YAXXZ 00042e60 f   gsmband.obj
 0001:00031e90       ??__EIOTA_BEGIN_NACK@@YAXXZ 00042e90 f   gsmband.obj
 0001:00031ec0       ??__EIOTA_END_ACK@@YAXXZ   00042ec0 f   gsmband.obj
 0001:00031ef0       ??__EIOTA_EXIT_MESSAGE@@YAXXZ 00042ef0 f   gsmband.obj
 0001:00031f20       ??__EIOTA_ALIVE_MESSAGE@@YAXXZ 00042f20 f   gsmband.obj
 0001:00031f50       ??__EIOTA_PING_MESSAGE@@YAXXZ 00042f50 f   gsmband.obj
 0001:00031f80       ??__EIOTA_PING_ACK@@YAXXZ  00042f80 f   gsmband.obj
 0001:00031fb0       ??__EIOTA_CRITICAL_ERROR@@YAXXZ 00042fb0 f   gsmband.obj
 0001:00031fe0       ??__EIOTA_NON_CRITICAL_ERROR@@YAXXZ 00042fe0 f   gsmband.obj
 0001:00032010       ??__EIOTA_KILL_ME@@YAXXZ   00043010 f   gsmband.obj
 0001:00032040       ??__EIOTA_UPDATE_STATUS@@YAXXZ 00043040 f   gsmband.obj
 0001:00032070       ??__EIOTA_DATAPORT_INUSE@@YAXXZ 00043070 f   gsmband.obj
 0001:000320a0       ??__EIOTA_DONE@@YAXXZ      000430a0 f   gsmband.obj
 0001:000320d0       ??__EIOTA_DIAL@@YAXXZ      000430d0 f   gsmband.obj
 0001:00032100       ??__EIOTA_1012_MIP_ERR@@YAXXZ 00043100 f   gsmband.obj
 0001:00032130       ??__EPHONEUTILS_BEGIN_MESSAGE@@YAXXZ 00043130 f   gsmband.obj
 0001:00032160       ??__EPHONEUTILS_END_MESSAGE@@YAXXZ 00043160 f   gsmband.obj
 0001:00032190       ??__EPHONEUTILS_BEGIN_ACK@@YAXXZ 00043190 f   gsmband.obj
 0001:000321c0       ??__EPHONEUTILS_BEGIN_NACK@@YAXXZ 000431c0 f   gsmband.obj
 0001:000321f0       ??__EPHONEUTILS_END_ACK@@YAXXZ 000431f0 f   gsmband.obj
 0001:00032220       ??__EPHONEUTILS_EXIT_MESSAGE@@YAXXZ 00043220 f   gsmband.obj
 0001:00032250       ??__EPHONEUTILS_ALIVE_MESSAGE@@YAXXZ 00043250 f   gsmband.obj
 0001:00032280       ??__EPHONEUTILS_PING_MESSAGE@@YAXXZ 00043280 f   gsmband.obj
 0001:000322b0       ??__EPHONEUTILS_PING_ACK@@YAXXZ 000432b0 f   gsmband.obj
 0001:000322e0       ??__EAW_BEGIN_MESSAGE@@YAXXZ 000432e0 f   gsmband.obj
 0001:00032310       ??__EAW_END_MESSAGE@@YAXXZ 00043310 f   gsmband.obj
 0001:00032340       ??__EAW_BEGIN_ACK@@YAXXZ   00043340 f   gsmband.obj
 0001:00032370       ??__EAW_BEGIN_NACK@@YAXXZ  00043370 f   gsmband.obj
 0001:000323a0       ??__EAW_END_ACK@@YAXXZ     000433a0 f   gsmband.obj
 0001:000323d0       ??__EAW_EXIT_MESSAGE@@YAXXZ 000433d0 f   gsmband.obj
 0001:00032400       ??__EAW_ALIVE_MESSAGE@@YAXXZ 00043400 f   gsmband.obj
 0001:00032430       ??__EAW_PING_MESSAGE@@YAXXZ 00043430 f   gsmband.obj
 0001:00032460       ??__EAW_PING_ACK@@YAXXZ    00043460 f   gsmband.obj
 0001:00032490       ??__EUPDATER_BEGIN@@YAXXZ  00043490 f   gsmband.obj
 0001:000324c0       ??__EUPDATER_END@@YAXXZ    000434c0 f   gsmband.obj
 0001:000324f0       ??__EUPDATER_BEGIN_ACK@@YAXXZ 000434f0 f   gsmband.obj
 0001:00032520       ??__EUPDATER_BEGIN_NACK@@YAXXZ 00043520 f   gsmband.obj
 0001:00032550       ??__EUPDATER_END_ACK@@YAXXZ 00043550 f   gsmband.obj
 0001:00032580       ??__EUPDATER_END_NACK@@YAXXZ 00043580 f   gsmband.obj
 0001:000325b0       ??__ERIL_STATUS_CHANGED@@YAXXZ 000435b0 f   gsmband.obj
 0001:000325e0       ??__ERIL_DBG_NOTIFY@@YAXXZ 000435e0 f   gsmband.obj
 0001:00032610       ??__ERIL_TECHHDR_NOTIFY@@YAXXZ 00043610 f   gsmband.obj
 0001:00032640       ??__ERIL_IOTA_STATUS_CHANGED@@YAXXZ 00043640 f   gsmband.obj
 0001:00032670       ??__ERIL_IOTA_WAP_URI@@YAXXZ 00043670 f   gsmband.obj
 0001:000326a0       ??__ERIL_PDSM_PD_DATA@@YAXXZ 000436a0 f   gsmband.obj
 0001:000326d0       ??__ERIL_PDSM_PD_DONE@@YAXXZ 000436d0 f   gsmband.obj
 0001:00032700       ??__ERIL_PDSM_PD_END@@YAXXZ 00043700 f   gsmband.obj
 0001:00032730       ??__ERIL_PDSM_PD_BEGIN@@YAXXZ 00043730 f   gsmband.obj
 0001:00032760       ??__ERIL_PDSM_PD_UPDATE_FAILURE@@YAXXZ 00043760 f   gsmband.obj
 0001:00032790       ??__ERIL_PDSM_PD_DLD_DATA@@YAXXZ 00043790 f   gsmband.obj
 0001:000327c0       ??__ERIL_PDSM_PD_DLD_DONE@@YAXXZ 000437c0 f   gsmband.obj
 0001:000327f0       ??__ERIL_PDSM_PD_DLD_END@@YAXXZ 000437f0 f   gsmband.obj
 0001:00032820       ??__ERIL_PDSM_PD_DLD_BEGIN@@YAXXZ 00043820 f   gsmband.obj
 0001:00032850       ??__ERIL_PDSM_PA_PARAM@@YAXXZ 00043850 f   gsmband.obj
 0001:00032880       ??__ERIL_CALL_BYTE_CTR@@YAXXZ 00043880 f   gsmband.obj
 0001:000328b0       ??__ERIL_CREATE_MAIN_LIST@@YAXXZ 000438b0 f   gsmband.obj
 0001:000328e0       ??__ERIL_STATUS_CHANGED@@YAXXZ 000438e0 f   iota.obj
 0001:00032910       ??__ERIL_STATUS_CHANGED@@YAXXZ 00043910 f   loopbackdlg.obj
 0001:00032940       ??__EPHONEUTILS_BEGIN_MESSAGE@@YAXXZ 00043940 f   mainfrm.obj
 0001:00032970       ??__EPHONEUTILS_END_MESSAGE@@YAXXZ 00043970 f   mainfrm.obj
 0001:000329a0       ??__EPHONEUTILS_BEGIN_ACK@@YAXXZ 000439a0 f   mainfrm.obj
 0001:000329d0       ??__EPHONEUTILS_BEGIN_NACK@@YAXXZ 000439d0 f   mainfrm.obj
 0001:00032a00       ??__EPHONEUTILS_EXIT_MESSAGE@@YAXXZ 00043a00 f   mainfrm.obj
 0001:00032a30       ??__EPHONEUTILS_END_MESSAGE@@YAXXZ 00043a30 f   msldlg.obj
 0001:00032a60       ??__ERIL_STATUS_CHANGED@@YAXXZ 00043a60 f   msldlg.obj
 0001:00032a90       ??__ERIL_STATUS_CHANGED@@YAXXZ 00043a90 f   network.obj
 0001:00032ac0       ??__EPHONEUTILS_END_MESSAGE@@YAXXZ 00043ac0 f   otksldlg.obj
 0001:00032af0       ??__ERIL_STATUS_CHANGED@@YAXXZ 00043af0 f   otksldlg.obj
 0001:00032b20       ??__EPHONEUTILS_END_MESSAGE@@YAXXZ 00043b20 f   passthrudlg.obj
 0001:00032b50       ??__EPHONEUTILS_END_MESSAGE@@YAXXZ 00043b50 f   rtndlg.obj
 0001:00032b80       ??__ERIL_STATUS_CHANGED@@YAXXZ 00043b80 f   rtndlg.obj
 0001:00032bb0       ??__ERIL_STATUS_CHANGED@@YAXXZ 00043bb0 f   simpleipdlg.obj
 0001:00032be0       ??__ERIL_STATUS_CHANGED@@YAXXZ 00043be0 f   sipdlg.obj
 0001:00032c10       ??__EPHONEUTILS_END_MESSAGE@@YAXXZ 00043c10 f   spcvalidation.obj
 0001:00032c40       ??__ERIL_STATUS_CHANGED@@YAXXZ 00043c40 f   spcvalidation.obj
 0001:00032c70       ??__EPOWER_ON@@YAXXZ       00043c70 f   stdafx.obj
 0001:00032ca0       ??__EPOWER_OFF@@YAXXZ      00043ca0 f   stdafx.obj
 0001:00032cd0       ??__EIOTA_BEGIN_MESSAGE@@YAXXZ 00043cd0 f   stdafx.obj
 0001:00032d00       ??__EIOTA_END_MESSAGE@@YAXXZ 00043d00 f   stdafx.obj
 0001:00032d30       ??__EIOTA_BEGIN_ACK@@YAXXZ 00043d30 f   stdafx.obj
 0001:00032d60       ??__EIOTA_BEGIN_NACK@@YAXXZ 00043d60 f   stdafx.obj
 0001:00032d90       ??__EIOTA_END_ACK@@YAXXZ   00043d90 f   stdafx.obj
 0001:00032dc0       ??__EIOTA_EXIT_MESSAGE@@YAXXZ 00043dc0 f   stdafx.obj
 0001:00032df0       ??__EIOTA_ALIVE_MESSAGE@@YAXXZ 00043df0 f   stdafx.obj
 0001:00032e20       ??__EIOTA_PING_MESSAGE@@YAXXZ 00043e20 f   stdafx.obj
 0001:00032e50       ??__EIOTA_PING_ACK@@YAXXZ  00043e50 f   stdafx.obj
 0001:00032e80       ??__EIOTA_CRITICAL_ERROR@@YAXXZ 00043e80 f   stdafx.obj
 0001:00032eb0       ??__EIOTA_NON_CRITICAL_ERROR@@YAXXZ 00043eb0 f   stdafx.obj
 0001:00032ee0       ??__EIOTA_KILL_ME@@YAXXZ   00043ee0 f   stdafx.obj
 0001:00032f10       ??__EIOTA_UPDATE_STATUS@@YAXXZ 00043f10 f   stdafx.obj
 0001:00032f40       ??__EIOTA_DATAPORT_INUSE@@YAXXZ 00043f40 f   stdafx.obj
 0001:00032f70       ??__EIOTA_DONE@@YAXXZ      00043f70 f   stdafx.obj
 0001:00032fa0       ??__EIOTA_DIAL@@YAXXZ      00043fa0 f   stdafx.obj
 0001:00032fd0       ??__EIOTA_1012_MIP_ERR@@YAXXZ 00043fd0 f   stdafx.obj
 0001:00033000       ??__EPHONEUTILS_BEGIN_MESSAGE@@YAXXZ 00044000 f   stdafx.obj
 0001:00033030       ??__EPHONEUTILS_END_MESSAGE@@YAXXZ 00044030 f   stdafx.obj
 0001:00033060       ??__EPHONEUTILS_BEGIN_ACK@@YAXXZ 00044060 f   stdafx.obj
 0001:00033090       ??__EPHONEUTILS_BEGIN_NACK@@YAXXZ 00044090 f   stdafx.obj
 0001:000330c0       ??__EPHONEUTILS_END_ACK@@YAXXZ 000440c0 f   stdafx.obj
 0001:000330f0       ??__EPHONEUTILS_EXIT_MESSAGE@@YAXXZ 000440f0 f   stdafx.obj
 0001:00033120       ??__EPHONEUTILS_ALIVE_MESSAGE@@YAXXZ 00044120 f   stdafx.obj
 0001:00033150       ??__EPHONEUTILS_PING_MESSAGE@@YAXXZ 00044150 f   stdafx.obj
 0001:00033180       ??__EPHONEUTILS_PING_ACK@@YAXXZ 00044180 f   stdafx.obj
 0001:000331b0       ??__EAW_BEGIN_MESSAGE@@YAXXZ 000441b0 f   stdafx.obj
 0001:000331e0       ??__EAW_END_MESSAGE@@YAXXZ 000441e0 f   stdafx.obj
 0001:00033210       ??__EAW_BEGIN_ACK@@YAXXZ   00044210 f   stdafx.obj
 0001:00033240       ??__EAW_BEGIN_NACK@@YAXXZ  00044240 f   stdafx.obj
 0001:00033270       ??__EAW_END_ACK@@YAXXZ     00044270 f   stdafx.obj
 0001:000332a0       ??__EAW_EXIT_MESSAGE@@YAXXZ 000442a0 f   stdafx.obj
 0001:000332d0       ??__EAW_ALIVE_MESSAGE@@YAXXZ 000442d0 f   stdafx.obj
 0001:00033300       ??__EAW_PING_MESSAGE@@YAXXZ 00044300 f   stdafx.obj
 0001:00033330       ??__EAW_PING_ACK@@YAXXZ    00044330 f   stdafx.obj
 0001:00033360       ??__EUPDATER_BEGIN@@YAXXZ  00044360 f   stdafx.obj
 0001:00033390       ??__EUPDATER_END@@YAXXZ    00044390 f   stdafx.obj
 0001:000333c0       ??__EUPDATER_BEGIN_ACK@@YAXXZ 000443c0 f   stdafx.obj
 0001:000333f0       ??__EUPDATER_BEGIN_NACK@@YAXXZ 000443f0 f   stdafx.obj
 0001:00033420       ??__EUPDATER_END_ACK@@YAXXZ 00044420 f   stdafx.obj
 0001:00033450       ??__EUPDATER_END_NACK@@YAXXZ 00044450 f   stdafx.obj
 0001:00033480       ??__ERIL_STATUS_CHANGED@@YAXXZ 00044480 f   stdafx.obj
 0001:000334b0       ??__ERIL_DBG_NOTIFY@@YAXXZ 000444b0 f   stdafx.obj
 0001:000334e0       ??__ERIL_TECHHDR_NOTIFY@@YAXXZ 000444e0 f   stdafx.obj
 0001:00033510       ??__ERIL_IOTA_STATUS_CHANGED@@YAXXZ 00044510 f   stdafx.obj
 0001:00033540       ??__ERIL_IOTA_WAP_URI@@YAXXZ 00044540 f   stdafx.obj
 0001:00033570       ??__ERIL_PDSM_PD_DATA@@YAXXZ 00044570 f   stdafx.obj
 0001:000335a0       ??__ERIL_PDSM_PD_DONE@@YAXXZ 000445a0 f   stdafx.obj
 0001:000335d0       ??__ERIL_PDSM_PD_END@@YAXXZ 000445d0 f   stdafx.obj
 0001:00033600       ??__ERIL_PDSM_PD_BEGIN@@YAXXZ 00044600 f   stdafx.obj
 0001:00033630       ??__ERIL_PDSM_PD_UPDATE_FAILURE@@YAXXZ 00044630 f   stdafx.obj
 0001:00033660       ??__ERIL_PDSM_PD_DLD_DATA@@YAXXZ 00044660 f   stdafx.obj
 0001:00033690       ??__ERIL_PDSM_PD_DLD_DONE@@YAXXZ 00044690 f   stdafx.obj
 0001:000336c0       ??__ERIL_PDSM_PD_DLD_END@@YAXXZ 000446c0 f   stdafx.obj
 0001:000336f0       ??__ERIL_PDSM_PD_DLD_BEGIN@@YAXXZ 000446f0 f   stdafx.obj
 0001:00033720       ??__ERIL_PDSM_PA_PARAM@@YAXXZ 00044720 f   stdafx.obj
 0001:00033750       ??__ERIL_CALL_BYTE_CTR@@YAXXZ 00044750 f   stdafx.obj
 0001:00033780       ??__ERIL_CREATE_MAIN_LIST@@YAXXZ 00044780 f   stdafx.obj
 0001:000337b0       ??__ERIL_STATUS_CHANGED@@YAXXZ 000447b0 f   systemdlg.obj
 0001:000337e0       ??__ERIL_STATUS_CHANGED@@YAXXZ 000447e0 f   usernamedlg.obj
 0001:00033810       ??__EPOWER_ON@@YAXXZ       00044810 f   versioninfo.obj
 0001:00033840       ??__EPOWER_OFF@@YAXXZ      00044840 f   versioninfo.obj
 0001:00033870       ??__EIOTA_BEGIN_MESSAGE@@YAXXZ 00044870 f   versioninfo.obj
 0001:000338a0       ??__EIOTA_END_MESSAGE@@YAXXZ 000448a0 f   versioninfo.obj
 0001:000338d0       ??__EIOTA_BEGIN_ACK@@YAXXZ 000448d0 f   versioninfo.obj
 0001:00033900       ??__EIOTA_BEGIN_NACK@@YAXXZ 00044900 f   versioninfo.obj
 0001:00033930       ??__EIOTA_END_ACK@@YAXXZ   00044930 f   versioninfo.obj
 0001:00033960       ??__EIOTA_EXIT_MESSAGE@@YAXXZ 00044960 f   versioninfo.obj
 0001:00033990       ??__EIOTA_ALIVE_MESSAGE@@YAXXZ 00044990 f   versioninfo.obj
 0001:000339c0       ??__EIOTA_PING_MESSAGE@@YAXXZ 000449c0 f   versioninfo.obj
 0001:000339f0       ??__EIOTA_PING_ACK@@YAXXZ  000449f0 f   versioninfo.obj
 0001:00033a20       ??__EIOTA_CRITICAL_ERROR@@YAXXZ 00044a20 f   versioninfo.obj
 0001:00033a50       ??__EIOTA_NON_CRITICAL_ERROR@@YAXXZ 00044a50 f   versioninfo.obj
 0001:00033a80       ??__EIOTA_KILL_ME@@YAXXZ   00044a80 f   versioninfo.obj
 0001:00033ab0       ??__EIOTA_UPDATE_STATUS@@YAXXZ 00044ab0 f   versioninfo.obj
 0001:00033ae0       ??__EIOTA_DATAPORT_INUSE@@YAXXZ 00044ae0 f   versioninfo.obj
 0001:00033b10       ??__EIOTA_DONE@@YAXXZ      00044b10 f   versioninfo.obj
 0001:00033b40       ??__EIOTA_DIAL@@YAXXZ      00044b40 f   versioninfo.obj
 0001:00033b70       ??__EIOTA_1012_MIP_ERR@@YAXXZ 00044b70 f   versioninfo.obj
 0001:00033ba0       ??__EPHONEUTILS_BEGIN_MESSAGE@@YAXXZ 00044ba0 f   versioninfo.obj
 0001:00033bd0       ??__EPHONEUTILS_END_MESSAGE@@YAXXZ 00044bd0 f   versioninfo.obj
 0001:00033c00       ??__EPHONEUTILS_BEGIN_ACK@@YAXXZ 00044c00 f   versioninfo.obj
 0001:00033c30       ??__EPHONEUTILS_BEGIN_NACK@@YAXXZ 00044c30 f   versioninfo.obj
 0001:00033c60       ??__EPHONEUTILS_END_ACK@@YAXXZ 00044c60 f   versioninfo.obj
 0001:00033c90       ??__EPHONEUTILS_EXIT_MESSAGE@@YAXXZ 00044c90 f   versioninfo.obj
 0001:00033cc0       ??__EPHONEUTILS_ALIVE_MESSAGE@@YAXXZ 00044cc0 f   versioninfo.obj
 0001:00033cf0       ??__EPHONEUTILS_PING_MESSAGE@@YAXXZ 00044cf0 f   versioninfo.obj
 0001:00033d20       ??__EPHONEUTILS_PING_ACK@@YAXXZ 00044d20 f   versioninfo.obj
 0001:00033d50       ??__EAW_BEGIN_MESSAGE@@YAXXZ 00044d50 f   versioninfo.obj
 0001:00033d80       ??__EAW_END_MESSAGE@@YAXXZ 00044d80 f   versioninfo.obj
 0001:00033db0       ??__EAW_BEGIN_ACK@@YAXXZ   00044db0 f   versioninfo.obj
 0001:00033de0       ??__EAW_BEGIN_NACK@@YAXXZ  00044de0 f   versioninfo.obj
 0001:00033e10       ??__EAW_END_ACK@@YAXXZ     00044e10 f   versioninfo.obj
 0001:00033e40       ??__EAW_EXIT_MESSAGE@@YAXXZ 00044e40 f   versioninfo.obj
 0001:00033e70       ??__EAW_ALIVE_MESSAGE@@YAXXZ 00044e70 f   versioninfo.obj
 0001:00033ea0       ??__EAW_PING_MESSAGE@@YAXXZ 00044ea0 f   versioninfo.obj
 0001:00033ed0       ??__EAW_PING_ACK@@YAXXZ    00044ed0 f   versioninfo.obj
 0001:00033f00       ??__EUPDATER_BEGIN@@YAXXZ  00044f00 f   versioninfo.obj
 0001:00033f30       ??__EUPDATER_END@@YAXXZ    00044f30 f   versioninfo.obj
 0001:00033f60       ??__EUPDATER_BEGIN_ACK@@YAXXZ 00044f60 f   versioninfo.obj
 0001:00033f90       ??__EUPDATER_BEGIN_NACK@@YAXXZ 00044f90 f   versioninfo.obj
 0001:00033fc0       ??__EUPDATER_END_ACK@@YAXXZ 00044fc0 f   versioninfo.obj
 0001:00033ff0       ??__EUPDATER_END_NACK@@YAXXZ 00044ff0 f   versioninfo.obj
 0001:00034020       ??__ERIL_STATUS_CHANGED@@YAXXZ 00045020 f   versioninfo.obj
 0001:00034050       ??__ERIL_DBG_NOTIFY@@YAXXZ 00045050 f   versioninfo.obj
 0001:00034080       ??__ERIL_TECHHDR_NOTIFY@@YAXXZ 00045080 f   versioninfo.obj
 0001:000340b0       ??__ERIL_IOTA_STATUS_CHANGED@@YAXXZ 000450b0 f   versioninfo.obj
 0001:000340e0       ??__ERIL_IOTA_WAP_URI@@YAXXZ 000450e0 f   versioninfo.obj
 0001:00034110       ??__ERIL_PDSM_PD_DATA@@YAXXZ 00045110 f   versioninfo.obj
 0001:00034140       ??__ERIL_PDSM_PD_DONE@@YAXXZ 00045140 f   versioninfo.obj
 0001:00034170       ??__ERIL_PDSM_PD_END@@YAXXZ 00045170 f   versioninfo.obj
 0001:000341a0       ??__ERIL_PDSM_PD_BEGIN@@YAXXZ 000451a0 f   versioninfo.obj
 0001:000341d0       ??__ERIL_PDSM_PD_UPDATE_FAILURE@@YAXXZ 000451d0 f   versioninfo.obj
 0001:00034200       ??__ERIL_PDSM_PD_DLD_DATA@@YAXXZ 00045200 f   versioninfo.obj
 0001:00034230       ??__ERIL_PDSM_PD_DLD_DONE@@YAXXZ 00045230 f   versioninfo.obj
 0001:00034260       ??__ERIL_PDSM_PD_DLD_END@@YAXXZ 00045260 f   versioninfo.obj
 0001:00034290       ??__ERIL_PDSM_PD_DLD_BEGIN@@YAXXZ 00045290 f   versioninfo.obj
 0001:000342c0       ??__ERIL_PDSM_PA_PARAM@@YAXXZ 000452c0 f   versioninfo.obj
 0001:000342f0       ??__ERIL_CALL_BYTE_CTR@@YAXXZ 000452f0 f   versioninfo.obj
 0001:00034320       ??__ERIL_CREATE_MAIN_LIST@@YAXXZ 00045320 f   versioninfo.obj
 0001:00034350       ??__EPHONEUTILS_END_MESSAGE@@YAXXZ 00045350 f   vocoderdlg.obj
 0001:00034380       ??__ERIL_STATUS_CHANGED@@YAXXZ 00045380 f   vocoderdlg.obj
